:020000040000fa
:080000000001040000000000f3
:020000040000fa
:04000800e20400000e
:020000040000fa
:04000c0024050000c7
:020000040000fa
:040010006405000083
:020000040000fa
:0400140002050000e1
:020000040000fa
:04001800440500009b
:020000040000fa
:04001c002e060000ac
:020000040000fa
:040020002e060000a8
:020000040000fa
:040024002e060000a4
:020000040000fa
:040028002e060000a0
:020000040000fa
:04002c002e0600009c
:020000040000fa
:040030002e06000098
:020000040000fa
:04003400be05000005
:020000040000fa
:040038002e06000090
:020000040000fa
:04003c002e0600008c
:020000040000fa
:040040002e06000088
:020000040000fa
:040044002e06000084
:020000040000fa
:040048002e06000080
:020000040000fa
:04004c002e0600007c
:020000040000fa
:040050002e06000078
:020000040000fa
:04005400f4050000af
:020000040000fa
:040058002e06000070
:020000040000fa
:04005c002e0600006c
:020000040000fa
:040060002e06000068
:020000040000fa
:040064002e06000064
:020000040000fa
:040068002e06000060
:020000040000fa
:04006c005c02000032
:020000040000fa
:040070002e06000058
:020000040000fa
:0400740084050000ff
:020000040000fa
:040078002e06000050
:020000040000fa
:04007c002e0600004c
:020000040000fa
:040080002e06000048
:020000040000fa
:040084002e06000044
:020000040000fa
:040088002e06000040
:020000040000fa
:04008c002e0600003c
:020000040000fa
:040090002e06000038
:020000040000fa
:040094002e06000034
:020000040000fa
:040098002e06000030
:020000040000fa
:04009c002e0600002c
:020000040000fa
:0400a0002e06000028
:020000040000fa
:0400a4002e06000024
:020000040000fa
:0400a8002e06000020
:020000040000fa
:0400ac002e0600001c
:020000040000fa
:0400b0002e06000018
:020000040000fa
:0400b4002e06000014
:020000040000fa
:0400b8002e06000010
:020000040000fa
:0400bc002e0600000c
:020000040000fa
:0400c0002e06000008
:020000040000fa
:0400c4002e06000004
:020000040000fa
:0400c8002e06000000
:020000040000fa
:0400cc002e060000fc
:020000040000fa
:0400d0002e060000f8
:020000040000fa
:0400d4002e060000f4
:020000040000fa
:0400d8002e060000f0
:020000040000fa
:0400dc002e060000ec
:020000040000fa
:0400e0002e060000e8
:020000040000fa
:0400e4002e060000e4
:020000040000fa
:0400e8002e060000e0
:020000040000fa
:0400ec002e060000dc
:020000040000fa
:0400f0002e060000d8
:020000040000fa
:0400f4002e060000d4
:020000040000fa
:0400f8002e060000d0
:020000040000fa
:0400fc002e060000cc
:020000040000fa
:040100002e060000c7
:020000040000fa
:040104002e060000c3
:020000040000fa
:040108002e060000bf
:020000040000fa
:04010c002e060000bb
:020000040000fa
:040110002e060000b7
:020000040000fa
:040114002e060000b3
:020000040000fa
:040118002e060000af
:020000040000fa
:04011c002e060000ab
:020000040000fa
:040120002e060000a7
:020000040000fa
:040124002e060000a3
:020000040000fa
:040128002e0600009f
:020000040000fa
:04012c002e0600009b
:020000040000fa
:040130002e06000097
:020000040000fa
:040134002e06000093
:020000040000fa
:040138002e0600008f
:020000040000fa
:04013c002e0600008b
:020000040000fa
:040140002e06000087
:020000040000fa
:040144002e06000083
:020000040000fa
:040148002e0600007f
:020000040000fa
:04014c002e0600007b
:020000040000fa
:040150002e06000077
:020000040000fa
:040154002e06000073
:020000040000fa
:040158002e0600006f
:020000040000fa
:04015c002e0600006b
:020000040000fa
:040160002e06000067
:020000040000fa
:040164002e06000063
:020000040000fa
:040168002e0600005f
:020000040000fa
:04016c002e0600005b
:020000040000fa
:040170002e06000057
:020000040000fa
:040174002e06000053
:020000040000fa
:040178002e0600004f
:020000040000fa
:04017c002e0600004b
:020000040000fa
:040180002e06000047
:020000040000fa
:040184002e06000043
:020000040000fa
:040188002e0600003f
:020000040000fa
:04018c002e0600003b
:020000040000fa
:040190002e06000037
:020000040000fa
:040194002e06000033
:020000040000fa
:040198002e0600002f
:020000040000fa
:04019c002e0600002b
:020000040000fa
:0401a0002e06000027
:020000040000fa
:0401a4002e06000023
:020000040000fa
:0401a8002e0600001f
:020000040000fa
:0401ac002e0600001b
:020000040000fa
:0401b0002e06000017
:020000040000fa
:0401b4002e06000013
:020000040000fa
:0401b8002e0600000f
:020000040000fa
:0401bc002e0600000b
:020000040000fa
:0401c0002e06000007
:020000040000fa
:0401c4002e06000003
:020000040000fa
:0401c8002e060000ff
:020000040000fa
:0401cc002e060000fb
:020000040000fa
:0401d0002e060000f7
:020000040000fa
:0401d4002e060000f3
:020000040000fa
:0401d8002e060000ef
:020000040000fa
:0401dc002e060000eb
:020000040000fa
:0401e0002e060000e7
:020000040000fa
:0401e4002e060000e3
:020000040000fa
:0401e8002e060000df
:020000040000fa
:0401ec002e060000db
:020000040000fa
:0401f0002e060000d7
:020000040000fa
:0401f4002e060000d3
:020000040000fa
:0401f8002e060000cf
:020000040000fa
:0401fc002e060000cb
:020000040000fa
:10020000ef1721000e7f24000e018800000000007f
:10021000000020000000e000020032000001200089
:100220002002880014000700c40207000000e0005c
:1002300003003a00c03e2c000100200002003700fd
:100240000000200001002000810f7000010032003a
:1002500014000700000020000000e000020032004f
:100260000000020000000000e0ac020000000000fe
:100270000040da000000fe004440a900204a2100ae
:100280000000e00003003200002020009001880000
:100290004440a800000006008a1f78008b1f7800e9
:1002a00000000600a1028800800478000000eb0036
:1002b0001f003700e284440054a0b4009905ba003e
:1002c000e284440054a0b4009906ba00e2844400d9
:1002d00054a0b4000006eb00476fde00fd07b2003b
:1002e000ae018800636ce10003003a00eaff0700fa
:1002f0000000eb000e003700606ce10008003a00df
:10030000004deb000a05e800020039003420ec0043
:100310000af0a0008b05e900f9ff3e000400370059
:100320006168e100010032000086eb000b0007006d
:1003300019c7ba001905ba000e04e00003003a001c
:100340000a00e000dbff3a0000000600fe07b200f2
:10035000ae0288008a047800f5ff37000cd0a300b5
:10036000e20f4d001c00390089027800354dba00bb
:100370000a05e800020039003420ec000af0a00071
:100380008b05e9000f003200254dba000a05e80090
:10039000020039003420ec000af0a0008b05e900cf
:1003a000080032000c00e0000600320015cdba0053
:1003b0000a05e800020039003420ec000af0a00031
:1003c0008b05e9008984e80054a0b4000b00e0002c
:1003d000e2ff3a00000006009902ba00055d7800cd
:1003e0008b05e900f7ff3200c82ade00055d7800c2
:1003f0008b05e900f3ff32000c00e000f1ff320052
:1004000019ddba00eeff370052ba04000000000008
:10041000c6ba040000000000f2aa040000000000b8
:100420001acb0400000000003aca040000000000db
:1004300066aa04000000000050aa040000000000aa
:100440001eaa04000000000066ab040000000000cb
:100450004aaa040000000000c0c20400000000001e
:1004600022c204000000000066c204000000000078
:10047000d2c304000000000078c3040000000000a4
:1004800028a7040000000000caa704000000000024
:1004900010a70400000000001ca7040000000000da
:1004a000d81a040000000000ae160400000000008e
:1004b00024120400000000003600f800809fbe00f7
:1004c000829fbe00849fbe00869fbe000000fa008f
:1004d0008a20a900f124800000082000008060002c
:1004e0000000e000090032009ee4a9000828ef00a7
:1004f0007040800064004000100078008000eb0035
:10050000010878000e28ef002701370040408000e6
:100510008000eb00b200200003002000820f50009a
:10052000838f580014013e00006001000b0037006b
:100530004700370087003700b00037000b01370055
:10054000de003700f100370008013700f300370004
:1005500009013700420037006000370000802000aa
:100560006400400010007800620060000000e000bd
:100570000c013a00008020000080e80010007800a4
:1005800070408800008020000080e80010007800a3
:10059000104078000ae8b700008020000080e800e2
:1005a000100078000080e8001000780060408800ab
:1005b000008020000080e80010007800e600400085
:1005c000008020000080e800010878000080200002
:1005d0000080e80090007800e0152100808f500036
:1005e00004003a0000802000811521000080e8000e
:1005f0000108780000802000e400400091007800ad
:100600000100a10064004000010878000080200083
:100610000080e80090007800008020001000780042
:10062000808f500006003a0000802000e400400067
:10063000910078000110a0006400400001087800db
:100640009a04a8002000200040408800d60037000f
:100650009a24a8002000200040408800d2003700e3
:10066000f124800000002800008060000000e0000d
:100670000a00320000802000660040001040780030
:100680008040e800008020006600400001487800bb
:1006900040002000845e0700c300370080408000d7
:1006a0008000d100f00f200000806000b02488009e
:1006b0008040800061006000004078000004e0009d
:1006c00003003200b000200040408800b600370030
:1006d0003000200040408800b3003700f124800043
:1006e00000002800008060000000e0000a003200e6
:1006f0000080200066004000104078008040e80044
:100700000080200066004000014878004000200082
:10071000655e0700a40037009a24a800804080008e
:100720004800de00e6006000000f200001007000bd
:1007300080408800804080000000a0008040880049
:1007400010c0b30012e8b70020002000404088002d
:100750009500370012c8bf00e14f50000c00320076
:100760006040800010007800804088006040800079
:100770006400400010007800a040880060408000c5
:100780000080e8001040780016e8b700010037004c
:100790001268ef0081408000f00f2000808f500031
:1007a00009003600804080004800de00e60060005e
:1007b000000f200001007000b0248800a00020007d
:1007c000404088007800370080408000b0248800d6
:1007d0008040800061006000004078000004e0007c
:1007e0000300320050002000404088006e003700b7
:1007f00030002000404088006b003700f12480006a
:1008000000002800008060000000e0000b003200c3
:100810000080200066004000104078008040e80022
:100820000080200066004000014878009fe4a90095
:10083000500020001c5e07005b00370016c8bf0098
:100840008080fb008100e900cf08de008140780055
:100850000040e90016e8b7000104e0001000320093
:100860006040800066004000604088000ac8bf0009
:100870000040e9000ae8b7000ac8bf000004e00031
:1008800003003a0020002000075e07004600370002
:100890009a24a80020002000404088004200370031
:1008a000a0408000904078008180fb00b124880047
:1008b0000000e800a04088003b003700f1248000e1
:1008c00000002800008060000000e0000b00320003
:1008d0000080200066004000104078008040e80062
:1008e00000802000660040000148780040002000a1
:1008f000ed5d07009fe4a9002b0037009a64a80073
:100900008000200040408800270037008000200041
:10091000404088009a64a80023003700a04080006f
:10092000a124800081407800014878000000e800a0
:10093000a040880016c8bf000040e90016e8b700d4
:1009400016c8bf000004e000040032009aa4a90009
:100950006000200040408800020037009aa4a800f0
:10096000c05d07009a84a8000f0037002000200017
:10097000cd5d07000c0037000080200066004000bd
:10098000104078008040e8000080200066004000b1
:100990000148780060002000c35d070000000000ef
:1009a00001003700000000000080fa004f03be0085
:1009b0004f02be004f01be004f00be003600f900de
:1009c000004006003600f800809fbe00829fbe00f7
:1009d000849fbe00869fbe000000fa008020a90010
:1009e0000000eb003c6507000080fa004f03be00ea
:1009f0004f02be004f01be004f00be003600f9009e
:100a0000004006003600f800809fbe00829fbe00b6
:100a1000849fbe00869fbe000000fa003365070079
:100a20008040a900100020002b6507000080fa001c
:100a30004f03be004f02be004f01be004f00be007c
:100a40003600f900004006003600f800809fbe0026
:100a5000829fbe00849fbe00869fbe000000fa00f9
:100a60008060a900200020001b6507000080fa00bc
:100a70004f03be004f02be004f01be004f00be003c
:100a80003600f900004006003600f800809fbe00e6
:100a9000829fbe00849fbe00869fbe000000fa00b9
:100aa0008080a900300020000b6507000080fa005c
:100ab0004f03be004f02be004f01be004f00be00fc
:100ac0003600f900004006003600f800809fbe00a6
:100ad000829fbe00849fbe00869fbe000000fa0079
:100ae0008600a90070002000fb6407000080fa0067
:100af0004f03be004f02be004f01be004f00be00bc
:100b00003600f900004006003600f800809fbe0065
:100b1000829fbe00849fbe00869fbe000000fa0038
:100b200050048000680060000000e0000c0032000b
:100b30002134800000082000008060000000e000f8
:100b400006003200104380000000e0000200320086
:100b5000104380000000010084e6a9008a60a9001b
:100b60000080fa004f03be004f02be004f01be00de
:100b70004f00be003600f900004006003600f800c5
:100b8000809fbe00829fbe00849fbe00869fbe00e5
:100b90000000fa00204380000000e0000200320064
:100ba0002043800000000100b017210010407800b1
:100bb0008040e800b017210001487800a01721000c
:100bc00011c0b300014878008860a9000080fa00d5
:100bd0004f03be004f02be004f01be004f00be00db
:100be0003600f900004006003600f800809fbe0085
:100bf000829fbe00849fbe00869fbe000200fa0056
:100c00008960a900b86107000004e0000c00320010
:100c10008e007800a08e2000985907000000e000a8
:100c2000070032009e007800f01c80000040780031
:100c30008048780011002000a08e2000ec590700a9
:100c40000080fa004f03be004f02be004f01be00fd
:100c50004f00be003600f900004006000040da00f8
:100c60000000fe00ec8747008e1f78006c8757005d
:100c700044002000041f7800000f78006c875700a4
:100c800002afbe00e1bf9f006c805700120c07004e
:100c90001e00be004f077800cf00b1000000060024
:100ca000ec8747008e1f780011002000a1bf9f0035
:100cb0006c875700002f78006c805700080c0700e5
:100cc0001e0078004f077800cf00b100000006003a
:100cd0000800fa008e81e80080097800640047006f
:100ce00001087800660047000208780066004700a7
:100cf000100f78000a0037006400470010007800e9
:100d000010407800e4004700910078000101e800fd
:100d1000e400470082087800676107001e0fe900c1
:100d20001e0078000000e000f3ff3a006600470074
:100d3000100078000080fa000000060000000500a6
:100d40001400200010043700f4ff2f000e043700b9
:100d50000001be00a20007000470a70003f0a1007c
:100d60006509b100160032000d0035006828e10069
:100d700006003500f0ff2f00f1ff27000300e00020
:100d800013003b00010028000000050000004000a7
:100d9000818048008502e900fcff3a000800370026
:100da000f88f420002003c008000eb0000000500cc
:100db0008100d1000080d3008502e800fcff3a00ea
:100dc0000300e00002003b0060001000e08018001b
:100dd000000006000001be00810007000470a700ab
:100de00003f0a10003f8a30013003a006509b10065
:100df00010003200090035006928e10002003500ca
:100e0000010028000000050000004000818048002b
:100e10008502e900fcff3a0000000600f88f42005e
:100e2000050035008100d1000080d3008502e80074
:100e3000fcff3a00000006008000eb000000050007
:100e4000881f7800030478000300e00007003d00dd
:100e500060001000e080180060011900e0811900b6
:100e600002003b0001f02d000300370007000700df
:100e700008f0a70001f0a0004f0478000000060071
:100e80004f89de0082017800edff3700889fbe00a9
:100e90008a9fbe000082700004027100048271000b
:100ea000260032000004be000200be006011b8003f
:100eb0006b092000950220000182cf000a00390052
:100ec0000541b1000082cf00070039000541b100a3
:100ed0000982cf00040039000541b1000882cf002b
:100ee000010039000541b1000542520012003200f4
:100ef0000a003b0082817100610164008100d10021
:100f00000080d3008984d3000884d3008b05e800d7
:100f10000442e800f7ff3a000700370008044400e5
:100f200089844c0000004800818048008b05e9005e
:100f30000442e900f9ff3a00030007004f05be0034
:100f40004f04be00000006008100200061805500b3
:100f50000b003d000b00200061fe2f000100e100ae
:100f60001d00340082817100610164008904d10098
:100f70000884d3000000e800faff3a007100200066
:100f8000610064000300700002006000090032008c
:100f900061044400e0844c000988a500050032008b
:100fa0008b05e8006808e10002003a008904d100de
:100fb0000884d300f20f20000258e10005003d0034
:100fc000c75ddd00f907b200898075000800780070
:100fd000000006000bf827008b00780000000500d9
:100fe000c70ade00f107b200f50fb20008003200b8
:100ff000e1cf4200020032000170a0002400050091
:10100000810f700001003200040805004400050053
:10101000810f700002003a00140005008502e9000b
:101020000000400081c04800fcff3b000170a000b0
:101030002400050007f82700078361000638e10057
:1010400004003a00f70720008783610087037100de
:1010500001003a0003f0a200889fbe008a9fbe00f4
:101060008c9fbe00470ade000480a100c71ade0084
:101070000580a100070028000785600087856100c2
:10108000f70f20000720e1009e0032000728e10052
:101090009c003200010678000400e000b400320039
:1010a000f7072000878060000170a0000500e000c5
:1010b000c0003200f7072000878161000370a000a4
:1010c000050652000f003a000b50e1000b00320001
:1010d0000308e10002003a000200e1007e00320055
:1010e0000204500083845800040031000001fd0018
:1010f0008101fd008402fd008a05fd006044b80006
:10110000210037000520e10005003d000001fd0041
:101110008101fd008402fd008a05fd0005065200e4
:101120007a60e100050035000170a1004722dd0072
:10113000848070008a807000630037006044b800cb
:10114000ef02660007ff2f00070666000500e000bb
:1011500006003400f08312008714dd000511de0064
:10116000071bdd00060171008519de007060e100db
:101170000500350009047800820478000301780036
:101180008001eb00700656000b50e10003003a00ae
:10119000020040008380480004003700600414000f
:1011a000e0841c0002005800838058000188a300de
:1011b000060032008100d1000080d3008984d30072
:1011c0000884d3000402e800270037000178a30058
:1011d00025003a000100e000030032008186cf00c4
:1011e000698656000a0037008c0020000000e000ed
:1011f00004003a0009007800880478000004eb003d
:10120000700252008086cf000d0646000c06e900f1
:101210007060e10006003500800078000900780069
:10122000880478000004eb0070065600700252003b
:101230000c00e0000c0034008c08dd00f003160008
:101240000703de00868070000c00dd00074bde0027
:10125000060070008c4cdd000743de0086847400bd
:101260000c44dd000c0252006120e100200035003a
:10127000610160000700280087816400f7ff2700f4
:1012800087836400070374000300e0000600320057
:1012900082037300040032000000e800e080480090
:1012a0000188a3000e003a00f70f20000720e1009c
:1012b0004a003d000170a1004722dd00810072005c
:1012c0008a8070000000be004f06be004f05be00c1
:1012d0004f04be00000006006000b800faff3700af
:1012e0008100d1000080d3000402e800eeff370047
:1012f0000401780089017400a10107008a80700050
:10130000f1ff3700f7010700070278000001fd0038
:101310008101fd00f3010700870278008503720058
:101320000778a300040032000001fd008101fd00e8
:1013300006020700e4ff3700850362000768a30088
:10134000080032000b50e10003003200f0ff2f00d4
:10135000f1ff2700dcff37000001fd008101fd00e7
:10136000d9ff37000468a300d7ff3200faff370027
:10137000f8ff2700888360000b003a000000e000bf
:1013800009003a0083036400828373000200320084
:101390000200be00ccff37000b50e100ceff3a0048
:1013a0000200be00c8ff3700140020008100640066
:1013b0003eff3700f8ff27008883610004003a00f1
:1013c0000200e00002003a008c007800beff370007
:1013d000150020008301640039ff370001f8270061
:1013e0000000200081007500b7ff3700889fbe0015
:1013f0008a9fbe008c9fbe001b0020000202be0020
:101400000586680006002800060666004709de001b
:10141000f20fb200820032000243e8008000320086
:10142000c729de00f30fb2007d0032000343e8005d
:101430007b003200f107b2000170a000f507b20096
:101440000570a000c708dd004903de00868070003b
:101450004700dd00c72add004923de0086827200d6
:101460004722dd0003055100040350008583580026
:101470000300310000004000818048000a05e900b7
:101480008c1f78008a9fbe000400500085805800a1
:101490000402420085824a0000004000818048002a
:1014a0000005eb000004be006033b8000406be0077
:1014b0000d48e10056003100110009004dccd80064
:1014c0000c01b8000d02b8008481410060824a001e
:1014d0008283530003045c0084845c0060055d002b
:1014e0000a00e00025003a00800578000d40e10088
:1014f00049003100880078000700780011000900d9
:101500004d88d8000c01b8000d02b800848141005c
:1015100060824a006003110083835b0004045c0066
:10152000e0845c000900e00021003a004f01be00a9
:101530000300e0002b003200e301600007067300a7
:101540008c81710001003200640070004200de00f6
:101550004e5edd000c007000c258de0001e0a0000d
:1015600083010700cf017800818071004f06be0023
:101570004f05be004f04be00000006008c834300f0
:101580000d044c00e0844c0060054d000000e900b3
:101590000a00e000d4ff32008c8343000d044c00ad
:1015a000e0844c0060054d000000e900ceff3700ec
:1015b0000c0343008d834b0060044c00e0844c001e
:1015c0000000e9000900e000d8ff32000c034300ee
:1015d0008d834b0060044c00e0844c000000e90067
:1015e000d2ff37004200de004e5edd000c007000ce
:1015f000c258de0001e0a000cf0178000300e00047
:10160000daff320060001000e0801800d7ff3700da
:10161000f0ff2f00aaff3700f0ff2f00b9ff3700bf
:101620000404be002f010700870678000004fd00b7
:101630008104fd002b010700078366000678a300e4
:10164000030032000960a7000800be002c0037002c
:101650000d78a300020032000800be002800370009
:101660000778a30026003a0001f0a10009f0a100cc
:101670000668a30003003200f1ff2700f0ff2f00ef
:10168000baff37000d68a300030032000800be0057
:101690008c807000b5ff37000768a30007003a0090
:1016a0000648a30003003200f1ff2700f0ff2f00df
:1016b000aeff37000d48a300030032006000b80001
:1016c0008c807000a9ff37000748a3000400320097
:1016d00001f82700000020008c807000a3ff370075
:1016e000760107000004fd008104fd00020578007a
:1016f000720107000802be008a01780059ff370016
:101700000160a000120220004243880097ff3700ca
:101710000100e000120032000500e000100032007d
:10172000889fbe008a9fbe008c9fbe000006eb0013
:1017300001f8a3000300320060001000e0801800f0
:101740000cf0a00005f8a3000300320060021200b4
:10175000e0821a000cf0a2008005eb0041ff370088
:101760006000b8000200050003836800070028003d
:1017700007036300470ade000480a100c71ade00e9
:101780000580a100f70f20000720e1004200320091
:101790000728e10040003200889fbe008a9fbe00fb
:1017a0008c1f7800f107b200f307b2000400e000dc
:1017b000640032000170a0000500e0006800320003
:1017c0000370a00085054200eb07b1000204b800d9
:1017d0000302b8008484440060854a00020ab8000d
:1017e000848444000a854a00030ab80004054500c1
:1017f000040033000804d0008984d2000a85d20096
:101800008b05e9006158e1003d0035000210200021
:10181000090161000308200089816100f7072000a9
:101820008783640008867300c84cde00c853dd005f
:10183000878474004855de000300e0000600320093
:1018400082037600040032008904e80060054d0040
:101850000a88a3000c003a00f70f20000758e100a7
:1018600044003d000a70a100c75ddd000a857500d7
:101870008a007300090078004f0678004f05be000b
:101880004f04be00000006000a05d1008984d30081
:101890008b05e800f0ff3700881f78000604780009
:1018a00090000700070278000001fd008101fd00a3
:1018b0008c00070087027800850372000778a30078
:1018c000050032000001fd008101fd009f000700be
:1018d0004f04780000000600850372000748a3004b
:1018e00003003200f0ff2f00f1ff2700f8ff370060
:1018f0000000200001f8270088807000f4ff370006
:10190000880178004848dd00808171004848de0089
:10191000c850dd0001007000c850de0006047800e9
:101920000b0178001600070088807000d2ff370096
:101930000500e00005003200170020003a00070013
:101940009dff370081037000f9ff3a0086007800a0
:101950004f0678004f05be004f04be000000050092
:1019600083037100f9ff3200270020002e000700da
:1019700094ff370001f8270086807000f4ff3700dd
:101980000100e00026003200610111007810e10042
:1019900023003c006022b8007010e1000400350014
:1019a00080027800010078008000eb007001510097
:1019b0000200e0000900340070031100062add0077
:1019c000822ade008603dd00878272000200de00cc
:1019d000860bdd00070070008208de008481710044
:1019e000f4ff270004826200848171000400280053
:1019f000848262006102600005f0a600000006001b
:101a000004827100070032000000e800e080480016
:101a1000000006000002be006000b800efff3700c3
:101a20006000b80000000600889fbe000004eb00c4
:101a30006138e10016003a000100e00008003a00b9
:101a4000c800de004800dd00880020000100e00042
:101a500003003a00c800de004800dd0068044400ce
:101a60008184cf00e9845400060034008908dd0039
:101a7000f08314008703de00878070000900dd001a
:101a800009044400610214004f04be000000060077
:101a90000300e00008003a00c811de004811dd0034
:101aa000880020000300e00003003a00c811de00b7
:101ab0004811dd00680444008384cf00e9845400a9
:101ac000060034008919dd00f08314008713de005e
:101ad000878171000911dd0009044400e10214004e
:101ae000e9ff37002700200001f0a70017002000c1
:101af000470bde00f60fb200040032000643e80098
:101b00000a0032004702b30000000600010378001b
:101b1000f607b2000603700002003a000703b300a4
:101b2000000006008702b3000000060001037800f1
:101b3000f607b20006037000020032000770a00032
:101b4000000006000760a000000006000478a30063
:101b5000040032000578a300030032000168a300ee
:101b600001003a000200be000160a0000000060073
:101b700081017000270032008002eb0001f8a30011
:101b80000300320060001000e08018001500200003
:101b9000f40720000202420020003400f703200076
:101ba0008703600006042000000363000208200091
:101bb000000161004700de00c909dd0000807100fe
:101bc000c708de000600e00008003200870371004d
:101bd000060032001000b0000180b0000188a300b0
:101be00002003200c108de000402e800f107b20082
:101bf000f30f20000320e10003003d004722dd0039
:101c0000810072002900370001f827000000eb0076
:101c1000260037006000b8000000060068021200cd
:101c20007f20e100020034006000b8001f00370090
:101c30006011b8007020e1000400350080017800d8
:101c4000010078008000eb00700252000400e00008
:101c500009003400f00312000719dd008419de00ca
:101c60000703dd00868171000400de00070bdd0044
:101c7000060070008408de00f7ff270083836300fe
:101c80008703710006002800030363000700320089
:101c90000700e00003003a00610160000281730068
:101ca000020032001000b0000180b0000500a60064
:101cb0000000060001f0a000000006004f0ade0050
:101cc0004709de00f107b200f20fb2000b0032004c
:101cd000f207b1000170a000c708dd00c901de00f5
:101ce000838070004700dd000400a60000000600ad
:101cf00060001000e080180000000600810f7000f6
:101d000001003a00000006008182cf000500e000db
:101d100010003e008082cf00ee8242007028e10079
:101d20000400390007003e00800078000000eb004e
:101d30000e003700708312008600de000500dd0013
:101d40000a003700708352008600dd000000eb00bf
:101d500006003700e28252008508dd007083120021
:101d60000603de00868070000500dd007507b00008
:101d70000501ea000400a600000006006000100053
:101d8000e080180000000600889fbe008a9fbe0009
:101d9000841f7800170007004f00780011003300ff
:101da000f0ff2f00838f6c0006003b0004056500e8
:101db0000a00a7000800370009f0a6001000200064
:101dc00008003700820f5400838f5c000300390045
:101dd0001000200001003e000000200009f0a700d4
:101de0000000ea004f05be004f04be000000e00006
:101df000000006000004be0079fc07000003be00de
:101e00000405be000200be0075fc0700844f75008b
:101e100000000600889fbe008a9fbe00300442007a
:101e2000b0844a0030054b0090854b006000b10043
:101e30000898be000a90be000440e10005c8e10019
:101e400006d0e10007d8e100020031006800400040
:101e50001008e8004f05be004f04be000000060059
:101e6000889fbe008a9fbe003004be002005be00d1
:101e70000418540005985c0006185d0007985d0082
:101e8000110020000440e10005c8e10006d0e10097
:101e900007d8e100010039008000eb001088100035
:101ea0004f05be004f04be0000000600f487470047
:101eb000889fbe008a9fbe008c9fbe008e1f780048
:101ec000d0b79f00e1b79f00f2b79f0083bf9f008c
:101ed0000605be000404be00cfae97000000eb0074
:101ee000c0b79f00b0b79f00a0b79f0090b79f00fa
:101ef00080b79f00000678004fb0970000014000b7
:101f00000000e00006003d003c0007000f0747000e
:101f1000450007000f004000beff07000500370026
:101f2000360007000f0747003f0007000f00400082
:101f3000cbff07004fb797000e00e0000c00350004
:101f40005fb29700efb297007fb397008fbb970007
:101f500010002000010020006011b8000002720093
:101f60008182720002037300838373001c000700e8
:101f70000c06e80001042000810f5600deff3a0045
:101f80000e00e00005003d000802be000a03be008e
:101f900000fe2f000f0040009eff07000d00e00034
:101fa00005003a000fb297009fb297002fb3970039
:101fb000bfb397000a0007005fb09700efb097002b
:101fc0007fb197008fb997004f0778004f06be008a
:101fd0004f05be004f04be004f01b10000000600d7
:101fe000010007000000060094b79f00a5b79f00fe
:101ff000b6b79f00c7b79f00000006009fb09700cc
:102000004f08de0002017000a2b79f000fb09700da
:102010004f01de00818040008100710091b79f0078
:102020000efe2f0000000600de0078004f09de00e3
:10203000000040000000710080b79f006fa897006b
:102040004f01de0081804000010f71000e0007008b
:102050004f3ade000000400004007000e0af9f0037
:10206000090007000402420085824a0006034b0073
:1020700087834b00dcff07000802be000a03be0096
:1020800000fe2f00000006001fb29700afb29700bd
:102090003fb39700cfb3970000000600881f780079
:1020a00018002000881f780080ff07008f87e90054
:1020b0004f04780000000600801feb007bff070044
:1020c0008f87e90000000600889fbe008a9fbe003f
:1020d000e00f5000e08f5800e00f5900e08f5900ea
:1020e0000c003d006044b8006055b800000054008a
:1020f00081805c0002015d0083815d00180020008a
:102100001500070008003d00180007000004eb0060
:10211000050037000004eb000f00070002003d003f
:102120001200070018002000dcff07000800e00094
:10213000060032006022b8006033b8000000520090
:1021400081805a0002015b0083815b004f05be0065
:102150004f04be0000000600e00f5200e08f5a005e
:10216000e00f5b00e08f5b00000006006044b800f9
:102170006055b8000402540085825c0006035d00cf
:1021800087835d0000000600889fbe008a9fbe0016
:102190008c1f7800e00f5000e08f5800e00f5900ce
:1021a000e08f59000d003d006044b8006055b80054
:1021b0000000540081805c0002015d0083815d00ad
:1021c0001c0020000820e10009a8e1000ab0e1009d
:1021d0000bb8e1000d003d00080037000006eb00e1
:1021e000e00f5200e08f5a00e00f5b00e08f5b00d1
:1021f00006003d006044b8006055b8000402540079
:1022000085825c0006035d0087835d00aaff0700ee
:102210000c00e000060032006022b8006033b80015
:102220000000520081805a0002015b0083815b0044
:102230004f0678004f05be004f04be0000000600a8
:102240000000fa004fb99700e88157008a020700a2
:102250000080fa0000000600af0007000701070039
:10226000b7010700df01070039013700800178005e
:1022700002003700b15978000201e9000200e000d5
:10228000fcff3a0000000600889fbe008a9fbe0047
:10229000800478000200e0005a003200014078001b
:1022a000814c780082814400f1f99f00e20f5100d7
:1022b0005400360091449800a1449800e1f99f0031
:1022c000d1f99f00e60f51004e003600b14498004e
:1022d000c1f99f00e80f51004a0036000905ea00e5
:1022e000630565000a8444000a055100c1ff2f0000
:1022f000010565000080fb008000eb00121020004b
:10230000131020006e060700008cbe000a01440076
:1023100060b99f0071b99f00e80f55003900360081
:10232000200498003104980040049800510498005b
:1023300020b99f0031b99f0040b99f0051b99f005b
:10234000f80f55002f0036006004980071049800c3
:10235000000c9800110c9800200c9800310c98008b
:10236000400c9800510c980020b19f0031b19f00a3
:1023700040b19f0051b19f0060b19f0071b19f00bb
:1023800000b99f0011b99f00640164007801410009
:1023900002044400020555006011b8000203be00ab
:1023a0000002be000403be006022b80000007200fc
:1023b0008180720002017300838173000f00370077
:1023c00008027800009abe00029abe00009abe0081
:1023d0000292be00000c9800110c9800220c98008c
:1023e000330c9800400c9800510c9800620c980037
:1023f000730c98000a02b1000802b000ff0f5500ec
:10240000efff3e00090078004f05be004f04be00fc
:1024100000000600518180009100780096040700ba
:10242000110020000000e000050035005081800010
:1024300090007800a0002000d3040700cf00de0049
:102440000100ea0000000600000006000003210071
:1024500000000600fdff0700708188006081880091
:102460000000060080007800040037003104e0001e
:1024700002003a000000510000000600010178004f
:102480000108a300f9ff3a008101780031017800ca
:10249000f4ef2f00020242000281ea000201620012
:1024a0000408280004016100f7ff3200830078006f
:1024b000010178003104e000fdff3a000000510006
:1024c000000006008001eb000200e0001000320076
:1024d0000002780001037800b44178000304e000b2
:1024e00008003200b14278000504e0000500320027
:1024f00082034000848f53000200320085cf5100d8
:10250000f4ff32008381fb001680fb0080815100c4
:102510000300780000000600ec874700889fbe009b
:102520008a9fbe008c9fbe008e1f78000006780038
:10253000010478001807900028059000980678009c
:10254000cdb79f00b80590003202be002203be0046
:102550000400be000601be004f18de006011b80086
:102560008000eb00d0b79f00e1b79f00f2b79f005b
:1025700083bf9f00800478000900e000060032005d
:102580006000b8006011b800040250008582580055
:1025900006035900878359000e00e0000200350051
:1025a0000d10a100cdb79f000900e00005003a0022
:1025b0004fb097000028a30002003a000038a300a3
:1025c000020032008a00e900010037008a0078002a
:1025d000f8815700a200200008007800860007005c
:1025e0000900e00003003a00cfb097000128a300e3
:1025f000080032000000e90000814500b1c2b300cc
:102600000900e00001003200d1c2b30001497800a6
:10261000050037000138a300030032000000e90084
:1026200001c2b30081757800480190000201e90001
:1026300000015100808045004fb297008a01780068
:102640000c007800e30107009c0090000188a300c3
:102650000400320098009000810f500001003d00fe
:10266000010078004f0778004f06be004f05be00fe
:102670004f04be00cf00b100000006000200fa00c7
:10268000889fbe008a9fbe00000578000104780084
:102690000200780018019000a805900098007800ca
:1026a000b1bf9f00b80490000200e00002003500b6
:1026b0000110a100b1bf9f00ea81570082002000f5
:1026c0008b0078003002be002003be0008007800b6
:1026d000490007003fb99700f00061000300320095
:1026e0000000e90001c3b300817478003fb997008e
:1026f000e8006100030032000000e90001c2b300fd
:1027000081747800480190000201e9000001510045
:10271000808044003fba97008b0178000a0078005f
:10272000ac0107009a0090000188a3000400320069
:1027300098009000810f500001003d0001007800da
:102740004f05be004f04be000080fa0000000600e6
:10275000ea874700889fbe008a9fbe008e1f7800d0
:1027600000047800030078007287570084e2260096
:1027700055c72600049fbe00c3962200030f7800b1
:102780006c875700004feb0011059000a1049000ea
:10279000910578000200e000020032000207780094
:1027a00001003700728757000000e00002003a0085
:1027b0000e0078002bff07000a00e0000300350040
:1027c0008a0f5000010036000a0078000b027800e2
:1027d00089017800000178008e00780008007800f8
:1027e0007c0107004f0778004f05be004f04be0074
:1027f000af00b10000000600f4874700889fbe00cc
:102800008a9fbe008c9fbe008e1f78000605be000a
:102810000404be0081bf9f0082b79f00f3b79f00f2
:10282000b0009000e1b79f001301780092b79f00bd
:1028300090069000400690000c06e9000d00e000b4
:1028400001003d001d002000efb197000c80410009
:102850000048eb001e0020001f0037000c06e900b6
:102860000fb09700cf80de006109b900a0b79f00cc
:10287000b1b79f00c2b79f00d3b79f000203be004d
:102880000002be000800be000a01be000afe0700ea
:1028900000077800efb097000c80400003c3b3003e
:1028a000034847008d06e9000fb897000000e900d3
:1028b00080bf9f002fb29700bfb297004fb3970021
:1028c000dfb397000800be000a01be00f3fd070059
:1028d0000205be000004be000c00e0000d00320046
:1028e000e00f5400e08f5c00e00f5d00e08f5d00c2
:1028f000daff3a000d00e000d8ff3c008fb89700e7
:102900000100e000030034001fb197000218a3008b
:10291000d2ff3a000e00e00002003a00ffb197003b
:102920001340a1000c0078004f0778004f06be004e
:102930004f05be004f04be004f01b100000006006d
:102940000200fa00889fbe008a9fbe0080047800c3
:10295000010478000200780018019000280590001a
:1029600098007800b1bf9f00b80590000200e00019
:10297000020035000110a100b1bf9f00ea8157009d
:10298000a20020008a0078003002be002003be00b2
:102990000800780098ff0700480190000201e90054
:1029a00000015100808045003fba97008a017800fd
:1029b0000900780007010700990090000188a30032
:1029c0000400320098009000810f500001003d008b
:1029d000010078004f05be004f04be000080fa00e1
:1029e00000000600fa874700889fbe008a9fbe004d
:1029f0008c9fbe008e1f7800800478000104780050
:102a000082057800180190002805900018077800ca
:102a1000b80090000200e000020035000e10a10096
:102a2000010037001200200070006700e0b79f002f
:102a3000090032003b02be002b03be00e00f520033
:102a4000e08f5a00e00f5b00e08f5b000200320075
:102a50008a86e900010037008a067800e8026700ec
:102a6000f5b79f00010032008d06e9003b02be0071
:102a70002b03be00e4af9f00f5af9f0086b79f0019
:102a800097b79f00480690000c06e9000c804000b4
:102a90000048eb00efb297007fb2970089037800ff
:102aa00081047800d8af9f00020478008bbf9f009c
:102ab0008a057800034578002a0037000c06e900f3
:102ac0006fab97006f006300e90f500002003c00fd
:102ad0000003b000010037007005b0000a03fb00de
:102ae0001604b100f90f53000c003e0000037800fb
:102af0000650a0001606b100f90f530007003e0073
:102b0000b4b79f00a5b79f00c7b79f009003070009
:102b1000cfb39700afb297003fb2970080747e00aa
:102b20000804e9008d06e9006fa89700ffa8970048
:102b30000fb197009fb19700460020008301d1009c
:102b40000281d3008180d3000080d3000603e90016
:102b5000faff3a00e0af9f00f1af9f0082b79f00fd
:102b600093b79f00e10f56000f0036006fa8970043
:102b7000ffa897000fb197009fb19700e00f50009a
:102b8000e08f5800e00f5900e08f5900cbff3a006a
:102b90000800e000c9ff3c000d00e0000200340026
:102ba0000e18a300c5ff3a0089007800f4b79f0013
:102bb000870478005fac97008a4178000b057800a5
:102bc0008fbd97000500e000100032003b02be0000
:102bd0002b03be00e4af9f00f5af9f0086b79f00b8
:102be00097b79f00e00f5200e08f5a00e00f5b00a4
:102bf000e08f5b00050032000c06e90083707e0068
:102c00000c06e90000c3b30080707e00ffb297009d
:102c10000500e000030032000c06e90000c2b3002a
:102c200080707e00480190000201e9000c01510013
:102c30008c8040000e0278008a017800090078003c
:102c400064000700990090000188a300040032008e
:102c500098009000810f500001003d0001007800b5
:102c60004f0778004f06be004f05be004f04be0060
:102c7000af01b10000000600f28747008e1f780008
:102c800002027800030178000000e0000200320038
:102c90000007780001003700728757008002eb00c0
:102ca0000100e000010032008102e900708057005d
:102cb000060009000018eb007280570000a8eb0026
:102cc0002310200093bf9f00aebf9f00b1bf9f00a5
:102cd000c5bf9f000100e00004003d00b0042000db
:102ce000e08b88000080eb0005003700004feb0010
:102cf000eebf9f00debf9f0084007800a3020700a4
:102d00004f0778002f01b10000000600889fbe0029
:102d10008a1f78008004780049009000020478003f
:102d2000800f54000100360000047800080178008c
:102d30006a8544001a0078004cfd07001a00440020
:102d4000000d7800e8844400990c14000048eb0062
:102d50004f0578004f04be00000006001000780008
:102d6000dbf73700900190000388a30001003200d8
:102d7000e6ff37000348a30001003a00f7ff070011
:102d800000000600889fbe008a1f7800800478003b
:102d90004900900002047800800f540001003600c2
:102da00000047800080178006a8544001a00780061
:102db0002efd07001a004400000d7800e88444004e
:102dc000990c14000048eb004f0578004f04be003a
:102dd00000000600f2874700889fbe008a9fbe0061
:102de0008c9fbe008e1f780080047800010578005b
:102df00002047800830578006107620002003a004f
:102e00008b0f540008003900080178008a00780010
:102e100009007800d3ff07008b0f5400020039002f
:102e2000880578001e003700088655000c017800e0
:102e3000f00f5600010036000201200001022000c0
:102e40007e80570010fd07008c06780005003700d3
:102e500002012000fe80570009007800c1ff070032
:102e6000f0865600ef8f5600f9ff3e004461de0009
:102e700000ff2f000091b90002014600fe805700bc
:102e800009007800b7ff07000e00e00004003a00d8
:102e9000080178008a00780009007800b1ff070077
:102ea0000b0078004f0778004f06be004f05be00ac
:102eb0004f04be002f01b100000006000000050015
:102ec0000000050000000500000178000040eb0054
:102ed0008080fb00818040002314210063c27800c1
:102ee0000404e00003003a003014210060c07800c0
:102ef0000000060092017800934f520004003a004f
:102f00003014210060c078000309e8000100370098
:102f10000040e800ea4f5000edff360000000600d8
:102f2000f6874700889fbe008a9fbe008c9fbe0028
:102f30008e1f7800800478000104780083057800f3
:102f4000040678000000eb00c0b79f008080eb0013
:102f5000d1b79f00e0b79f00f2b79f0000082000a4
:102f600080bf9f0098007800010078000005eb000a
:102f7000010037000a05e800304178000204e00053
:102f80000300320053c2b300834f5100f9ff3a00ef
:102f90000a00e000040032000a017800090078000d
:102fa00070ff0700180c45001807780050c2b300e6
:102fb0009e4f100033013a000e07e8000e0c780017
:102fc00010003700cfb097000100a0000b003700c1
:102fd000cfb097000110a00008003700cfb09700d5
:102fe0000120a00005003700cfb097000130a000fd
:102ff00002003700cfb097000140a000c1b79f008a
:10300000000ce8001800780090407800b2c2b300cd
:1030100082cf5000f1ff320007003c0002c2b30033
:1030200082cf5000f0ff320032c2b30082cf500096
:1030300007003a00efff3700d2c2b30082cf500042
:10304000e0ff320002c3b30082cf5000e0ff320045
:10305000a2c2b30082cf50000d003a00000ce8007d
:103060001c80e900000e780010007800e0b79f0097
:103070000000e0000f003d00cfb097000100a2006b
:10308000c1b79f000000ea00e0b79f0009003700c9
:1030900002020700e0b79f0001003700000ce800c3
:1030a000180078009000fb000103b100e98f500088
:1030b000faff36004fb097000008a300020032006c
:1030c0000010a100c0b79f0018007800e1c2b30053
:1030d00090cf100016003a008000eb00d1b79f009f
:1030e0000000e800000c7800a1c2b30090cf1000ef
:1030f00006003a00000ce8001c80e900000e780091
:1031000010007800d0b79f0009003700e3010700e6
:10311000d0b79f0001003700000ce80018007800cd
:103120009000fb000103b100e98f5000faff360068
:103130000800780064ff07008046780018007800d7
:103140001000fb00fb01070091062000810f5000da
:103150003800320012003c0041062000810f500070
:10316000340032000a003c0011062000810f50009c
:103170002000320031062000810f50009a003200fa
:1031800051022000810f5000ae003a00a700370026
:1031900071062000810f5000aa003c008200370019
:1031a00001072000810f50005c00320007003c0046
:1031b000e1062000810f500074003200f10620006b
:1031c000810f50009f003a0039003700510720005e
:1031d000810f50002700320081072000810f50002e
:1031e0004200320031072000810f500095003a0064
:1031f000850037008d80fb000c01780000fe2f0059
:103200000f004000d90107000000e0009c003200e0
:1032100018007800000ce8009041780002fe2f00b2
:103220000f014100f88057000900780024ff0700d3
:103230000e0037008d80fb008c017800120020000a
:1032400000fe2f000f004000e70107000000e00033
:103250008b003200180ce80002fe2f000f01410025
:10326000f880570009007800abfc07000005450016
:10327000840037008d80fb008c0178000001eb009a
:1032800000fe2f000f004000d70107000000e00003
:103290007b003200180ce80002fe2f000f014100f5
:1032a000f880570009007800a5fd0700efff370000
:1032b0008d80fb008c0178000001eb0000fe2f00e8
:1032c0000f004000c80107000000e0006c00320061
:1032d000180ce80002fe2f000f014100f880570093
:1032e00009007800e5fc0700e0ff37008d80fb0057
:1032f0008c0178000001eb0000fe2f000f00400061
:10330000b90107000000e0005d00320018007800fd
:10331000000ce80090417800160037008c0178001e
:103320000001eb00010f200000fe2f000f00400005
:10333000ad0107000000e00051003200180ce80069
:103340000fb097009fb097002fb19700bfb19700c3
:10335000e00f5000e08f5800e00f5900e08f590057
:1033600003003a008001eb00c21321004000370047
:1033700083c7b30002fe2f000f014100f880570001
:103380000900780097fd0700b8ff37000b014500e2
:103390008d80fb008c01780000fe2f000f004000a4
:1033a000ea010700360037008d80fb000c01780031
:1033b00000fe2f000f0040006c0107000000e0003d
:1033c0002f00320018007800000ce80090417800cf
:1033d00002fe2f000f014100f8805700090078001d
:1033e000b7fe0700a1ff370000c8b30080cf56002a
:1033f00023003a00180ce8001c80e900000e780059
:10340000104078000d00370000c8b30080cf560090
:103410001b003a00180ce8001c80e900000e780040
:103420008001eb00100178001100370001c8b300e3
:1034300081cf560012003a00180ce800e0df9f0030
:103440000800370050c2b300e0df9f000e0c780088
:103450000000eb00c0b79f00e0b79f008080eb004a
:10346000d1b79f0013002000e2fd2f000f014100a3
:10347000f880570009007800b5fc07007bff370093
:10348000180ce8000a0078004f0778004f06be00cd
:103490004f05be004f04be006f01b10000000600e2
:1034a0008200fa00889fbe008a1f7800000578001d
:1034b00082047800c13f9f000004eb001000370039
:1034c0000902780088017800a2f72f000f0141005f
:1034d00081f72f008f8040000a00780090fe0700df
:1034e00008004000880f500004003d00b004200098
:1034f000e08b88000084eb000400370000047800b3
:103500004f3897001004e000edff3a000800780003
:103510004f0578004f04be000080fa00000006004e
:10352000889fbe008a1f780000047800010578009b
:103530000000eb000800e0001a00320018009000c4
:103540000058a3000c003200ea0444006800900018
:10355000990f100008003600b80990000001eb0038
:103560008200780008007800030001000080eb0072
:103570001900e0000b003200740044000008eb006a
:103580006c0044000008eb006a0044000008eb00f7
:103590000000eb000a00e000020032001800780092
:1035a000bff507004f0578004f04be00000006007d
:1035b000889fbe008a1f78000004be000000eb0058
:1035c0000800e00029003200180090000058a30015
:1035d000120032006a054400680090009a0f100043
:1035e00008003600b80990000001eb008200780066
:1035f00008007800030001000080eb001a00e000e2
:103600001a003200740044000008eb006c00440013
:103610000008eb006a0044000008eb00780a900004
:1036200008109000800f5200060031000002520086
:1036300011002000cfa2de00612bb9001800780035
:1036400088f5070000022000080040000008eb0099
:103650007e0044000008eb000000eb000900e000e1
:1036600002003200180078008df507004f05780041
:103670004f04be0000000600889fbe008a1f78002d
:1036800080047800010578000900780075fb0700c8
:10369000000478008a0178000801780011002000f9
:1036a000090078000a000700800078000080eb0025
:1036b000888f500001003a000000eb004f057800b1
:1036c0004f04be00000006001000780080f53700af
:1036d000889fbe008a9fbe008104780002047800a3
:1036e00009c5b9000900e00001003a000004eb0040
:1036f0000a017800800078000300780097fd070039
:10370000800078008a8f5000030032001100090009
:103710008980d80000047800080078004f05be00ba
:103720004f04be00000006000200fa00000178000d
:1037300001007800e2ff9f00900090000188a30044
:1037400006003200ea0140009300780082587800b9
:103750000280fb0081097800090037001200200078
:103760008f80e9007dfd0700800078000080eb007d
:103770000100e00002003200eff897000180fb003a
:103780000080fa0000000600e7ff37000200fa00a0
:10379000881f780000047800e2bf9f006481570012
:1037a000080078003eff0700980090000148a30041
:1037b000010032000080eb004f0478000080fa0026
:1037c000000006000000fa00cfb89700688157009b
:1037d0005081800010007800ecff07000080fa00a4
:1037e00000000600dafb37000000fa00cfb89700af
:1037f000688157005081800010007800e3ff0700c7
:103800000080fa000000060043fb07009bfb070056
:10381000cffb07004afc070072fc37000000fa00eb
:10382000cfb8970068815700508180001000780061
:10383000d6ff07000080fa000000060036fb0700f4
:103840008efb07003efc070066fc0700c0fb37004c
:103850000000fa00cfb897006881570050818000bf
:1038600010007800c9ff07000080fa000000060081
:10387000b7fb370080007800100020000202200013
:10388000828f500004003200e9805000e48f500025
:10389000010036000000eb0000000600889fbe001b
:1038a0008a1f780080047800090478008804780072
:1038b000394578000a00fb00eeff07000000e00039
:1038c000f9ff3a00b0c2b300804f55000500320046
:1038d000d0c2b3008000eb00804f550005003a00d5
:1038e000020037008000eb000100370011002000cb
:1038f0000804e8000000eb00030037006a02b9008a
:10390000020052000003b0003801fb0003fd2f004d
:1039100082814100e98f5100f8ff36000100e0008c
:1039200001003a000000ea004f0578004f04be0095
:1039300000000600f1fb2f0080804000f98f50004e
:1039400001003e000050a00000000600f9ff370013
:10395000f1f92f0080804000f98f500001003e00f7
:10396000f005b20000000600f9ff3700881f78005c
:103970000004780000082000808f500017003500f8
:1039800010082000808f50000b0034003008200009
:10399000808f500011003a0092007800688050003b
:1039a000000978003002be002003be00049cbe0067
:1039b0000694be000700370092027800648052002f
:1039c000000978001000be009e000700009cbe00a9
:1039d0000294be0010002000010037000000eb0040
:1039e0004f0478000000060084082000848f5000f7
:1039f0001d0032000d003c0014082000848f500090
:103a00002700320002003c000408200004003700b8
:103a100024082000848f50002a003200440820002f
:103a2000848f500048003a003b003700040a200011
:103a3000848f50002c00320004003c000409200058
:103a4000848f500040003a002d003700020c200007
:103a5000828f50001e003200020f2000828f500023
:103a600039003a00300037009380e9000200e0009e
:103a700005003200810978001102fb00cfa2de00b0
:103a8000612bb9002d0037008109780011427800c0
:103a90000482fb008002eb006033b800270037008f
:103aa00013027800e40052000200e0000a00320035
:103ab000810978001102be004fabde00860378005a
:103ac0001e00370093027800e88052000e00370095
:103ad00093027800e4805200810978001102be0050
:103ae0006033b800150037009380e9008109780041
:103af00011027800cfa2de00612bb9000f00370061
:103b000013037800e8005300810978003102be00f9
:103b10002103be00090037009380e9000200e000a5
:103b200002003200f1ff37009380e900810978003c
:103b3000110278008002eb006033b8000498be00e8
:103b40000690be001000050000000500440820009b
:103b5000848f5000270032000a003c001408200027
:103b6000848f50001c00320024082000848f5000f5
:103b70002600320004082000848f50002c003a00f8
:103b80001c00370004092000848f50001f00320001
:103b900004003c0084082000848f500024003a0078
:103ba00007003700040a2000848f50001100320003
:103bb000040c2000848f50001d003a0006003700de
:103bc0009380e9008109780091007800010878006d
:103bd00082487800150037009380e9008109780059
:103be0009100780001087800cf91de008288be0045
:103bf0000e0037009380e900810978009100780079
:103c00000108780082087800080037009380e900f6
:103c10008109780091007800010878006112b900ec
:103c2000612bb9008498be008690be00100005008c
:103c3000000005000000060006fa0700fdff07006f
:103c4000fcff370081037800e5f407000001be00a7
:103c50006000b8000478a30013003a006220e1007d
:103c600015003e000d0039008301d1000281d30010
:103c70008180d3008301d1000281d3008180d300f1
:103c80008301d1000281d3008180d3000538b000c8
:103c9000c42add00f300b2008381720007f0a700a0
:103ca00003f0a0000000060083ff270002002000b0
:103cb0006110b900f9ff370003ff2700f7ff370055
:103cc000020ab900001bb9000200b80081004200de
:103cd000810043000000060000c0da00000006007a
:083ce00000c0da00000006003c
:020000040000fa
:103ce800010000000500000012000000fcff0000b9
:103cf8000e00000011000000feff00000b00000095
:103d0800130000000100000009000000100000007e
:103d1800fcff00000a000000130000000000000083
:103d28000c00000014000000000000000500000066
:103d380011000000040000000e0000001100000047
:103d4800feff00000b00000017000000020000004a
:103d58000700000011000000feff00000e00000038
:103d68001800000003000000060000001800000012
:103d7800040000000c000000160000000000000015
:103d88000500000010000000040000000c00000006
:103d980011000000030000000900000011000000ed
:103da800020000000700000012000000fcff0000f5
:103db8000b00000012000000feff000007000000da
:103dc80012000000ffff00000600000017000000be
:103dd800020000000d00000014000000fdff0000bc
:103de8000b000000140000000300000006000000a3
:103df8001400000003000000050000001600000089
:103e08000300000005000000100000000200000090
:103e18000800000011000000030000000900000075
:103e280013000000030000000a0000001200000058
:103e3800feff00000500000016000000040000005e
:103e48000700000010000000fcff00000c0000004c
:103e580010000000fcff00000b000000170000002d
:103e6800fcff00000600000018000000ffff000033
:103e78000b00000011000000030000000d0000000e
:103e88000f00000003000000070000001100000000
:103e9800fdff00000a0000001600000001000000fd
:103ea8000e00000014000000fdff000008000000e4
:103eb80017000000feff00000c00000013000000c7
:103ec800020000000c0000001700000000000000c5
:103ed8000d0000000f0000000200000008000000b4
:103ee80012000000fdff000006000000170000009f
:103ef800ffff00000d00000012000000020000009b
:103f0800050000001000000001000000050000008e
:103f18001000000003000000090000001500000068
:103f2800030000000700000012000000fcff000072
:103f38000a0000000f000000fbff00001000000056
:103f48002300000001000000140000002a00000007
:103f5800feff00001500000024000000ffff000025
:103f68001100000025000000fbff00000f0000000a
:103f780027000000040000001400000029000000d1
:103f8800030000001200000024000000fdff0000f4
:103f98000f0000002a000000fbff000010000000d6
:103fa80028000000030000001000000028000000a6
:103fb800fdff00001700000026000000ffff0000c2
:103fc8000f0000002c000000fdff00000f000000a3
:103fd80026000000fbff0000140000002b0000007a
:103fe800fbff0000180000002b000000fdff000090
:103ff800130000002c000000feff00001600000067
:10400800240000000400000012000000230000004b
:10401800fcff00001000000029000000feff000067
:10402800170000002a000000ffff00000f0000003a
:104038002500000004000000170000002800000010
:1040480001000000130000002c000000feff00002b
:10405800180000002b000000fdff00001800000001
:104068002900000004000000120000002b000000de
:10407800fdff0000150000002b00000004000000f8
:104088001800000028000000fcff000010000000dd
:104098002c000000ffff00001600000025000000b3
:1040a80004000000140000002b000000fbff0000cb
:1040b800180000002b000000ffff000012000000a5
:1040c8002b000000fbff000010000000270000008c
:1040d80001000000100000002c0000000400000097
:1040e8000f0000002700000002000000110000007f
:1040f8002900000003000000140000002c0000004c
:1041080002000000150000002a0000000100000065
:10411800180000002600000003000000180000003e
:104128002b000000fbff00000f000000240000002f
:10413800030000001400000023000000feff000040
:104148001700000028000000010000001700000010
:104158002c000000000000001400000023000000f4
:10416800020000001300000027000000fdff00000f
:1041780010000000270000000400000015000000e7
:1041880026000000fcff00001000000029000000cd
:1041980004000000190000003800000004000000be
:1041a8002000000037000000fbff00001d00000099
:1041b80039000000feff0000210000003a00000066
:1041c800fbff00001c0000003b000000fcff00009b
:1041d8001e0000003e000000010000001e0000005c
:1041e80039000000020000001d000000400000002f
:1041f800fcff00001f0000003c000000040000005d
:10420800210000003d000000fdff00001b00000031
:104218003d000000fcff0000220000003b00000001
:10422800fdff0000190000003f000000fbff000038
:10423800190000003c000000040000001900000004
:1042480037000000000000001a00000038000000dd
:10425800fcff00001b0000003f000000fbff000007
:104268001e00000040000000ffff000022000000c8
:104278003a000000010000001d0000003c000000a2
:1042880004000000200000003a000000ffff0000ca
:104298001f00000037000000ffff000020000000a2
:1042a8003700000002000000200000003b00000072
:1042b800fbff00001c0000003b00000003000000a2
:1042c800220000003e000000040000002200000060
:1042d8003e000000fcff00001a000000380000004b
:1042e800fdff000021000000400000000200000067
:1042f8001b0000003e000000fdff00001c00000045
:1043080040000000ffff0000190000003c00000012
:104318000100000020000000400000000200000032
:104328001c0000003f000000030000001a0000000d
:104338003800000003000000210000003a000000df
:10434800fcff00001e0000003a000000feff000015
:104358001b0000003c000000040000001a000000e0
:1043680040000000010000001a0000003e000000ac
:10437800020000001a00000039000000ffff0000e2
:104388001c000000380000000200000019000000b6
:104398003a000000000000001e0000003c00000081
:1043a800fdff00001c0000003d000000ffff0000b2
:1043b8001f0000003800000001000000200000007d
:1043c8003a000000fdff0000200000003800000057
:1043d800010000001f0000003f0000000000000076
:1043e8001e00000038000000030000001c00000050
:1043f8003900000003000000220000003e00000019
:10440800010000001e0000003d0000000100000047
:104418001e00000039000000fcff00001c00000026
:104428003f00000000000000210000003e000000e6
:10443800020000001d0000003a000000000000001b
:104448002200000037000000fcff00001e000000f2
:1044580038000000010000001c0000003e000000c1
:10446800fcff0000200000003900000004000000ec
:10447800190000003d000000000000001d000000c1
:104488003d000000fbff000020000000400000008d
:10449800030000001f0000003a00000000000000b8
:1044a8001900000037000000040000001b00000095
:1044b8003c000000000000001f0000004000000059
:1044c80004000000220000003f000000030000007c
:1044d8002000000039000000ffff00001f0000005e
:1044e800400000000000000022000000380000002a
:1044f80002000000210000003c000000fcff00005a
:10450800210000003e000000000000001f00000025
:104518003f000000fdff00001c0000003f000000fd
:10452800020000001a0000003a000000020000002b
:104538001b0000003c000000040000001e000000fa
:1045480039000000fdff00001d0000003f000000d2
:10455800000000001e0000003d000000feff0000fb
:104568001c00000040000000030000001b000000c9
:104578003d00000003000000220000004000000091
:10458800fdff00002200000040000000fdff0000c9
:104598001f00000040000000ffff00001f00000097
:1045a80038000000fcff00001f0000003a00000077
:1045b800feff0000190000003b000000feff0000a5
:1045c8002200000037000000feff00001b00000072
:1045d8003a000000fbff000019000000390000004d
:1045e800feff00001c0000003e000000fdff000070
:1045f8001c0000003e000000000000002200000037
:104608003b00000003000000210000004000000003
:10461800000000001f000000400000000000000033
:104628001e0000003d000000010000001e00000008
:104638003e000000020000001e00000039000000db
:10464800ffff0000100000002a0000000200000028
:104658001500000023000000020000001200000006
:1046680028000000010000001300000029000000dd
:10467800040000001000000025000000fcff0000fe
:10468800110000002b000000fcff000013000000d8
:1046980024000000fdff00001200000026000000ba
:1046a80003000000180000002c000000feff0000be
:1046b80010000000230000000400000014000000a7
:1046c8002800000004000000170000002700000078
:1046d800fcff00001400000026000000000000009d
:1046e8001200000025000000040000001000000077
:1046f8002700000000000000110000002c0000004e
:10470800040000001700000024000000030000005f
:104718001800000025000000fdff00001500000043
:1047280026000000ffff0000130000002600000024
:10473800fdff0000150000002a0000000000000036
:10474800130000002b000000030000001700000009
:104758002c000000ffff0000160000002a000000e7
:10476800ffff0000110000002b0000000300000004
:104778001800000023000000ffff000018000000e0
:104788002b00000003000000140000002a000000b5
:10479800ffff00001100000028000000fdff0000de
:1047a8001800000027000000ffff000018000000ac
:1047b8002900000004000000160000002500000089
:1047c800ffff0000160000002300000001000000a9
:1047d8000f0000002b000000fdff00001200000089
:1047e8002a00000004000000170000002b00000051
:1047f80001000000160000002c000000020000006c
:104808000f0000002a000000ffff00001400000055
:104818002a000000fcff0000100000002300000038
:10482800040000001100000024000000ffff000049
:104838001300000023000000030000001600000021
:1048480029000000fbff00000f000000240000000a
:1048580003000000180000002c0000000300000006
:104868001300000029000000feff000013000000f4
:1048780025000000000000001300000024000000d4
:10488800020000001000000028000000feff0000e9
:104898001300000026000000ffff00000a000000cf
:1048a80013000000fbff00000600000013000000da
:1048b800fcff0000060000000f00000003000000dd
:1048c8000800000011000000ffff00000e000000bb
:1048d80013000000fcff00000700000012000000a9
:1048e800020000000900000015000000fbff0000a6
:1048f8000800000013000000020000000c00000087
:1049080010000000fcff00000b0000001100000078
:10491800ffff000005000000140000000100000077
:104928000500000010000000030000000600000061
:1049380015000000fdff0000080000001300000043
:10494800020000000e00000010000000020000003d
:104958000500000015000000010000000e00000026
:1049680016000000fdff00000b0000001000000012
:10497800fdff00000e000000100000000200000013
:104988000d00000017000000fcff000007000000f9
:1049980015000000020000000600000014000000de
:1049a800010000000800000018000000ffff0000e0
:1049b8000600000015000000ffff000007000000cf
:1049c80011000000fcff00000d0000000f000000b7
:1049d800030000000a0000000f00000003000000b0
:1049e8000500000010000000020000000b0000009d
:1049f80013000000030000000d0000001400000078
:104a08000200000005000000140000000300000080
:104a18000700000016000000020000000b00000064
:104a280012000000010000000a000000120000004f
:104a3800fdff000007000000170000000400000050
:104a48000700000015000000040000000a00000034
:104a58001400000004000000080000001500000019
:104a6800030000000a0000000f0000000100000021
:104a78000a00000010000000fdff00000800000010
:104a880010000000000000000900000017000000ee
:104a9800fdff00000e00000010000000feff0000f7
:104aa8000b00000015000000fcff00000d000000d6
:104ab80014000000020000000800000018000000b8
:104ac800ffff00000d00000018000000fbff0000c1
:104ad80007000000100000000400000009000000aa
:104ae80012000000fdff0000050000000f0000009c
:104af800feff00000a00000017000000feff000093
:104b08000d00000012000000feff00000800000079
:104b1800130000000300000007000000110000005f
:104b2800000000000e00000014000000ffff00005d
:104b38000800000018000000040000000b0000003e
:104b480012000000000000000e000000100000002d
:104b5800fbff00000a000000150000000300000031
:104b68000b00000016000000000000000e0000000e
:104b780018000000030000000500000013000000fa
:104b8800fcff00000700000013000000fcff00000d
:104b98000900000013000000feff000007000000ed
:104ba80010000000ffff0000070000000f000000d9
:104bb80001000000050000000f00000003000000d5
:104bc8000a000000140000000200000005000000b8
:104bd80018000000010000000a0000001700000093
:104be800000000000a000000160000000400000099
:104bf8000900000014000000feff00000b00000088
:104c08001500000003000000070000001500000068
:104c1800fcff00000900000013000000ffff000077
:104c28000a0000000f00000000000000050000005e
:104c38000f000000fdff0000090000001200000046
:104c4800fbff00000800000018000000040000003e
:104c58000500000013000000fbff00000500000035
:104c680010000000010000000d0000000f0000000f
:104c7800040000000800000012000000020000000c
:104c880006000000170000000300000006000000f6
:104c980015000000ffff00000900000015000000db
:104ca800010000000800000016000000fdff0000e1
:104cb8000600000010000000fcff00000a000000d1
:104cc80013000000fdff00000c0000000f000000b2
:104cd80003000000080000001400000004000000a9
:104ce8000b00000016000000fdff00000800000097
:104cf800120000000400000006000000130000007d
:104d0800040000000700000016000000fcff00007f
:104d18000800000018000000feff00000e00000060
:104d280012000000ffff0000090000001200000050
:104d3800020000000a0000000f000000fdff000054
:104d48000a00000013000000fbff00001200000032
:104d580025000000020000001100000024000000ef
:104d6800feff00001100000024000000feff00000c
:104d780015000000260000000000000018000000d8
:104d880024000000ffff00001800000024000000bd
:104d9800fdff00001500000029000000feff0000d4
:104da8001500000027000000010000000f000000af
:104db8002c00000003000000160000002600000080
:104dc800ffff0000120000002b000000fbff0000a6
:104dd8000f00000023000000030000001200000084
:104de80026000000ffff00000f0000002300000065
:104df800010000001000000023000000feff00007a
:104e08001700000025000000ffff00000f00000051
:104e180023000000ffff0000130000002500000031
:104e2800feff00001400000023000000ffff000048
:104e38001700000028000000fcff0000140000001c
:104e48002a00000001000000110000002b000000f3
:104e5800fbff000010000000280000000100000017
:104e6800160000002b000000fcff000018000000e6
:104e780026000000040000001200000024000000ca
:104e8800010000001100000026000000fdff0000e6
:104e98001800000023000000fcff000013000000c1
:104ea80028000000ffff000017000000230000009a
:104eb800ffff0000110000002700000000000000b4
:104ec800120000002500000000000000170000008c
:104ed8002700000000000000110000002b00000067
:104ee80003000000120000002a000000ffff00007d
:104ef8001200000028000000030000001700000056
:104f08002a000000fdff0000180000002400000037
:104f1800fbff0000160000002a000000040000004b
:104f28001600000024000000feff00000f00000033
:104f380024000000feff000016000000270000000b
:104f48000400000016000000230000000400000018
:104f580016000000290000000400000011000000f5
:104f680024000000040000001100000029000000d7
:104f7800ffff00000f0000002300000004000000f5
:104f880012000000290000000100000014000000c9
:104f980023000000fdff00001800000024000000ae
:104fa800feff00001f0000003800000001000000a4
:104fb8001d0000003b000000fbff00001f00000078
:104fc8003f000000ffff00001a000000380000004a
:104fd800fcff00001e00000040000000fcff000075
:104fe8001d00000037000000fbff00001f0000004c
:104ff8003a000000fcff00001d0000003f00000018
:10500800000000001d000000400000000300000038
:105018001b0000003e000000010000001d00000011
:1050280038000000000000001d0000003e000000e5
:10503800030000001e0000003b000000fcff000011
:10504800220000003d0000000300000020000000d6
:105058003a000000feff00001f0000003a000000b8
:10506800feff0000190000003e00000000000000e4
:10507800190000003d000000fdff000019000000bd
:1050880040000000fdff0000220000003f0000007b
:10509800feff0000190000004000000000000000b2
:1050a8001900000038000000ffff00001e0000008b
:1050b8003c000000fbff00001f0000004000000053
:1050c800feff00001b0000003f000000ffff000083
:1050d800200000003a000000040000002100000049
:1050e80037000000feff0000190000003d0000002e
:1050f800fdff00001c0000003e000000fdff000056
:105108001900000040000000feff00001e00000023
:1051180038000000030000001e00000039000000f5
:10512800feff00001d0000003a0000000200000021
:105138001c0000003a000000020000001a000000f5
:1051480039000000fdff00001d0000003e000000c7
:10515800fdff0000190000003d00000000000000f5
:105168002100000039000000030000001f000000bb
:105178003b00000002000000210000003800000091
:1051880002000000190000003e00000000000000be
:105198001f0000003f000000040000002200000083
:1051a80040000000ffff00001b0000003900000065
:1051b800030000001e00000037000000010000008e
:1051c800190000003a000000fdff0000190000006f
:1051d80040000000fdff0000210000003b0000002f
:1051e80002000000210000003f0000000300000052
:1051f8001c00000038000000fbff00001a0000003f
:1052080039000000feff00001c000000370000000d
:10521800030000001c0000003a000000020000002b
:105228001d0000003d000000040000001d000000fb
:1052380038000000fdff00002100000038000000d9
:10524800030000001a0000003900000001000000ff
:10525800220000003e000000fcff000019000000d2
:105268003900000000000000210000003f0000009d
:10527800feff00001a00000040000000ffff0000d1
:105288001f0000003f000000010000002100000096
:105298003b000000fcff00001b0000003c00000079
:1052a800fdff00001b0000003d000000040000009e
:1052b8001d0000003f000000000000001900000071
:1052c80039000000ffff0000210000003700000047
:1052d800030000001d0000003c0000000200000068
:1052e8001c0000003a000000020000001c00000042
:1052f8003c000000020000001b0000003a00000013
:10530800feff000019000000380000000200000045
:105318001f0000003d000000020000001e00000009
:1053280038000000010000001a0000003e000000e4
:1053380004000000190000003e0000000100000009
:1053480022000000400000000000000021000000d2
:1053580038000000ffff00001e0000003e000000b3
:10536800fcff00001900000039000000fdff0000ec
:105378001b000000370000000400000020000000af
:1053880040000000040000001e000000370000007c
:10539800fdff00001b0000003900000001000000b4
:1053a8001c00000037000000fcff00002200000085
:1053b80040000000030000001a0000004000000048
:1053c800feff000019000000370000000100000087
:1053d800200000003f000000000000001e00000048
:1053e8003e000000feff000019000000370000002a
:1053f800fcff00002000000038000000040000004e
:10540800190000003e000000030000001f0000001b
:1054180039000000fbff0000210000003e000000f2
:10542800040000001e0000003d0000000100000014
:105438001c00000037000000040000001b000000f2
:105448003b000000feff0000220000003c000000be
:1054580002000000100000002a0000000400000004
:105468001200000029000000fdff000014000000e9
:105478002b000000feff00000f00000024000000c9
:1054880003000000160000002c000000fdff0000d3
:1054980012000000270000000000000016000000b5
:1054a8002b000000fdff0000150000002800000090
:1054b800feff0000180000002b000000fcff0000a9
:1054c800120000002b000000fdff00001300000088
:1054d80027000000feff0000130000002a00000063
:1054e800040000000f000000260000000200000079
:1054f8001700000024000000feff0000100000005c
:105508002a0000000400000013000000230000002f
:105518000400000010000000250000000300000047
:10552800110000002b000000ffff00001000000029
:105538002500000002000000150000002300000004
:10554800ffff00000f0000002a000000ffff00001e
:1055580013000000270000000400000016000000ef
:105568002b000000ffff00001600000027000000cd
:10557800ffff0000170000002c00000002000000e0
:105588001100000026000000fdff000013000000cd
:105598002a000000feff000018000000290000009b
:1055a80003000000150000002a00000004000000ad
:1055b800150000002a00000004000000110000008f
:1055c8002c000000fbff0000100000002800000075
:1055d800000000001000000027000000010000008b
:1055e8001000000023000000fbff00000f00000077
:1055f80023000000fcff000014000000250000004c
:10560800fbff00001300000027000000fbff000064
:105618001200000027000000fdff0000110000003c
:1056280024000000feff0000120000002b00000014
:10563800020000001200000023000000fbff000031
:105648001600000026000000000000001400000002
:105658002a00000004000000170000002c000000d1
:1056680000000000160000002c00000004000000ec
:10567800180000002c0000000000000018000000c6
:105688002b000000030000001700000025000000a8
:10569800010000001100000027000000fcff0000ce
:1056a80010000000250000000200000008000000b3
:1056b80011000000000000000700000015000000b5
:1056c800fdff00000a00000013000000fcff0000be
:1056d8000a00000013000000fbff000008000000a3
:1056e8001200000000000000080000001500000083
:1056f800010000000800000013000000fbff00008c
:105708000a00000013000000fdff00000600000072
:1057180013000000fbff0000090000001300000058
:10572800ffff00000c00000018000000fcff000054
:105738000800000012000000feff00000a00000040
:105748000f000000010000000d0000001100000023
:10575800010000000c00000016000000ffff000020
:105768000d00000014000000030000000e000000ff
:1057780015000000010000000600000018000000ed
:10578800010000000c0000001800000002000000ea
:105798000800000011000000fdff00000c000000e0
:1057a80010000000040000000700000013000000c3
:1057b800feff00000d00000011000000ffff0000c8
:1057c80007000000130000000400000006000000ad
:1057d80012000000feff00000a0000001700000091
:1057e800fdff00000700000010000000000000009e
:1057f8000d00000012000000ffff0000050000007f
:105808001000000000000000070000001400000065
:10581800020000000d00000016000000fcff000060
:105828000900000016000000fcff0000080000004e
:1058380015000000020000000a000000100000002f
:10584800feff00000900000017000000ffff000035
:10585800080000000f000000fbff0000050000002a
:1058680013000000020000000500000017000000ff
:10587800ffff00000b00000017000000feff000003
:105888000600000012000000fbff000006000000f8
:1058980014000000feff00000600000010000000d9
:1058a800fcff0000090000001000000004000000d8
:1058b8000b00000012000000040000000c000000b3
:1058c80011000000000000000c00000010000000a3
:1058d80003000000050000001700000001000000a0
:1058e8000700000010000000000000000c0000008d
:1058f800150000000400000005000000150000006d
:10590800040000000900000014000000020000006c
:105918000b00000011000000020000000a00000057
:1059280010000000fbff000006000000110000004e
:10593800fdff00000c000000140000000300000040
:105948000d00000015000000fcff0000060000002c
:1059580011000000fdff0000050000001400000019
:1059680001000000080000000f0000000200000015
:105978000b00000011000000000000000c000000f7
:1059880011000000000000000900000014000000e1
:10599800feff00000c0000001400000000000000e2
:1059a8000b000000140000000100000007000000c8
:1059b80010000000feff00000800000010000000ba
:1059c800fcff0000090000001300000000000000b8
:1059d8000b00000012000000020000000700000099
:1059e800120000000200000009000000170000007b
:1059f800010000000b00000018000000fcff000080
:105a0800050000000f000000fdff00000700000077
:105a180012000000000000000a000000150000004d
:105a2800ffff0000050000000f000000fcff000061
:105a3800070000000f000000020000000d00000039
:105a48001300000004000000050000000f00000023
:105a58000000000009000000140000000000000021
:105a68000600000016000000feff00000c00000009
:105a780014000000020000000600000018000000ea
:105a8800feff00000500000012000000fcff0000ff
:105a98000800000016000000feff000007000000dc
:105aa80015000000ffff00000500000015000000c1
:105ab800ffff00000700000010000000fdff0000cd
:105ac8000500000010000000feff00000d000000af
:105ad8001100000003000000090000001000000091
:105ae8000400000009000000140000000400000089
:105af8000600000010000000030000000b0000007a
:105b080014000000030000000d0000001200000057
:105b1800000000000c00000014000000fbff000063
:105b28000e0000000f000000feff0000050000004e
:105b3800160000000000000006000000120000002f
:105b4800fdff00000c000000100000000100000034
:105b58000e00000015000000fdff0000130000000b
:105b680024000000ffff00001800000026000000cd
:105b7800ffff0000150000002c000000fdff0000e2
:105b88001100000029000000fcff000014000000c4
:105b98002700000003000000170000002500000097
:105ba800ffff0000180000002b00000004000000a8
:105bb8001700000023000000fcff00001300000095
:105bc8002700000002000000160000002b00000063
:105bd8000100000010000000240000000200000086
:105be8000f00000025000000fbff00001600000069
:105bf80027000000ffff000018000000240000003c
:105c08000400000017000000290000000100000047
:105c1800160000002800000001000000110000002c
:105c280026000000fdff0000120000002500000013
:105c380000000000100000002a000000fdff000026
:105c48000f00000026000000020000001400000001
:105c58002c000000feff00000f0000002b000000d9
:105c6800feff00001500000025000000fdff0000f9
:105c78001800000026000000fdff000010000000d2
:105c88002a000000ffff00000f00000026000000af
:105c9800fcff00000f0000002700000002000000c9
:105ca8001500000028000000ffff0000120000009f
:105cb8002a00000000000000170000002800000073
:105cc800040000001700000027000000ffff00008c
:105cd800120000002300000004000000170000006c
:105ce80024000000fdff0000150000002600000051
:105cf800000000001000000026000000fcff00006b
:105d08001000000026000000000000001300000042
:105d180027000000ffff0000170000002700000018
:105d2800ffff00001300000026000000fcff000039
:105d3800170000002a000000010000001400000005
:105d48002b000000feff00001800000025000000e6
:105d5800feff000011000000270000000400000002
:105d68001300000028000000fbff000015000000e1
:105d780026000000010000001700000023000000ba
:105d8800ffff00001100000026000000feff0000d9
:105d980017000000260000000200000016000000a6
:105da80026000000fdff000016000000250000008e
:105db800feff00001c0000003e0000000300000081
:105dc8002100000038000000020000001b00000055
:105dd8003900000004000000200000003a00000024
:105de800feff00001c00000040000000fbff000058
:105df800190000003e000000000000001a0000002a
:105e080040000000fbff00001e0000003a000000f8
:105e1800000000001c0000003f000000000000001f
:105e28001a0000003e000000feff00001a000000fb
:105e38003f000000fcff00001a00000040000000c6
:105e4800010000001c0000003a000000ffff0000f5
:105e58001b0000003d000000fbff000021000000c7
:105e680040000000ffff00001c0000003e00000092
:105e7800010000001f0000003700000001000000c2
:105e88001f00000038000000000000002100000092
:105e98003e000000fdff0000190000003a0000006d
:105ea800030000001c0000003d000000fdff000092
:105eb8002200000039000000030000001900000063
:105ec8003d000000fdff0000220000003700000038
:105ed800feff00001a0000003d000000fbff00006c
:105ee8001e0000003e000000010000001900000034
:105ef8003b000000010000001d0000003d00000004
:105f0800000000001f0000003c000000ffff000030
:105f18001b00000038000000000000002100000005
:105f28003a000000fcff00001f00000040000000d5
:105f3800fcff00001a00000040000000fcff000009
:105f48001f0000003a000000000000001c000000d4
:105f58003d000000040000001900000037000000a8
:105f6800fbff00001c0000003d000000ffff0000d8
:105f7800190000003c000000feff00001f000000a8
:105f880039000000fcff0000210000003d00000077
:105f9800020000001c0000003f000000feff00009f
:105fa8001b00000039000000040000001e00000073
:105fb8003a00000000000000190000003b0000004b
:105fc800ffff0000210000003a000000040000006c
:105fd8001b00000040000000020000001900000043
:105fe8003c000000030000001b0000003700000018
:105ff800fcff00002000000040000000030000003b
:106008001e0000003d0000007b22000076650000b5
:1060180072730000696f00006e2200003a250000cc
:10602800642c000022730000616d0000706c000099
:10603800655f00007261000074650000223a00008c
:10604800256400002c220000736100006d700000c0
:106058006c650000735f000070650000725f0000ef
:1060680070610000636b000065740000223a000054
:10607800256400002c220000636f00006c7500008e
:106088006d6e00005f6c00006f63000061740000bb
:10609800696f00006e2200003a7b000000220000b9
:1060a80041630000636500006c650000726f0000ca
:1060b8006d6500007465000072580000223a000007
:1060c800256400002c0000002241000063630000ea
:1060d800656c0000657200006f6d0000657400005b
:1060e80065720000592200003a250000642c000067
:1060f8000022000041630000636500006c65000039
:10610800726f00006d65000074650000725a00002f
:10611800223a0000256400002c00000022470000fd
:10612800797200006f730000636f000070650000f3
:10613800582200003a250000642c000000220000cc
:1061480047790000726f0000736300006f700000f1
:1061580065590000223a0000256400002c00000068
:1061680022470000797200006f730000636f00001f
:10617800706500005a2200003a2500006400000003
:106188007d7d00000a000000537400006172000069
:106198007475000070200000004500005252000095
:1061a8004f5200003a200000736500006e73000033
:1061b8006f720000206900006e6900007420000002
:1061c80072650000737500006c740000203d0000cb
:1061d80020250000640a000000450000525200001b
:1061e8004f5200003a200000736500006e730000f3
:1061f8006f720000206300006f6e00006669000087
:106208006775000072610000746900006f6e00001d
:106218002072000065730000756c00007420000097
:106228003d200000256400000a000000626d0000a7
:10623800693100003630000000730000656e000010
:10624800736f000072200000747900007065000010
:106258002069000073200000257300000a00000078
:10626800736500006e7300006f72000020730000f9
:10627800616d0000706c0000652000007261000014
:106288007465000020730000657400002061000040
:106298007420000025640000487a00000a0000000d
:1062a8007a000000790000007800000061630000b7
:1062b800636500006c650000726f00006d6500008a
:1062c80074650000722000006178000065730000aa
:1062d80020250000732500007325000073200000ae
:1062e800656e0000616200006c65000064200000bb
:1062f800776900007468000020720000616e000079
:1063080067650000207300006574000020610000cc
:10631800742000002b2f00002d250000644700008a
:10632800730a000000670000797200006f6d0000ba
:106338006574000065720000206100007865000047
:1063480073200000257300002573000025730000ea
:10635800206500006e610000626c0000656400004a
:106368002077000069740000682000007261000056
:106378006e6700006520000073650000742000004f
:1063880061740000202500006444000050530000a0
:106398000a00000045520000524f0000523a000027
:1063a800204700006f740000206100002062000098
:1063b8006164000020730000656e0000736f0000c8
:1063c800722000007374000061740000757300008f
:1063d8003a200000256400000a0000000a0a0000b4
:1063e8000a4f00007665000072720000756e0000aa
:1063f800210a00000a000000496e000076610000d2
:106408006c6900006420000063610000746500008e
:10641800676f000072790000206600006f7200004c
:106428002074000068690000732000006d6f000090
:10643800646500006c000000556e00006b6e000083
:106448006f7700006e200000636c0000617300002d
:1064580073690000666900006361000069740000e8
:106468006f6e0000007200003a20000025640000f2
:1064780020630000617400003a20000025640000d9
:1064880020700000696400003a20000025640000c4
:106498000a0000004e650000757200006f6e000073
:1064a800202500006420000065720000726f000063
:1064b80072200000256400000a00000055700000ea
:1064c80064610000746900006e670000204e0000df
:1064d80065750000726f00006e20000025640000e2
:1064e800207400006f200000636100007420000029
:1064f800256400000a0000007b22000049440000d7
:10650800223a0000256400002c22000045520000b9
:10651800522200003a250000640000002c220000ee
:1065280025640000223a000025640000007d000078
:106538000a0000007b2200004d6f00006465000027
:106548006c4e0000756d000062650000722200004c
:106558003a250000642c0000224300006c61000012
:1065680073730000696600006963000061740000cd
:10657800696f00006e2200003a25000064000000e8
:106588002c2200004665000061740000757200004e
:10659800654c0000656e000067740000682200000a
:1065a8003a250000642c00002246000065610000c6
:1065b8007475000072650000566500006374000081
:1065c8006f720000223a00005b00000025640000a2
:1065d80000250000730d00000a000000636f000032
:1065e8006e6e0000656300007400000064690000be
:1065f800736300006f6e00006e6500006374000036
:106608000000000004040000011000002040000009
:1066180080020000010800000802000004000000d9
:04662800030000006b
:020000040000fa
:10662c001200fa00889fbe006a024700004a7800f8
:10663c006c004700010878006e00470002087800e3
:10664c0070004700030878000f0478000f007800f2
:10665c00800478000040eb00004f78007000470089
:10666c00100078004002b000104078000080fb0061
:10667c00ee00470091007800810040006400470064
:10668c000108780064004700100078008000780052
:10669c000101e900e6004700820878000000e800ec
:1066ac000000e8000000d100800040000f007800de
:1066bc00818747000000e8000000d1000000400086
:1066cc00e8004700800878008000eb000e80e800ae
:1066dc000108780070004700100078000000e0000e
:1066ec000600320070004700100078007c0040006b
:1066fc00100078000000e00003003a0000c0eb003e
:10670c00004f7800420037006e0047001000780000
:10671c000000e00003003a0040cfb300004f7800c7
:10672c003b00370070004700100078000080e80044
:10673c0010407800e14f500006003a006a00470014
:10674c0010407800804078000174a0006a00470077
:10675c000148780070004700100078007c00400071
:10676c001002780068004700900078007000470025
:10677c00100078000000e800104078006401470029
:10678c009201780001017800ea00470091407800fe
:10679c0004000100004f78001e4078000004e00067
:1067ac0019003a00110037006c0047009000780087
:1067bc000e80e8001000780000804000e8004700e0
:1067cc00110178008e80e800910078008100410072
:1067dc0091407800014878000e80e80010007800a5
:1067ec008000e8000e80e800010878000e80e800c8
:1067fc00900078006e00470010007800808f5000e9
:10680c00e9ff390002003700e0cfb300004f7800f9
:10681c001e40780089077800880778004f04be0076
:10682c000080fa00000006000a00fa000e82e80060
:10683c00004a7800640047000108780066004700b1
:10684c000208780068004700030878000040eb005d
:10685c00004f78008040eb000e00e8000148780003
:10686c0068004700100078000000e00006003200cd
:10687c0068004700100078007e004000100078008f
:10688c000000e00003003a0000c0eb00004f78006d
:10689c006a00370066004700100078000000e00036
:1068ac0003003a0040cfb300004f7800630037007c
:1068bc0068004700100078000080e8001040780065
:1068cc00e14f500006003a000e80e80010407800be
:1068dc00804078000174a1000e80e8000148780027
:1068ec0068004700100078006a00400010407800f3
:1068fc00f14f50000600320068004700100078008d
:10690c007200400010407800f54f50003e003a00f5
:10691c0068004700100078007e00400010027800ec
:10692c0068004700100078000000e8001040780074
:10693c00e600470091017800e4004700110178005f
:10694c008e80e8009140780004000100004f780030
:10695c0068004700100078000002b00010017800b9
:10696c001000200001002000020001002e00370062
:10697c0068004700100078007e004000100278008c
:10698c000e00e800104078000080fb00e400470097
:10699c00910078008080400068004700100078006b
:1069ac000000e8001040780013002000010178007e
:1069bc008e80e8009140780004000100004f7800c0
:1069cc000e80e800104078008040e8000e80e8005f
:1069dc000148780068004700100078000002b00001
:1069ec0010017800100020000100200002000100be
:1069fc000e00e800104078008040e8000e00e8002f
:106a0c000148780001003700000000000e00e8008b
:106a1c00104078000080fb00e600470091007800f1
:106a2c00810f5000d2ff39001e4078000004e000b6
:106a3c0002003200e0cfb300004f78001e40780017
:106a4c000080fa00000006000600fa00e40047008f
:106a5c008008780031c0b3000e00e80001487800cf
:106a6c0064004700100078006b0b0700004f7800a3
:106a7c0064004700100078000080e80010407800a7
:106a8c00e14f500006003a00640047001000780007
:106a9c0011c0b3004002b000014878000500370077
:106aac0064004700100078008040eb004002b0000a
:106abc00014878001e4078000004e0000e003a0007
:106acc0064004700100078000080e8001040780057
:106adc00e14f500008003a000e80e800e400470047
:106aec00910178001200200080007800f0c7b300fc
:106afc00cbfe0700004f78001e4078000004e00039
:106b0c0036003a0064004700900078000040eb002b
:106b1c0080487800090037006400470010007800b6
:106b2c00e4004700910178001200200080007800fa
:106b3c000040eb00bafe0700004f78000e00e800a2
:106b4c00104078000080fb000000ea004f00de00df
:106b5c00004078008e00e800914078000141e90087
:106b6c008e00e800824878000004e0000600320045
:106b7c0064004700100078009040780010cdb300fe
:106b8c0080cf5000e4ff3a001e4078000004e00083
:106b9c0010003a0064004700100078009040780024
:106bac0010cdb30080cf50000a003a0064004700bb
:106bbc00100078008080eb00640040000108780031
:106bcc00640047001000780007000700004f7800b1
:106bdc0002003700d0cfb300004f78001e40780081
:106bec000080fa00000006000400fa008e80e80025
:106bfc008008780061cbb3000e00e80001487800f3
:106c0c000e80e800100078000000e0000600320062
:106c1c000e80e800100078000002b0001000780030
:106c2c000000e00003003a0000c0eb00004f7800c9
:106c3c00260037000e00e8008e80e80091017800f5
:106c4c001200200080007800e0c7b300f6fe0700b9
:106c5c00004f78000e80e800100078000002b000b1
:106c6c00100178001000200001002000020001003b
:106c7c001e4078000004e0000e003a000e80e80090
:106c8c00100078000080e80010407800e14f5000c0
:106c9c0008003a000e00e8008e80e80091017800b0
:106cac001200200080007800f0c7b3005cfe0700e3
:106cbc00004f78001e4078000004e00003003a000a
:106ccc000e80e80010007800f40a07001e407800df
:106cdc000080fa00000006000400fa008e80e80034
:106cec00800878000040eb00004f78000e80e80030
:106cfc00100078000000e000060032000e80e80072
:106d0c00100078000002b000100078000000e000d5
:106d1c0003003a0000c0eb00004f78001900370068
:106d2c000e80e800100078000c0b0700004f780074
:106d3c001e4078000004e00012003a000e80e800cb
:106d4c00100078004c0c0700004f78001e407800b3
:106d5c000004e0000b003a000e80e8001000780000
:106d6c000b000700004f78001e4078000004e00084
:106d7c0004003a000e80e80010007800060c0700b2
:106d8c00004f78001e4078000080fa0000000600da
:106d9c000400fa008e80e800800878000040eb00c8
:106dac00004f78000e80e800100078000000e00032
:106dbc00060032000e80e800100078000002b000df
:106dcc00100078000000e00003003a0000c0eb0067
:106ddc00004f78000b0037000e80e80010007800a0
:106dec00330d0700004f78001e4078000004e000cf
:106dfc0004003a000e80e80010007800d10d070066
:106e0c00004f78001e4078000080fa000000060059
:106e1c000600fa000e81e8000009780064004700c3
:106e2c00010878000040eb00004f78008040eb0038
:106e3c000e00e8000148780064004700100078005c
:106e4c000000e000060032006400470010007800eb
:106e5c000002b000100078000000e00003003a00cf
:106e6c0000c0eb00004f7800260037000e00e80051
:106e7c00e4004700910178001200200080007800a7
:106e8c0030c0b300e6fd0700004f78001e407800cc
:106e9c000004e0001b003a000e00e80010407800ef
:106eac00e34060000e80e800100078000080e800ed
:106ebc00014878000e00e800104078000080fb00cc
:106ecc006c0060004280de00804078000e80e8009c
:106edc00100078000000e800014878000e00e8007f
:106eec00104078008080fb000003200000806000d0
:106efc004480de00004078008e80e800910078002d
:106f0c00804878001e4078000080fa0000000600df
:106f1c000c00fa0064024700004a78006600470043
:106f2c000108780068004700020878006a004700f2
:106f3c00030878000040eb00004f78008040eb0025
:106f4c000e00e8000148780064004700104078000b
:106f5c00e74060000e80e800014878000e80e800f1
:106f6c00104078000080fb0064006000c280de00ee
:106f7c0063004700014878000e80e800104078005c
:106f8c00e34060000e80e800014878006300470091
:106f9c0010407800e14f500003003a0031c0b300bc
:106fac000e00e800014878006a00470010007800e5
:106fbc000000e000430032000e80e8001040780032
:106fcc000080fb00e20f500014003200e30f500071
:106fdc0022003200e10f500037003a0066004700f3
:106fec00100078000000e00003003a0000c0eb0045
:106ffc00004f7800350037006a0047001001780018
:10700c0066004700900078000e00e8001040780001
:10701c00a60d0700004f78002c00370068004700d1
:10702c00100078000000e00003003a0000c0eb0004
:10703c00004f7800250037006a00470010017800e7
:10704c0068004700900078000e00e80010407800bf
:10705c007e0e0700004f78001c00370068004700c8
:10706c00100078000000e0000400320066004700c9
:10707c00100078000000e00004003a0000c0eb00b3
:10708c00004f780000000000100037006a00470035
:10709c0090017800680047001001780066004700f6
:1070ac00900078000e00e80010407800e20f070016
:1070bc00004f780005003700b0cfb300004f7800c8
:1070cc000200370000c0eb00004f78001e40780033
:1070dc000080fa00000006000600fa000e81e800ad
:1070ec000009780064004700010878000040eb00bc
:1070fc00004f78000e80e800100078000080e80057
:10710c00100078008000eb00d2002000030020006b
:10711c00820f5000838f58006a003e00006001000f
:10712c000d00370013003700270037001f00370011
:10713c001e0037002b003700310037003e003700af
:10714c003600370012003700420037004800370085
:10715c004e00370054003700640047009000780060
:10716c000e80e800100078006f070700004f7800d1
:10717c005500370064004700900078000e80e8004e
:10718c0010007800f7070700004f78004e0037001a
:10719c0064004700900078000e80e8001000780032
:1071ac001c080700004f78004700370064004700b8
:1071bc00900078000e80e800100078008607070029
:1071cc00004f7800400037006400470090007800c2
:1071dc000e80e800100078003a080700004f780095
:1071ec003900370064004700900078000e80e800fa
:1071fc00100078006f080700004f7800320037004d
:10720c0064004700900078000e80e80010007800c1
:10721c00a4080700004f78002b00370064004700db
:10722c00900078000e80e80010007800d908070064
:10723c00004f78002400370064004700900078006d
:10724c000e80e8001000780017090700004f780046
:10725c001d00370064004700900078000e80e800a5
:10726c001000780093070700004f780016003700d5
:10727c0064004700900078000e80e8001000780051
:10728c00a91e0700004f78000f003700640047006c
:10729c00900078000e80e80010007800001f0700b6
:1072ac00004f780008003700640047009000780019
:1072bc000e80e8001000780040090700004f7800ad
:1072cc0001003700000000001e4078000080fa002a
:1072dc00000006000600fa000e81e8000049780064
:1072ec0064004700010878008040eb000e00e800c5
:1072fc000148780064004700100078004609070038
:10730c00004f78001e4078000004e00003003200bb
:10731c0000c0eb00004f7800260037000e00e8009c
:10732c00e4004700910178001200200080007800f2
:10733c00b0c7b300bafc0700004f78001e407800bd
:10734c000004e0001b003a000e80e80010407800ba
:10735c00e14f500009003a000e80e8001040780020
:10736c00c300dd000e00e8001040780080c0700003
:10737c000e00e80001487800060037000e00e80017
:10738c0010407800804078000134a1000e00e80025
:10739c00014878000e00e800e400470091017800f5
:1073ac001200200080007800b0c7b3001efd07005b
:1073bc00004f78001e4078000080fa0000000600a4
:1073cc000c00fa0068014700000978006a004700c9
:1073dc00010878008040eb00650047000148780008
:1073ec008040eb0066004700014878008000eb000d
:1073fc000e80e800010878008040eb006400470034
:10740c00014878006a004700100078000209070064
:10741c00004f78001e4078000004e00003003200aa
:10742c0000c0eb00004f78001d00370065004700de
:10743c00ea004700910178002200200080007800cb
:10744c0080c7b30076fc0700004f78001e40780020
:10745c000004e00012003a0064004700e500470019
:10746c001148780066004700104078000080fb004f
:10747c00c800dd000e80e8000108780064004700b9
:10748c00104078000080fb008e80e80091007800ae
:10749c0080807000680047001000780001087800b8
:1074ac001e4078000080fa00000006000c00fa0074
:1074bc0064024700004a7800660047000108780023
:1074cc0068004700020878006a004700030878004b
:1074dc000040eb00004f78008000eb000e80e800cd
:1074ec00010878006a004700100078000000e000f6
:1074fc00060032006a004700100078007c00400053
:10750c00100078000000e00003003a0000c0eb001f
:10751c00004f78001e0037006a004700100078000a
:10752c007600400010007800610060000000e00070
:10753c00150032000e80e800ea0047009100780048
:10754c00ab170700004f78001e4078000004e000e5
:10755c000f003a000e80e80010007800ea004700a7
:10756c0011027800e800470091017800e60047001e
:10757c0011017800e400470091407800e117070002
:10758c00004f780002003700b0cfb300004f7800f6
:10759c001e4078000080fa00000006000a00fa0085
:1075ac000e82e800004a7800640047000108780069
:1075bc00660047000208780068004700030878005e
:1075cc000040eb00004f78008040eb000e00e8001c
:1075dc000148780068004700100078000000e000c7
:1075ec000600320068004700100078007e00400062
:1075fc00100078000000e0003f003a0000c0eb00f3
:10760c00004f780044003700680047009001780074
:10761c00120020006400470090007800f0c4b30012
:10762c0081fc0700004f78006800470010007800cc
:10763c000002b00010017800a00020000100200022
:10764c00020001001e4078000004e00024003a0013
:10765c000e80e800e800470091017800120020003d
:10766c0080007800e0c4b3006ffc0700004f780086
:10767c0068004700100078000002b000100178008c
:10768c00a000200001002000020001001e40780034
:10769c000004e00012003a000e00e80010407800f0
:1076ac008080fb0066004700100078000000e900b5
:1076bc00808f50000a0031006400470010007800f1
:1076cc008000e80064004700010878000e80e800a4
:1076dc00104078008040e8000e80e80001487800f7
:1076ec000e00e800104078008040e8000e00e80032
:1076fc000148780001003700000000000e00e8008f
:10770c00104078000080fb00e600470091007800f4
:10771c00810f5000bcff39001e4078000080fa0039
:10772c00000006000400fa008e80e8008008780053
:10773c000e80e8001000780037080700004f780032
:10774c001e4078000004e0000300320000c0eb0093
:10775c00004f78000e0037000e80e8001000780013
:10776c007600400010007800610060000000e0002e
:10777c00050032000e80e80010007800501707005a
:10778c00004f780002003700b0cfb300004f7800f4
:10779c001e4078000080fa00000006000600fa0087
:1077ac000e81e800000978006400470001087800a9
:1077bc00640047001000780017080700004f78009d
:1077cc001e4078000004e0000300320000c0eb0013
:1077dc00004f78002e00370064004700100078003e
:1077ec007600400010007800610060000000e000ae
:1077fc002500320064004700900178001200200040
:10780c000e80e80090007800d0c4b30006fc07009e
:10781c00004f780064004700100078000002b000b0
:10782c0010017800a00020000100200002000100df
:10783c001e4078000004e00015003a006400470088
:10784c0010007800c1160700004f78001e40780029
:10785c000004e0000e003a006400470010007800bd
:10786c00f6004000910078000110a1007600400065
:10787c00010878006400470010007800070007003a
:10788c00004f780002003700b0cfb300004f7800f3
:10789c001e4078000080fa00000006000600fa0086
:1078ac00e40047008008780064004700100078006e
:1078bc007700400010407800004040008040780085
:1078cc000e00e800014878008040eb000e80e800d4
:1078dc00014878000e00e8000000e800e4004700d2
:1078ec00910178001200200080007800c0c4b30021
:1078fc004bfb0700004f78001e4078000004e000ae
:10790c0030003a000e80e80010407800804078008b
:10791c000174a1006400470010007800760040005c
:10792c00100078000000d100614060000080fb0076
:10793c004700dd000040780000c0700080407800f7
:10794c000e80e800014878000e80e80010407800b6
:10795c0080407800c0cfb30080c060006400470056
:10796c001000780076004000100078004200de0025
:10797c00634060006340600000c07000804078008d
:10798c000e80e800014878000e00e800e400470093
:10799c00910178002200200080007800b0c4b30070
:1079ac00a1fb0700004f780064004700100078002e
:1079bc000002b00010017800a0002000010020009f
:1079cc00020001001e4078000080fa000000060052
:1079dc000600fa000e81e8000009780064004700f8
:1079ec000108780064004700100078008a0707003f
:1079fc00004f78001e4078000004e00003003200c5
:107a0c0000c0eb00004f78001900370064004700fd
:107a1c0010007800760040001000780061006000d3
:107a2c000000e000100032006400470010007800f5
:107a3c007600400010007800620060000000e0005a
:107a4c0009003a0064004700900178008200200091
:107a5c000e80e8009000780040c0b300f0fa0700f8
:107a6c00004f780002003700b0cfb300004f780011
:107a7c001e4078000080fa00000006000600fa00a4
:107a8c000e81e80000497800640047000108780086
:107a9c008040eb000e00e8000148780064004700cd
:107aac00100078005c070700004f78001e4078003b
:107abc000004e0000300320000c0eb00004f78002f
:107acc00300037000e80e800104078000080fb008a
:107adc00e10f500003003200e20f500006003200ac
:107aec001600370064004700100078006f1b070079
:107afc00004f780015003700640047001000780034
:107b0c0051c1b3006e00400001487800640047008a
:107b1c00100078009efc0700004f78001e40780093
:107b2c000004e00008003a006400470010007800f0
:107b3c001a1c0700004f780004003700b0cfb300c8
:107b4c00004f780001003700000000001e40780054
:107b5c000004e000060035000e00e8001e48780026
:107b6c0064004700100078001ffc0700004f7800ed
:107b7c001e4078000004e00002003a000e00e8000d
:107b8c00104f78001e4078000080fa0000000600bc
:107b9c000800fa00e6004700800878000040eb007f
:107bac00004f78008000eb0064004700010878006b
:107bbc008000eb000e80e8000108780066004700aa
:107bcc00100078000000e00007003200660047005b
:107bdc00100078007a004000100078001000780047
:107bec000000e00003003a0000c0eb00004f7800fa
:107bfc00520037006600470010007800071d070090
:107c0c0064004700e600470091007800251d07003e
:107c1c00004f78001e4078000004e00047003a0056
:107c2c0066004700100078007a0040009000780051
:107c3c000e80e8008180e80011087800660047009b
:107c4c00100078007a004000100078000080e800f6
:107c5c00900078006400470010007800808f50007e
:107c6c000800360066004700100078007a004000db
:107c7c009000780064004700100178000180e80053
:107c8c000208780066004700100078007a00400077
:107c9c00100078006400400010407800e24f500063
:107cac0014003a006400470010007800790040008e
:107cbc008e80e80091007800810f50000d003e008e
:107ccc0066004700100078007a0040001001780030
:107cdc0066004700100078007a0040001000780021
:107cec000080e80010007800f90040000280e800f5
:107cfc000108780066004700100078007a00400008
:107d0c00100078000080e8009000780066004700c2
:107d1c00100078007a004000100078001000780005
:107d2c00660147009201780001017800800078001c
:107d3c0040c2b3003afa0700004f78001e407800aa
:107d4c000080fa00000006000600fa00e40047007c
:107d5c00800878000040eb00004f780001cbb300a6
:107d6c000e80e80001487800e1c7b3000e00e8007f
:107d7c000148780064004700100078000000e00023
:107d8c0003003a0000c0eb00004f780009003700f8
:107d9c000e80e800e40047009101780012002000fa
:107dac00800078000e00e800104078009efa070072
:107dbc00004f78001e4078000080fa00000006009a
:107dcc000800fa00e401470080497800650047008c
:107ddc000148780066004700020878000040eb007c
:107dec00004f78008040eb006300470001487800aa
:107dfc0071c4b3000e00e80001487800640047002d
:107e0c0010407800804078000104a1000e80e8004a
:107e1c000148780066004700100078000000e00080
:107e2c0003003a0000c0eb00004f78005900370007
:107e3c0063004700e6004700910178001200200023
:107e4c00800078000e00e80010407800f4f907007c
:107e5c00004f78001e4078000004e0004d003a000e
:107e6c000e80e800104078000004e000150032009d
:107e7c006500470010407800e14f500008003a00c0
:107e8c0063004700904078000e80e80010407800b6
:107e9c0080c070006300470001487800090037007b
:107eac000e80e8001040780080c0ea0063004700b4
:107ebc001040780000c060008040780063004700ec
:107ecc000148780063004700e60047009101780004
:107edc0012002000800078000e00e80010407800ae
:107eec0051fa0700004f78001e4078000004e000b3
:107efc0028003a0063004700e60047009101780033
:107f0c0012002000800078000e00e800104078007d
:107f1c00c3f90700004f78001e4078000004e00011
:107f2c001c003a0066004700100078007a00400000
:107f3c00100178006300470010407800f0406000aa
:107f4c006500410001487800660047001000780089
:107f5c007a004000100178006300470090407800e0
:107f6c0000ceb30080c0600066004100014878007c
:107f7c0066004700100078007a004000100178007d
:107f8c006300470010407800e2406000640041004c
:107f9c00014878001e4078000080fa0000000600be
:107fac000800fa00640147000049780066004700a9
:107fbc00010878000040eb00004f78008040eb0097
:107fcc000e80e8000148780051c4b3000e00e800b0
:107fdc000148780066004700100078000000e000bf
:107fec0003003a0000c0eb00004f78001c00370083
:107ffc000e80e800e6004700910178001200200096
:10800c00800078000e00e8001040780084f907002a
:10801c00004f78001e4078000004e00010003a0089
:10802c000e80e80090407800640047001040780013
:10803c0080c070000e80e800014878000e80e800d7
:10804c00e6004700910178001200200080007800c3
:10805c000e00e80010407800f3f90700004f78009c
:10806c001e4078000080fa00000006000800fa00ac
:10807c006401470000497800660047000108780059
:10808c000040eb00004f78000e80e800e400470051
:10809c001148780061c4b3000e00e8000148780074
:1080ac0066004700100078000000e00003003a0072
:1080bc0000c0eb00004f7800090037000e80e8008c
:1080cc00e600470091017800120020008000780043
:1080dc000e00e80010407800d3f90700004f78003c
:1080ec001e4078000080fa00000006000e00fa0026
:1080fc00e8014700800978006a0047000108780011
:10810c006c004700020878000040eb00004f78003c
:10811c008000eb000e80e800010878008000eb0086
:10812c0064004700010878008040eb0066004700bf
:10813c00014878008040eb000e00e8000148780010
:10814c006c004700100078000000e0000d003200c9
:10815c006c004700100078007a0040001000780096
:10816c000000e000070032006c00470010007800af
:10817c007a00400010007800100078000000e00049
:10818c0003003a0000c0eb00004f780041003700bc
:10819c006c004700100078007a0040001000780056
:1081ac0065004000104078000004e00032003a0006
:1081bc00e40047000e80e8006c0147009201780053
:1081cc006a01470012017800dc1b0700160037001b
:1081dc000e80e800ec00470091007800272507008e
:1081ec006c004700100078007a0040009000780086
:1081fc000e00e800e680400011487800e6004700d9
:10820c000e80e8006c014700120278000e01e800b5
:10821c0092417800010178008000780068004700e6
:10822c0010007800431c07000e80e80090007800d6
:10823c006400470010007800808f5000e4ff390084
:10824c006600470010407800ea0047009100780073
:10825c00804878006c004700100078007a004000dd
:10826c00900078000e80e8001001780068804000d3
:10827c0002087800070037006c00470010017800f6
:10828c006a004700900078006800470010007800f2
:10829c00db1d07001e4078000080fa00000006007d
:1082ac000e00fa00e8014700800978006a004700d8
:1082bc00010878006c004700020878000040eb00d1
:1082cc00004f78008000eb000e80e8000108780079
:1082dc008000eb0064004700010878008040eb0050
:1082ec0066004700014878008040eb000e00e80073
:1082fc00014878006c004700100078000000e00096
:10830c00070032006c004700100078007a00400033
:10831c0010007800100078000000e00003003a0024
:10832c0000c0eb00004f7800410037006c004700a4
:10833c00100078007a0040001000780065004000c2
:10834c00104078000004e00032003a00e4004700de
:10835c000e80e8006c014700920178006a0147002a
:10836c00120178008f1e0700160037000e80e800ff
:10837c00ec00470091007800c02407006c00470017
:10838c00100078007a004000900078000e00e800a1
:10839c00e680400011487800e60047000e80e800b7
:1083ac006c014700120278000e01e800924178003f
:1083bc000101780080007800680047001000780008
:1083cc00f61e07000e80e80090007800640047005d
:1083dc0010007800808f5000e4ff390066004700e1
:1083ec0010407800ea00470091007800804878003f
:1083fc006c004700100078007a0040009000780074
:10840c000e80e800100178006a80400002087800b5
:10841c00070037006c004700100178006a00470025
:10842c009000780068004700100078008d2007004d
:10843c001e4078000080fa00000006000e00fa00d2
:10844c00e8014700800978006a00470001087800bd
:10845c006c004700020878000040eb00004f7800e9
:10846c008000eb000e80e800010878008000eb0033
:10847c0064004700010878008040eb00660047006c
:10848c00014878008040eb000e00e80001487800bd
:10849c006c004700100078000000e0000b00320078
:1084ac006c004700100078007a0040001000780043
:1084bc00100078000000e000040032006800470063
:1084cc00100078000000e00003003a0000c0eb0050
:1084dc00004f7800410037006c0047001000780016
:1084ec007a004000100078006500400010407800d1
:1084fc000004e00032003a00e40047000e80e8007f
:10850c006c014700920178006a0147001201780063
:10851c003d210700160037000e80e800ec004700f4
:10852c0091007800552407006c004700100078007b
:10853c007a004000900078000e00e800e6804000d1
:10854c0011487800e60047000e80e8006c014700f7
:10855c00120278000e01e8009241780001017800c7
:10856c00800078006800470010007800a321070005
:10857c000e80e8009000780064004700100078003e
:10858c00808f5000e4ff39006600470010407800ef
:10859c00ea00470091007800804878006c004700a2
:1085ac00100078007a004000900078000e80e800ff
:1085bc00100178006c80400002087800070037003a
:1085cc006c004700100178006a00470090007800aa
:1085dc006800470010007800392307001e4078001f
:1085ec000080fa00000006000800fa008e81e80006
:1085fc008009780064004700010878006600470095
:10860c00020878006600470010007800820407001a
:10861c00004f78001e4078000004e0000300320098
:10862c0000c0eb00004f7800640037006600470084
:10863c00900078000e80e8001000780017250700e5
:10864c00004f78001e4078000004e0005b003a0008
:10865c000e00e800e60047009101780012002000af
:10866c008000780090c6b300edf70700004f78004b
:10867c000e00e80010407800804078000164a100f2
:10868c000e80e80010007800104078000080fb009d
:10869c004600dd00004078000044b20000c07000cd
:1086ac00804078000e00e800014878000e00e800d9
:1086bc001040780080407800f0ccb30080c060009f
:1086cc000e80e800100078000000e80010407800f0
:1086dc000080fb004400dd00004078000043b20045
:1086ec0000c07000804078000e00e800014878005f
:1086fc000e00e800104078008040780030cfb300c6
:10870c0080c060000e80e800100078000080e80057
:10871c00104078000080fb004200dd000040780033
:10872c006c40600000c07000804078000e00e800d3
:10873c00014878000e00e800104078008040780076
:10874c00c0cfb30080c060000e80e800100078003d
:10875c0063004000104078006340600000c070006f
:10876c00804078000e00e800014878001e40780038
:10877c000004e00011003a000e00e800e60047009b
:10878c0091017800120020008000780090c6b300a0
:10879c0025f80700004f78001e4078000004e00028
:1087ac0006003a006600470090007800640047001d
:1087bc0010007800fd240700004f78001e40780060
:1087cc000080fa00000006001600fa007201470053
:1087dc000009780074004700010878007400470015
:1087ec00100078000c040700004f78001e40780041
:1087fc000004e0000300320000c0eb00004f7800e2
:10880c00920037006a004700f4004700910178009d
:10881c00720020008000780010c7b30080f70700ba
:10882c00004f78006a00470010407800f2004700c3
:10883c0091007800804878006b0047001040780069
:10884c008040780072004700100078000000e800bb
:10885c00014878006c004700104078008040780098
:10886c0072004700100078000080e8000148780092
:10887c000e00e800ed00470011487800700047003a
:10888c0010407800e34060000e80e800014878005a
:10889c000e80e800104078000080fb00ce00dd0068
:1088ac0064004700010878000e00e80010407800d2
:1088bc000080fb00c600dd00660047000108780060
:1088cc0064004700900078006600470010007800b4
:1088dc0081007000680047000108780068004700bc
:1088ec00100078000000e00001003d00f003b00033
:1088fc004680de008000780072004700100078008f
:10890c0064004000010878000e00e800ee0047000b
:10891c001148780070004700104078000080fb0080
:10892c006c006000c280de000e80e8000148780018
:10893c000e80e800104078000080fb00ce00dd00c7
:10894c0064004700010878000e00e8001040780031
:10895c000080fb00c600dd006600470001087800bf
:10896c006400470090007800660047001000780013
:10897c00810070006800470001087800680047001b
:10898c00100078000000e00001003d00f003b00092
:10899c004680de00800078007200470010007800ee
:1089ac0066004000010878000e00e800ef00470068
:1089bc001148780070004700104078008080fb0060
:1089cc000003200000806000c480de000e80e80000
:1089dc00014878000e80e800104078000080fb0011
:1089ec00ce00dd0064004700010878000e00e800ae
:1089fc00104078000080fb00c600dd0066004700d8
:108a0c000108780064004700900078006600470079
:108a1c0010007800810070006800470001087800a1
:108a2c0068004700100078000000e00001003d00e5
:108a3c00f003b0004680de00800078007200470032
:108a4c001000780068004000010878001e40780093
:108a5c000080fa00000006001200fa00ec0147004a
:108a6c00800978006e00470001087800700047000c
:108a7c0002087800700047001000780066030700b9
:108a8c00004f78001e4078000004e0000300320024
:108a9c0000c0eb00004f78007c0037006e004700f0
:108aac001000780010407800804078006400470087
:108abc00014878006e004700100078000000e800c4
:108acc00104078008040780065004700014878002d
:108adc006e004700100078000080e800104078001d
:108aec008040780066004700014878006e0047001f
:108afc00100078006400400010007800804078007e
:108b0c0067004700014878006e00470010007800ad
:108b1c006600400010007800804078006800470034
:108b2c00014878006e004700100078006800400093
:108b3c0010007800804078006900470001487800f8
:108b4c006e00470010007800640040009000780030
:108b5c000030200000806000c880de000e00e800bd
:108b6c00014878006e004700100078006600400055
:108b7c00900078000030200000806000c880de008b
:108b8c000e80e800014878006e0047001000780065
:108b9c0068004000900078000030200000806000e9
:108bac00c880de006300470001487800630047007e
:108bbc00104078000080fb004400dd00804078000d
:108bcc000e80e800104078000080fb004200dd00c1
:108bdc000040780080c070000e00e8001040780063
:108bec0000c07000804078006a004700014878009f
:108bfc006a00470010407800804078000174a100a2
:108c0c006c004700100078006500400010407800b0
:108c1c000080fb004700dd000040780000c07000c1
:108c2c00804078006a004700014878006a004700dd
:108c3c0010407800804078000164a1006c0047006f
:108c4c001000780064004000104078000080fb00a9
:108c5c004600dd00004078000044b20000c0700007
:108c6c00804078006a0047000148780064004700a3
:108c7c00f00047009101780072002000800078001d
:108c8c0010c7b300e8f60700004f78001e407800cc
:108c9c000080fa00000006000600fa00e40047001d
:108cac008008780001cab3000e80e8000148780003
:108cbc000e00e800e400470091017800120020004b
:108ccc0080007800a0c6b30055f60700004f78006e
:108cdc001e4078000004e0003a003a000e00e80064
:108cec0010407800804078000114a0000e00e800cd
:108cfc00014878000e00e800e4004700910178007c
:108d0c001200200080007800a0c6b300c6f6070051
:108d1c00004f78001e4078000004e00029003a0063
:108d2c000e80e800e400470091017800120020005a
:108d3c0080007800e0c7b300bbf60700004f780056
:108d4c001e4078000004e0001e003a000e00e8000f
:108d5c00e4004700910178001200200080007800a8
:108d6c00b0c1b3002ef60700004f78001e4078000b
:108d7c000004e00013003a000e00e80010407800f8
:108d8c000080fb00700060004480de0080407800b2
:108d9c000e00e800014878000e00e8001040780052
:108dac00e14f5000070032006400470010007800cb
:108dbc000002b0001001780090012000010020009a
:108dcc00020001001e4078000080fa00000006003e
:108ddc000800fa008e81e8008009780064004700e2
:108dec000108780066004700020878000040eb009c
:108dfc00004f78000e80e80010007800ef0f500054
:108e0c000a003a006400470010007800e6004700b2
:108e1c00910178004200200080007800c0c1b300ae
:108e2c00fff50700004f78003c0037000e80e8008b
:108e3c001000780061006000004078000004e00041
:108e4c00090032006400470010007800e60047007b
:108e5c00910178001200200080007800c0c1b3009e
:108e6c00eff50700004f78000e80e8001000780046
:108e7c00620060000000e0000a003200640047005d
:108e8c00100078000000e800e6004700910178002f
:108e9c001200200080007800d0c1b300e0f507007c
:108eac00004f78000e80e80010007800640060002d
:108ebc000000e0000a003200640047001000780057
:108ecc000080e800e60047009101780012002000c5
:108edc0080007800e0c1b300d1f50700004f7800a6
:108eec000e80e80010007800680060000000e000d0
:108efc000a00320064004700100078006300400054
:108f0c00e6004700910178001200200080007800f4
:108f1c00f0c1b300c2f50700004f78001e40780086
:108f2c000080fa00000006000800fa006401470007
:108f3c0000097800660047000108780066004700c9
:108f4c001000780034020700004f78001e407800b3
:108f5c000004e00004003a006400470010007800b0
:108f6c000000e00003003a0000c0eb00004f780066
:108f7c00160037006400470010007800e60040003f
:108f8c000e80e80001087800660047009000780029
:108f9c000e80e80010007800a9090700004f780047
:108fac001e4078000004e00008003a00660047000c
:108fbc00100178000e80e8009000780064004700f3
:108fcc0010007800e30b0700004f78001e4078007b
:108fdc000080fa00000006000800fa006401470057
:108fec000009780066004700010878006600470019
:108ffc001000780008020700004f78001e4078002f
:10900c000004e00004003a006400470010007800ff
:10901c000000e00003003a0000c0eb00004f7800b5
:10902c00210037006400470010007800e600400083
:10903c000e80e800010878006600470010017800f7
:10904c000e80e80090007800640047001000780063
:10905c001e0f0700004f78001e4078000004e0004f
:10906c0011003a0066004700900078006400470049
:10907c0010007800d1010700004f78001e407800e6
:10908c000004e00008003a00660047001001780078
:10909c000e80e80090007800640047001000780013
:1090ac005f0f0700004f78001e4078000080fa0028
:1090bc00000006000600fa000e81e80000097800a6
:1090cc006400470001087800640047001000780035
:1090dc00d1010700004f78001e4078000004e0002a
:1090ec0004003a000e80e800100078000000e00058
:1090fc0003003a0000c0eb00004f78001600370068
:10910c006400470010007800c40b0700004f780083
:10911c001e4078000004e0000f003a006400470095
:10912c00900078000e80e80010007800a301070082
:10913c00004f78001e4078000004e00006003a0062
:10914c0064004700900078000e80e8001000780062
:10915c00800a0700004f78001e4078000080fa005b
:10916c00000006000800fa006401470000097800be
:10917c006600470001087800660047001000780080
:10918c00a5010700004f78001e4078000004e000a5
:10919c0004003a0064004700100078000000e00072
:1091ac0003003a0000c0eb00004f780016003700b7
:1091bc006400470010007800e60040000e80e800d4
:1091cc000108780066004700900078000e80e800e7
:1091dc0010007800ee0c0700004f78001e4078005d
:1091ec000004e00008003a00660047001001780017
:1091fc000e80e800900078006400470010007800b2
:10920c00270d0700004f78001e4078000080fa0000
:10921c00000006000800fa0064014700000978000d
:10922c0066004700010878006600470010007800cf
:10923c0079010700004f78001e4078000004e00020
:10924c0004003a0064004700100078000000e000c1
:10925c0003003a0000c0eb00004f78001600370006
:10926c006400470010007800e60040000e80e80023
:10927c000108780066004700900078000e80e80036
:10928c0010007800900b0700004f78001e4078000b
:10929c000004e00008003a00660047001001780066
:1092ac000e80e80090007800640047001000780001
:1092bc00dc0b0700004f78001e4078000080fa009d
:1092cc00000006000800fa0064014700000978005d
:1092dc00660047000108780066004700100078001f
:1092ec004d010700004f78001e4078000004e0009c
:1092fc0004003a0064004700100078000000e00011
:10930c0003003a0000c0eb00004f78002600370045
:10931c006400470010007800e60040000e80e80072
:10932c000108780066004700900078000e80e80085
:10933c0010007800a80d0700004f78001e40780040
:10934c000004e00018003a00660047009000780026
:10935c00640047001000780018010700004f7800e7
:10936c001e4078000004e0000f003a006600470041
:10937c009000780064004700100078005509070041
:10938c00004f78001e4078000004e00006003a0010
:10939c0066004700900078000e80e800100078000e
:1093ac00c20d0700004f78001e4078000080fa00c4
:1093bc00000006000800fa0064014700000978006c
:1093cc00660047000108780066004700100078002e
:1093dc0011010700004f78001e4078000004e000e7
:1093ec0004003a0064004700100078000000e00020
:1093fc0003003a0000c0eb00004f78002600370055
:10940c006400470010007800e60040000e80e80081
:10941c000108780066004700900078000e80e80094
:10942c0010007800cc100700004f78001e40780028
:10943c000004e00018003a00660047009000780035
:10944c006400470010007800dc000700004f780033
:10945c001e4078000004e0000f003a006600470050
:10946c00900078006400470010007800190907008c
:10947c00004f78001e4078000004e00006003a001f
:10948c0066004700900078000e80e800100078001d
:10949c00e8100700004f78001e4078000080fa00aa
:1094ac00000006000800fa0064014700000978007b
:1094bc00660047000108780066004700100078003d
:1094cc00d5000700004f78001e4078000004e00033
:1094dc0004003a0064004700100078000000e0002f
:1094ec0003003a0000c0eb00004f78002600370064
:1094fc006400470010007800e60040000e80e80091
:10950c000108780066004700900078000e80e800a3
:10951c00100078006a110700004f78001e40780098
:10952c000004e00018003a00660047009000780044
:10953c006400470010007800a0000700004f78007e
:10954c001e4078000004e0000f003a00660047005f
:10955c00900078006400470010007800dd080700d8
:10956c00004f78001e4078000004e00006003a002e
:10957c0066004700900078000e80e800100078002c
:10958c0084110700004f78001e4078000080fa001c
:10959c00000006000800fa0064014700000978008a
:1095ac00660047000108780066004700100078004c
:1095bc0099000700004f78001e4078000004e0007e
:1095cc0004003a0064004700100078000000e0003e
:1095dc0003003a0000c0eb00004f78002f0037006a
:1095ec006400470010007800e60040000e80e800a0
:1095fc000108780066004700900078000e80e800b3
:10960c0010007800cd110700004f78001e40780044
:10961c000004e00021003a0066004700900078004a
:10962c00640047001000780064000700004f7800c9
:10963c001e4078000004e00018003a006600470065
:10964c00900078006400470010007800a108070023
:10965c00004f78001e4078000004e0000f003a0034
:10966c0066004700900078000e80e800100078003b
:10967c00ea110700004f78001e4078000004e0005b
:10968c0006003a0066004700900078000e80e80063
:10969c001000780018120700004f78001e40780068
:1096ac000080fa00000006000800fa006401470080
:1096bc000009780066004700010878006600470042
:1096cc001000780054000700004f78001e4078000e
:1096dc000004e00004003a00640047001000780029
:1096ec000000e00003003a0000c0eb00004f7800df
:1096fc002f0037006400470010007800e60040009f
:10970c000e80e800010878006600470090007800a1
:10971c000e80e8001000780053120700004f78000c
:10972c001e4078000004e00021003a00660047006b
:10973c009000780064004700100078001f000700bc
:10974c00004f78001e4078000004e00018003a003a
:10975c006600470090007800640047001000780015
:10976c005c080700004f78001e4078000004e00001
:10977c000f003a0066004700900078000e80e80069
:10978c001000780094120700004f78001e407800fb
:10979c000004e00006003a006600470090007800e4
:1097ac000e80e80010007800c0120700004f78000f
:1097bc001e4078000080fa00000006000600fa0047
:1097cc000e81e80000097800640047000108780069
:1097dc0064004700900078000e80e80010007800cc
:1097ec00f9120700004f78001e4078000004e000da
:1097fc0006003a0064004700900078000e80e800f4
:10980c0010007800c0130700004f78001e4078004d
:10981c000080fa00000006000400fa008e80e800c8
:10982c00800878000e80e800100078000000e0004e
:10983c00120032000e80e800100078007c0040001e
:10984c00100078000000e0000c0032000e80e800f0
:10985c00100078007e004000100078000000e0004e
:10986c00060032000e80e800100078000002b00004
:10987c00100078000000e00003003a0000c0eb008c
:10988c00004f7800020037000040eb00004f7800da
:10989c001e4078000080fa00000006000200fa006a
:1098ac00000f78001e00780021c0b3006900400052
:1098bc00014878001e00780081c0b30067004000aa
:1098cc00014878001e00780001c1b300660040001a
:1098dc00014878001e00780031c0b30068004000d9
:1098ec00014878001e00780021c0b30071004000d0
:1098fc00014878001e00780081c0b3006f00400062
:10990c00014878001e00780041c1b3006e00400091
:10991c00014878001e0078008040eb007000400089
:10992c00014878001e0078009e0078006a00400014
:10993c00e680400031187800211078001e00780075
:10994c009e00780072004000ee80400031187800d4
:10995c00211078000080fa00000006000600fa00d2
:10996c00e400470080087800e1004700010009008e
:10997c008058eb000e00e800e400470091007800ee
:10998c0036000700004f78001e4078000004e0000d
:10999c002f003a000e00e800e40047009101780027
:1099ac00120020008000780000c4b3009ef3070072
:1099bc00004f78001e4078000004e00024003a00bc
:1099cc006400470010007800670040009040780069
:1099dc0064004700100078006b00400001487800dc
:1099ec006400470010007800690040009040780047
:1099fc0064004700100078006d00400001487800ba
:109a0c000e00e8000000e800e40047009101780037
:109a1c00120020008000780010c4b30082f307000d
:109a2c00004f78001e4078000004e00008003a0067
:109a3c0064004700100078006800400090407800f7
:109a4c0064004700100078006c004000014878006a
:109a5c001e4078000080fa00000006000600fa00a4
:109a6c000e81e800000978006400470001087800c6
:109a7c006400470090017800220020000e80e8006e
:109a8c009000780000c4b300e5f20700004f7800a6
:109a9c001e4078000004e00019003a006400470002
:109aac00900078000e80e800100078001700070086
:109abc00004f78001e4078000004e00010003a00cf
:109acc0064004700900078000e80e80010007800d9
:109adc0046000700004f78001e4078000004e000ac
:109aec0007003a000e80e800100078000000e80043
:109afc00e4004700910078006f000700004f7800e9
:109b0c001e4078000080fa00000006000800fa00f1
:109b1c0064014700000978006600470001087800de
:109b2c000040eb00004f78008040eb000e00e80096
:109b3c00014878008040eb000e80e8000148780076
:109b4c006600470010007800670040001040780065
:109b5c00ef4f500020003e006600470010007800d8
:109b6c0067004000904078006600470010007800c5
:109b7c006b0040001040780080cf5000180032007d
:109b8c0066004700900078000e80e800e7804000f7
:109b9c00114878006400470010007800904078006d
:109bac0000cfb30080c060000e00e80001487800d0
:109bbc000e80e80010407800ef4060000e00e800d6
:109bcc001040780000c07000e4004700910078005d
:109bdc008048780002003700c0cfb300004f7800f7
:109bec001e4078000080fa00000006000800fa0011
:109bfc0064014700000978006600470001087800fe
:109c0c000040eb00004f78008040eb000e00e800b5
:109c1c00014878008040eb000e80e8000148780095
:109c2c006600470010007800690040001040780082
:109c3c00e24f50001b003e00660047001000780009
:109c4c0069004000904078006600470010007800e2
:109c5c006d0040001040780080cf5000130032009f
:109c6c0066004700900078000e80e800e980400014
:109c7c00114878006400470010007800904078008c
:109c8c00f0c8b30080c060000e00e8000148780006
:109c9c0064004700900078000e00e80090487800bf
:109cac0002003700c0cfb300004f78001e40780090
:109cbc000080fa00000006000800fa00640147006a
:109ccc000009780066004700010878000040eb00ae
:109cdc00004f78008040eb000e00e800014878004f
:109cec008040eb000e80e8000148780066004700d9
:109cfc00100078006800400010407800ec4f5000d5
:109d0c0020003e006600470010007800680040000c
:109d1c009040780066004700100078006c0040000e
:109d2c001040780080cf50001800320066004700c9
:109d3c00900078000e80e800e88040001148780020
:109d4c0064004700100078009040780000cfb3000a
:109d5c0080c060000e00e800014878000e80e8002a
:109d6c0010407800ef4060000e00e80010407800d2
:109d7c0000c07000e4004700910078008048780033
:109d8c0002003700c0cfb300004f78001e407800af
:109d9c000080fa00000006000400fa008e80e80043
:109dac00800878008040eb000e00e8000148780045
:109dbc000e00e8008e80e80091017800120020006f
:109dcc008000780020c0b30015f20700004f780027
:109ddc000e00e800104078000080fb000000d1006d
:109dec00804078000e00e800014878000e00e80082
:109dfc0010407800ef4060000e00e8000148780049
:109e0c000e00e80010407800e14f500003003a00cb
:109e1c00a0cfb300004f7800140037000e00e8000c
:109e2c0010407800e24f500003003a0090cfb3008e
:109e3c00004f78000d0037000e00e800104078004d
:109e4c00e34f500003003a0080cfb300004f78007e
:109e5c00060037000e00e80010407800e74f500075
:109e6c0002003a0070cfb300004f78001e4078001b
:109e7c000080fa00000006000600fa00e40047002b
:109e8c0080087800e1004700010009008058eb00d1
:109e9c000e00e800e400470091007800360007004f
:109eac00004f78001e4078000004e0002f003a00bc
:109ebc000e00e800e4004700910178001200200039
:109ecc008000780020c4b30057f20700004f7800e0
:109edc001e4078000004e00024003a0064004700b3
:109eec00100078006f00400090407800640047003c
:109efc0010007800730040000148780064004700af
:109f0c001000780071004000904078006400470019
:109f1c001000780075004000014878000e00e80041
:109f2c000000e800e40047009101780012002000d6
:109f3c008000780030c4b3003bf20700004f78007b
:109f4c001e4078000004e00008003a00640047005e
:109f5c0010007800700040009040780064004700ca
:109f6c001000780074004000014878001e40780012
:109f7c000080fa00000006000600fa000e81e800de
:109f8c00000978006400470001087800640047006d
:109f9c0090017800220020000e80e80090007800ec
:109fac0020c4b3009ef10700004f78001e407800db
:109fbc000004e00019003a006400470090007800ab
:109fcc000e80e8001000780017000700004f7800a2
:109fdc001e4078000004e00010003a0064004700c6
:109fec00900078000e80e800100078004600070012
:109ffc00004f78001e4078000004e00007003a0093
:10a00c000e80e800100078000000e800e400470033
:10a01c00910078006e000700004f78001e40780019
:10a02c000080fa00000006000800fa0064014700f6
:10a03c000009780066004700010878000040eb003a
:10a04c00004f78008040eb000e00e80001487800db
:10a05c008040eb000e80e800014878006600470065
:10a06c00100078006f00400010407800ed4f500059
:10a07c0020003e0066004700100078006f00400092
:10a08c009040780066004700100078007300400094
:10a09c001040780080cf5000180032006600470056
:10a0ac00900078000e80e800ef80400011487800a6
:10a0bc0064004700100078009040780000cfb30097
:10a0cc0080c060000e00e800014878000e80e800b7
:10a0dc0010407800ef4060000e00e800104078005f
:10a0ec0000c07000e40047009100780080487800c0
:10a0fc0002003700c0cfb300004f78001e4078003c
:10a10c000080fa00000006000800fa006401470015
:10a11c000009780066004700010878000040eb0059
:10a12c00004f78008040eb000e00e80001487800fa
:10a13c008040eb000e80e800014878006600470084
:10a14c00100078007100400010407800e24f500081
:10a15c001a003e0066004700900078000e80e80070
:10a16c00f18040001148780064004700100078002e
:10a17c0090407800f0ccb30080c060000e00e80086
:10a18c00014878000e80e800104078000080fb0049
:10a19c004400dd000040780002c3b3008240600040
:10a1ac000e00e8001040780000c07000e40047008a
:10a1bc00910078008048780002003700c0cfb300cf
:10a1cc00004f78001e4078000080fa000000060066
:10a1dc000800fa0064014700000978006600470097
:10a1ec00010878000040eb00004f78008040eb0045
:10a1fc000e00e800014878008040eb000e80e8007b
:10a20c00014878006600470010007800700040009c
:10a21c0010407800e44f500020003e0066004700dc
:10a22c0010007800700040009040780066004700f5
:10a23c0010007800740040001040780080cf50006f
:10a24c001800320066004700900078000e80e8008d
:10a25c00f08040001148780064004700100078003e
:10a26c009040780080cfb30080c060000e00e80002
:10a27c00014878000e80e80010407800e74060004c
:10a28c000e00e8001040780000c07000e4004700a9
:10a29c00910078008048780002003700c0cfb300ee
:10a2ac00004f78001e4078000080fa000000060085
:10a2bc000400fa008e80e800800878000040eb0073
:10a2cc00004f78008040eb000e00e8000148780059
:10a2dc000e80e80010007800660040001040780006
:10a2ec00ef4f5000380036000e80e8001000780068
:10a2fc006600400010407800f24f500032003e00e3
:10a30c000e80e80010007800660040009040780055
:10a31c000e80e800100078006a00400010407800c1
:10a32c0080cf50002c0032000e00e8008e80e80038
:10a33c00910078002b000700004f78001e40780039
:10a34c000004e00023003a000e80e80010007800c2
:10a35c00660040008e80e800910178001200200019
:10a36c0080007800e0c7b3002ff10700004f7800a1
:10a37c000e80e800100078006a0040001040780061
:10a38c00f04f500007003a000e80e80010007800f3
:10a39c000002b000100178005000200001002000e5
:10a3ac00020001000e80e8001000780066004000fa
:10a3bc00904078000e80e800100078006a004000a1
:10a3cc000148780004003700c0cfb300004f78007c
:10a3dc0001003700000000001e4078000080fa00e9
:10a3ec00000006000800fa0064014700000978002c
:10a3fc0066004700010878008040eb000e00e80082
:10a40c00014878008040eb000e80e800014878009d
:10a41c00660047009001780012002000640047009d
:10a42c009000780000c4b3007df00700004f780066
:10a43c001e4078000004e0003f003a006600470030
:10a44c00100078006600400010407800f24f500079
:10a45c0021003a006400470010007800104078009a
:10a46c00804078000174a1000e00e80001487800db
:10a47c000e00e800104078000074a000e4004700d3
:10a48c0091007800804878006600470090017800c1
:10a49c0012002000640047009000780000c4b30054
:10a4ac00e1f00700004f78001e4078000004e00047
:10a4bc0021003a000e80e800e60047009101780088
:10a4cc00220020008000780080c5b300d6f0070081
:10a4dc00004f780018003700640047001000780027
:10a4ec00104078000004e00013003d0064004700b9
:10a4fc001000780010407800804078000174a100b2
:10a50c000e00e800014878006400470090007800d5
:10a51c000e00e80090487800660047009001780033
:10a52c0012002000640047009000780000c4b300c3
:10a53c00bdf00700004f78001e4078000080fa0044
:10a54c00000006000400fa008e80e8008008780005
:10a55c000040eb00004f78000e80e80010007800ff
:10a56c006e00400010407800f44f50000c00320098
:10a57c000e80e800100078006e004000104078005b
:10a58c00f54f5000060032000e80e80010007800f5
:10a59c006e00400010407800f74f50003e003a002b
:10a5ac000e80e800100078006e00400090407800ab
:10a5bc000e80e80010007800720040001040780017
:10a5cc0080cf5000360032000e80e800100078007a
:10a5dc006e0040008e80e80091017800120020008f
:10a5ec0080007800e0c7b3008ff00700004f7800c0
:10a5fc000e80e800100078007200400010407800d7
:10a60c00f44f500008003a000e80e800100078006b
:10a61c000002b0001001780010052000010020009d
:10a62c0002000100130037000e80e80010007800d3
:10a63c007200400010407800f74f50000d003a00b7
:10a64c000e80e800100078006e004000104078008a
:10a65c00f54f500007003a000e80e800100078001b
:10a66c000002b00010017800a000200001002000c2
:10a67c00020001000e80e800100078006e0040001f
:10a68c00904078000e80e8001000780072004000c6
:10a69c000148780002003700c0cfb300004f7800ab
:10a6ac001e4078000080fa00000006001e00fa0030
:10a6bc00f8014700804978007a00470001087800cb
:10a6cc007c004700020878008040eb000e00e80098
:10a6dc0001487800ee004700030009008018eb00e9
:10a6ec008058eb008040eb000e80e80001487800b9
:10a6fc008000eb0064004700010878006000b8009f
:10a70c00660147000089be007800470010407800c1
:10a71c000080fb0066004000800078006e0047005f
:10a72c007c014700920178000101780080007800dc
:10a73c0020c1b300baef0700004f78001e4078002c
:10a74c000004e000bc003a000e00e8001040780065
:10a75c000080fb00800047006a004700ee8040004c
:10a76c00114878000e00e800104078008040e800a6
:10a77c000e00e800014878000e00e8001040780058
:10a78c000080fb00800047006b004700ee8040001b
:10a79c00114878000e00e800104078008040e80076
:10a7ac000e00e800014878006b004700104078006c
:10a7bc000080fb00c800dd006a00470010407800f4
:10a7cc000080fb00810070006c00470001087800dd
:10a7dc007a004700900078006c00470090087800e1
:10a7ec000e00e800104078000080fb00800047005d
:10a7fc006a004700ee804000114878000e00e80027
:10a80c00104078008040e8000e00e8000148780015
:10a81c000e00e800104078000080fb00800047002c
:10a82c006b004700ee804000114878000e00e800f5
:10a83c00104078008040e8000e00e80001487800e5
:10a84c006b004700104078000080fb00c800dd0062
:10a85c006a004700104078000080fb008100700007
:10a86c006c004700010878007a004700100078005f
:10a87c000080e800ec004700110878000e00e800aa
:10a88c00104078000080fb00800047006a00470001
:10a89c00ee804000114878000e00e800104078006f
:10a8ac008040e8000e00e800014878000e00e80047
:10a8bc00104078000080fb00800047006b004700d0
:10a8cc00ee804000114878000e00e800104078003f
:10a8dc008040e8000e00e800014878006b0047005b
:10a8ec00104078000080fb00c800dd006a004700c3
:10a8fc00104078000080fb00810070006c00470065
:10a90c00010878007a0047001000780064004000cd
:10a91c00ec004700110878007800470010407800e0
:10a92c00e34f50003e003a000e00e8001040780063
:10a93c000080fb00800047000e80e800ee804000a5
:10a94c00114878000e00e800104078008040e800c4
:10a95c000e00e800014878000e00e8001040780076
:10a96c000080fb00000047006e00400010407800a3
:10a97c000080fb00c800dd0064004700010878007f
:10a98c000e00e800104078008040e8000e00e8005f
:10a99c00014878000e00e800104078000080fb00b1
:10a9ac00000047006e004000104078000080fb0063
:10a9bc008000eb00c000dd000000200066014700b5
:10a9cc000089be000e00e800104078008040e800ce
:10a9dc000e00e80001487800640047001000780081
:10a9ec006101b800660047001000be000001710054
:10a9fc00818171000e80e800104078000080fb001f
:10aa0c008000eb0000007100818071007a0147002a
:10aa1c0012017800660141000089be000800370071
:10aa2c007a004700100178006000b8006601410010
:10aa3c000089be0002003700e0cfb300004f780061
:10aa4c001e4078000080fa00000006002400fa0086
:10aa5c00fe01470080497800000220000e004000f3
:10aa6c0001087800200220000e0040000208780047
:10aa7c008040eb000e00e80001487800ee00470033
:10aa8c00060009008018eb008058eb008040eb00ba
:10aa9c000e80e800014878008000eb00640047005d
:10aaac00010878006000b800660147000089be000c
:10aabc007e004700104078000004e0008d003a0052
:10aacc006e004700210220008e804000910178002a
:10aadc006200200080007800c0c0b300d0ee0700f8
:10aaec00004f78001e4078000004e0007e003a0021
:10aafc000e00e800104078000080fb00800047004a
:10ab0c006a004700ee804000114878000e00e80013
:10ab1c00104078008040e8000e00e8000148780002
:10ab2c000e00e800104078000080fb008000470019
:10ab3c006b004700ee804000114878000e00e800e2
:10ab4c00104078008040e8000e00e80001487800d2
:10ab5c006b004700104078000080fb00c800dd004f
:10ab6c006a004700104078000080fb0081007000f4
:10ab7c006c00470001087800000220000e00400025
:10ab8c00900078006c004700900878000e00e800f8
:10ab9c00104078000080fb00800047006a004700ee
:10abac00ee804000114878000e00e800104078005c
:10abbc008040e8000e00e800014878000e00e80034
:10abcc00104078000080fb00800047006b004700bd
:10abdc00ee804000114878000e00e800104078002c
:10abec008040e8000e00e800014878006b00470048
:10abfc00104078000080fb00c800dd006a004700b0
:10ac0c00104078000080fb00810070006c00470051
:10ac1c0001087800000220000e00400010007800af
:10ac2c000080e800ec004700110878000e00e800f6
:10ac3c00104078000080fb00800047006a0047004d
:10ac4c00ee804000114878000e00e80010407800bb
:10ac5c008040e8000e00e800014878000e00e80093
:10ac6c00104078000080fb00800047006b0047001c
:10ac7c00ee804000114878000e00e800104078008b
:10ac8c008040e8000e00e800014878006b004700a7
:10ac9c00104078000080fb00c800dd006a0047000f
:10acac00104078000080fb00810070006c004700b1
:10acbc0001087800000220000e004000100078000f
:10accc0064004000ec0047001108780000022000ee
:10acdc000e004000100178006000b80066014100d1
:10acec000089be00d1003700e0cfb300004f7800e0
:10acfc00ce0037007e004700104078000080fb003b
:10ad0c006c004000800078006e004700220220009a
:10ad1c000e0141009201780001017800800078005a
:10ad2c00c0c0b3003eee0700004f78001e40780014
:10ad3c000004e000bb003a000e00e8001040780070
:10ad4c000080fb00800047006a004700ee80400056
:10ad5c00114878000e00e800104078008040e800b0
:10ad6c000e00e800014878000e00e8001040780062
:10ad7c000080fb00800047006b004700ee80400025
:10ad8c00114878000e00e800104078008040e80080
:10ad9c000e00e800014878006b0047001040780076
:10adac000080fb00c800dd006a00470010407800fe
:10adbc000080fb00810070006c00470001087800e7
:10adcc00000220000e004000900078006c0047004c
:10addc00900878000e00e800104078000080fb001e
:10adec00800047006a004700ee8040001148780060
:10adfc000e00e800104078008040e8000e00e800eb
:10ae0c00014878000e00e800104078000080fb003c
:10ae1c00800047006b004700ee804000114878002e
:10ae2c000e00e800104078008040e8000e00e800ba
:10ae3c00014878006b004700104078000080fb0050
:10ae4c00c800dd006a004700104078000080fb005d
:10ae5c00810070006c00470001087800000220009f
:10ae6c000e004000100078000080e800ec00470065
:10ae7c00110878000e00e800104078000080fb00fc
:10ae8c00800047006a004700ee80400011487800bf
:10ae9c000e00e800104078008040e8000e00e8004a
:10aeac00014878000e00e800104078000080fb009c
:10aebc00800047006b004700ee804000114878008e
:10aecc000e00e800104078008040e8000e00e8001a
:10aedc00014878006b004700104078000080fb00b0
:10aeec00c800dd006a004700104078000080fb00bd
:10aefc00810070006c0047000108780000022000ff
:10af0c000e0040001000780064004000ec00470088
:10af1c00110878000e00e80010407800e640400070
:10af2c000e00e800014878000e00e80010407800a0
:10af3c000080fb00800047000e80e800ee8040009f
:10af4c00114878000e00e800104078008040e800be
:10af5c000e00e800014878000e00e8001040780070
:10af6c000080fb00000047006e004000104078009d
:10af7c000080fb00c800dd00640047000108780079
:10af8c000e00e800104078008040e8000e00e80059
:10af9c00014878000e00e800104078000080fb00ab
:10afac00000047006e004000104078000080fb005d
:10afbc008000eb00c000dd000000200066014700af
:10afcc000089be000e00e800104078008040e800c8
:10afdc000e00e8000148780064004700100078007b
:10afec006101b800660047001000be00000171004e
:10affc00818171000e80e800104078000080fb0019
:10b00c008000eb00000071008180710002022000c2
:10b01c000e01410012017800660141000089be005a
:10b02c0002003700e0cfb300004f78001e407800dc
:10b03c000080fa00000006002600fa007e0247009d
:10b04c00004a7800000220000e0040000108780041
:10b05c00200220000e004000020878004002200070
:10b06c000e004000030878008040eb000e00e80062
:10b07c0001487800ee004700060009008018eb003c
:10b08c008058eb008040eb000e80e800014878000f
:10b09c008000eb0064004700010878006000b800f5
:10b0ac00660147000089be007e0047001040780012
:10b0bc000080fb006c004000800078006e004700b0
:10b0cc00420220000e01410092017800010178003b
:10b0dc0080007800c0c0b30051ed0700004f78002d
:10b0ec001e4078000004e00050013a000e00e80019
:10b0fc00104078000080fb00800047006a00470089
:10b10c00ee804000114878000e00e80010407800f6
:10b11c008040e8000e00e800014878000e00e800ce
:10b12c00104078000080fb00800047006b00470057
:10b13c00ee804000114878000e00e80010407800c6
:10b14c008040e8000e00e800014878006b004700e2
:10b15c00104078000080fb00c800dd006a0047004a
:10b16c00104078000080fb00810070006c004700ec
:10b17c0001087800200220000e00400090007800aa
:10b18c006c004700900878000e00e8001040780032
:10b19c000080fb00800047006a004700ee80400002
:10b1ac00114878000e00e800104078008040e8005c
:10b1bc000e00e800014878000e00e800104078000e
:10b1cc000080fb00800047006b004700ee804000d1
:10b1dc00114878000e00e800104078008040e8002c
:10b1ec000e00e800014878006b0047001040780022
:10b1fc000080fb00c800dd006a00470010407800aa
:10b20c000080fb00810070006c0047000108780092
:10b21c00200220000e004000100078000080e800a2
:10b22c00ec004700110878000e00e8001040780090
:10b23c000080fb00800047006a004700ee80400061
:10b24c00114878000e00e800104078008040e800bb
:10b25c000e00e800014878000e00e800104078006d
:10b26c000080fb00800047006b004700ee80400030
:10b27c00114878000e00e800104078008040e8008b
:10b28c000e00e800014878006b0047001040780081
:10b29c000080fb00c800dd006a0047001040780009
:10b2ac000080fb00810070006c00470001087800f2
:10b2bc00200220000e0040001000780064004000c6
:10b2cc00ec004700110878000e00e80010407800f0
:10b2dc000080fb00800047006a004700ee804000c1
:10b2ec00114878000e00e800104078008040e8001b
:10b2fc000e00e800014878000e00e80010407800cd
:10b30c000080fb00800047006b004700ee8040008f
:10b31c00114878000e00e800104078008040e800ea
:10b32c000e00e800014878006b00470010407800e0
:10b33c000080fb00c800dd006a0047001040780068
:10b34c000080fb00810070006c0047000108780051
:10b35c00000220000e004000900078006c004700b6
:10b36c00900878000e00e800104078000080fb0088
:10b37c00800047006a004700ee80400011487800ca
:10b38c000e00e800104078008040e8000e00e80055
:10b39c00014878000e00e800104078000080fb00a7
:10b3ac00800047006b004700ee8040001148780099
:10b3bc000e00e800104078008040e8000e00e80025
:10b3cc00014878006b004700104078000080fb00bb
:10b3dc00c800dd006a004700104078000080fb00c8
:10b3ec00810070006c00470001087800000220000a
:10b3fc000e004000100078000080e800ec004700d0
:10b40c00110878000e00e800104078000080fb0066
:10b41c00800047006a004700ee8040001148780029
:10b42c000e00e800104078008040e8000e00e800b4
:10b43c00014878000e00e800104078000080fb0006
:10b44c00800047006b004700ee80400011487800f8
:10b45c000e00e800104078008040e8000e00e80084
:10b46c00014878006b004700104078000080fb001a
:10b47c00c800dd006a004700104078000080fb0027
:10b48c00810070006c004700010878000002200069
:10b49c000e0040001000780064004000ec004700f3
:10b4ac00110878007e00470010407800e34f5000f0
:10b4bc0051003a000e00e800104078000080fb00bc
:10b4cc00800047000e80e800ee80400011487800b4
:10b4dc000e00e800104078008040e8000e00e80004
:10b4ec00014878000e00e800104078000080fb0056
:10b4fc00000047006e004000104078000080fb0008
:10b50c00c800dd0064004700010878000e00e80068
:10b51c00104078008040e8000e00e80001487800f8
:10b52c000e00e800104078000080fb00000047008f
:10b53c006e004000104078000080fb008000eb00a3
:10b54c00c000dd0000002000660147000089be003d
:10b55c000e00e800104078008040e8000e00e80083
:10b56c000148780064004700100078006101b800c1
:10b57c00660047001000be0000017100818171005f
:10b58c000e80e800104078000080fb008000eb008b
:10b59c000000710081807100020220000e01410048
:10b5ac0012017800660141000089be00640047006a
:10b5bc00100078006101b800660047001000be0062
:10b5cc0000017100818171000e80e800104078004c
:10b5dc000080fb008000eb00000071008180710096
:10b5ec00220220000e014100120178006601410088
:10b5fc000089be000f003700000220000e00400042
:10b60c00100178006000b800660141000089be009e
:10b61c00200220000e004000100178006000b800ed
:10b62c00660141000089be0002003700e0cfb30084
:10b63c00004f78001e4078000080fa0000000600e1
:10b64c000800fa0064014700000978006600470012
:10b65c00010878008040eb000e80e800014878007b
:10b66c008040eb000e00e800014878000e80e800f6
:10b67c00e60047009101780012002000800078005d
:10b68c0000c5b300e6eb0700004f78001e407800c1
:10b69c000004e0005b003a006400470010007800f2
:10b6ac0010407800614060000004e000420032006d
:10b6bc000e80e80010407800804078000104a10062
:10b6cc000e00e80001487800640047001000780084
:10b6dc001080fb000000d10061406000e140600080
:10b6ec000e00e8001040780000c070008040780028
:10b6fc000e80e800014878000e80e80010407800c9
:10b70c00804078000114a1000e00e8000148780088
:10b71c0064004700100078001080fb004200de003f
:10b72c00614060000080fb00000040000040780099
:10b73c00e24060000e00e8001040780000c070008d
:10b74c00804078000e80e800014878000e80e80008
:10b75c0010407800804078000124a1000e00e80021
:10b76c000148780064004700100078001080fb004e
:10b77c004300de00614060000080fb004200dd0001
:10b78c0000407800e44060000e00e80010407800b3
:10b79c0000c07000804078000e80e80001487800fe
:10b7ac0066004700100078008000eb006400400049
:10b7bc00010878000b0037000e80e80090407800fc
:10b7cc0080cfb30080c060000e80e8000148780094
:10b7dc0066004700100078008080eb006400400099
:10b7ec00010878000e80e800e6004700910178001f
:10b7fc00120020008000780000c5b3000aec07009e
:10b80c00004f78001e4078000080fa00000006000f
:10b81c000600fa00e4004700800878008040eb0046
:10b82c000e80e800014878008040eb000e00e80034
:10b83c00014878000e80e800e40047009101780090
:10b84c00120020008000780020c6b30074eb0700c3
:10b85c00004f78001e4078000004e0001a003a0007
:10b86c000e80e80010407800e24060000e00e80016
:10b87c00014878000e00e800104078000004e00059
:10b88c00110032000e80e8001040780080407800f3
:10b89c000114a1000e00e800014878000e80e800b9
:10b8ac008e00e800114878000e80e800e4004700a4
:10b8bc0091017800120020008000780020c6b300af
:10b8cc00d9eb0700004f78001e4078000080fa008a
:10b8dc00000006000c00fa0068014700000978001f
:10b8ec006a004700010878008040eb000e00e80079
:10b8fc00014878008040eb000e80e8000148780099
:10b90c008040eb0063004700014878008040eb006a
:10b91c0064004700014878008040eb006500470058
:10b92c00014878008040eb00660047000148780031
:10b93c000e00e800ea004700910178003200200078
:10b94c008000780050c5b30035eb0700004f78003d
:10b95c001e4078000004e0007b003a000e00e80076
:10b96c001040780080407800680047001000780094
:10b97c000080e8001001780060302b0002004000cd
:10b98c001040780000c0ea0000c0600080407800e1
:10b99c0064004700014878006300470010407800bd
:10b9ac008040780068004700100078000080e800b4
:10b9bc001001780060302b0002004000104078002d
:10b9cc0000c0ea0000c060008040780066004700bc
:10b9dc0001487800680047001000780010007800db
:10b9ec00e10f500010003200e10f5000050039004b
:10b9fc00e20f50001d003200e30f50002c0032000b
:10ba0c004400370064004700904078000e00e800c6
:10ba1c0001487800660047009040780063004700ba
:10ba2c00014878003d0037006400470090407800e2
:10ba3c0068004700100078000080e80010017800d2
:10ba4c0060302b00020040001040780080c0700075
:10ba5c000e00e8000148780066004700904078002e
:10ba6c0063004700014878002c003700660047004f
:10ba7c009040780068004700100078000080e800d3
:10ba8c001001780060302b0002004000104078005c
:10ba9c0080c07000630047000148780064004700d4
:10baac00904078000e00e800014878001b00370039
:10babc006400470090407800680047001000780050
:10bacc000080e8001001780060302b00020040007c
:10badc001040780080c070000e00e800014878002b
:10baec00660047009040780068004700100078001e
:10bafc000080e8001001780060302b00020040004c
:10bb0c001040780080c07000630047000148780046
:10bb1c0002003700c0cfb300004f78001e40780001
:10bb2c000004e00008003a000e00e800ea004700bc
:10bb3c0091017800320020008000780050c5b300dd
:10bb4c0039eb0700004f78001e4078000080fa00a7
:10bb5c00000006000800fa006401470000097800a4
:10bb6c0066004700010878008040eb000e80e8007a
:10bb7c00014878008040eb000e00e8000148780096
:10bb8c000e80e800e60047009101780012002000ca
:10bb9c008000780060c5b300a1ea0700004f780070
:10bbac001e4078000004e0006d003a00640047007d
:10bbbc00100078000080e8009000780060302b00c6
:10bbcc00010040001040780080c0ea000e80e800c0
:10bbdc001040780080c060000e00e800014878003a
:10bbec0064004700100078000080e80090007800a6
:10bbfc0060302b0001004000104078004400dd0054
:10bc0c0080c0ea000e00e8001040780080c06000a0
:10bc1c000e00e8000148780064004700100078002e
:10bc2c0010007800e10f50000b003200e10f5000c3
:10bc3c0005003900e20f500015003200e30f5000f0
:10bc4c0020003200390037000e80e8008e00e8003a
:10bc5c001148780037003700640047001000780066
:10bc6c000080e8009000780060302b00010040005c
:10bc7c0010407800c400dd000e00e8001040780091
:10bc8c0080c070000e80e800014878002900370061
:10bc9c0064004700100078000080e80090007800f5
:10bcac0060302b0001004000904078000e00e8004e
:10bcbc001040780080c070000e80e80001487800c9
:10bccc001c00370064004700100078000080e8007a
:10bcdc009000780060302b0001004000904078000c
:10bcec000e00e8001040780080c070000e80e80064
:10bcfc000148780064004700100078000080e800dc
:10bd0c009000780060302b0001004000104078005b
:10bd1c00c400dd000e80e8001040780080c0700088
:10bd2c000e80e8000148780002003700c0cfb30055
:10bd3c00004f78001e4078000004e00008003a0034
:10bd4c000e80e800e6004700910178001200200008
:10bd5c008000780060c5b300b3ea0700004f78009c
:10bd6c001e4078000080fa00000006000800fa006f
:10bd7c00640147000009780066004700010878005c
:10bd8c008040eb000e80e800014878008040eb001a
:10bd9c000e00e800014878000e80e800e60047003d
:10bdac0091017800120020008000780090c5b3004b
:10bdbc001bea0700004f78001e4078000004e000ea
:10bdcc001c003a000e80e80010407800804078009b
:10bddc000174a1000e00e8000148780064004700df
:10bdec00100078001080fb004600de00614060000f
:10bdfc000080fb004700dd00804078000e00e8006a
:10be0c001040780000c07000804078000e80e80080
:10be1c00014878000e80e800e600470091017800a8
:10be2c00120020008000780090c5b3007eea070065
:10be3c00004f78001e4078000080fa0000000600d9
:10be4c000a00fa0066014700000978006800470004
:10be5c00010878008040eb0063004700014878003f
:10be6c008040eb000e00e800014878008000eb00f9
:10be7c00640047000108780063004700e8004700b1
:10be8c00910178001200200080007800f0c5b3000a
:10be9c00e3e90700004f78001e4078000004e00042
:10beac0029003a0066004700100078001080fb0063
:10bebc004400de00e34060000e80e800014878009a
:10becc006300470090407800c0cfb30080c0600092
:10bedc000e00e800014878000e80e80090407800e1
:10beec0000c8b30080c060000e00e800104078006d
:10befc0000c0700080407800630047000148780063
:10bf0c0063004700904078006400470001487800c7
:10bf1c0066004700100078000000e80090407800b0
:10bf2c00650047000148780064004700e8004700be
:10bf3c00910178002200200080007800f0c5b30049
:10bf4c0039ea0700004f78001e4078000080fa00a4
:10bf5c00000006000800fa008e81e80080097800d5
:10bf6c00640047000108780066004700020878006a
:10bf7c0066004700900078000e80e8001000780002
:10bf8c000ef60700004f78001e4078000004e00019
:10bf9c001f003a0066004700100078001cfe0700e6
:10bfac00004f78001e4078000004e00018003a00b2
:10bfbc0066004700900078000e80e80010007800c2
:10bfcc0044fe0700004f78001e4078000004e0009b
:10bfdc000f003a00660047009000780064004700ac
:10bfec001000780061ff0700004f78001e407800b9
:10bffc000004e00006003a0066004700900078005c
:10c00c0064004700100078008dff0700004f780097
:10c01c001e4078000080fa00000006000600fa00be
:10c02c00e4004700800878008040eb000e80e800b8
:10c03c00014878008040eb000e00e80001487800d1
:10c04c000e80e800e4004700910178001200200007
:10c05c008000780010c5b30071e90700004f78002c
:10c06c001e4078000004e00014003a000e80e80046
:10c07c0010407800804078000144a1000e00e800d8
:10c08c00014878000e00e8001040780080407800ed
:10c09c000144a0000e80e800014878000e80e80002
:10c0ac00e400470091017800120020008000780025
:10c0bc0010c5b300dce90700004f78001e40780083
:10c0cc000080fa00000006000800fa006401470036
:10c0dc000009780066004700010878008040eb00fa
:10c0ec000e80e800014878008040eb000e00e8006c
:10c0fc00014878000e80e800e600470091017800c6
:10c10c00120020008000780020c5b30044e907002d
:10c11c00004f78001e4078000004e0003e003a001a
:10c12c006400470010007800100078006100600087
:10c13c000000e0000c0032000e80e8001040780097
:10c14c00804078000104a1000e00e800014878004e
:10c15c000e00e80010407800804078000104a00038
:10c16c000e80e80001487800640047001000780059
:10c17c0010007800620060000000e0000c0032004b
:10c18c000e80e80010407800804078000114a10077
:10c19c000e00e800014878000e00e800104078001e
:10c1ac00804078000114a0000e80e800014878005f
:10c1bc0064004700100078001000780064006000f4
:10c1cc000000e0000c0032000e80e8001040780007
:10c1dc00804078000124a1000e00e800014878009e
:10c1ec000e00e80010407800804078000124a00088
:10c1fc000e80e800014878000e80e800e600470059
:10c20c0091017800120020008000780020c5b30056
:10c21c0085e90700004f78001e4078000080fa0086
:10c22c00000006000800fa008e81e8008009780002
:10c23c006400470001087800660047000208780097
:10c24c0066004700900078000e80e800100078002f
:10c25c005af50700004f78001e4078000004e000fb
:10c26c0018003a0066004700900078000e80e80045
:10c27c001000780097fd0700004f78001e407800f2
:10c28c000004e0000f003a006600470090007800c0
:10c29c0064004700100078000d000700004f780084
:10c2ac001e4078000004e00006003a0066004700db
:10c2bc0090007800640047001000780039000700f7
:10c2cc00004f78001e4078000080fa000000060045
:10c2dc000800fa0064014700000978006600470076
:10c2ec00010878008040eb000e80e80001487800df
:10c2fc008040eb000e00e800014878000e80e8005a
:10c30c00e6004700910178001200200080007800c0
:10c31c0090c5b300c2e80700004f78001e407800bb
:10c32c000004e0001c003a000e80e8001040780089
:10c33c00804078000174a1000e00e80001487800ec
:10c34c006400470010007800100078004a00de00fe
:10c35c00614060000080fb004700dd0080407800f9
:10c36c000e00e8001040780000c07000804078009b
:10c37c000e80e800014878000e80e800e6004700d7
:10c38c0091017800120020008000780090c5b30065
:10c39c0025e90700004f78001e4078000080fa0065
:10c3ac00000006000c00fa00680147000009780044
:10c3bc006a004700010878008040eb0064004700e9
:10c3cc00014878008040eb000e00e800014878003e
:10c3dc008040eb000e80e80001487800e500470043
:10c3ec00010009008058eb00f1c5b3006300470061
:10c3fc000148780064004700ea004700910178008a
:10c40c001200200080007800630047001040780084
:10c41c0083e80700004f78001e4078000004e0001d
:10c42c0058003a006400470010407800e340600078
:10c43c000e00e80001487800680047001000780002
:10c44c00100078004300de00f043b2000080fb00d7
:10c45c004200dd00804078000e00e80010407800bb
:10c46c0000c07000804078006400470001487800ec
:10c47c0064004700ea004700910178001200200098
:10c48c00800078006300470010407800e6e8070061
:10c49c00004f78001e4078000004e00039003a009c
:10c4ac0021c6b300630047000148780064004700d0
:10c4bc00ea0047009101780012002000800078000b
:10c4cc00630047001040780055e80700004f7800e3
:10c4dc001e4078000004e0002a003a006400470087
:10c4ec0010407800804078000104a1000e00e800a4
:10c4fc0001487800680047001000780010007800b0
:10c50c004900de00e14060000e80e8000148780040
:10c51c000e00e800904078000e80e8001040780093
:10c52c0080c0700064004700014878006400470038
:10c53c00904078006600470001487800680047008a
:10c54c00100078000080e8009040780065004700fb
:10c55c000148780011c6b300630047000148780019
:10c56c0065004700ea004700910178002200200096
:10c57c00800078006300470010407800aae80700ac
:10c58c00004f78001e4078000080fa000000060082
:10c59c000800fa00640147000009780066004700b3
:10c5ac00010878008040eb000e80e800014878001c
:10c5bc008040eb000e00e800014878000e80e80097
:10c5cc00e6004700910178001200200080007800fe
:10c5dc0000c5b30012e80700004f78001e40780039
:10c5ec000004e0002b003a006400470010007800c3
:10c5fc00104078000042b2000004e000120032004b
:10c60c000e80e8009040780080cfb30080c06000be
:10c61c000e00e800014878000e00e8001040780099
:10c62c00804078007140b3000e80e800014878002b
:10c63c0066004700100078001100200064004000e4
:10c64c00010878000b0037000e80e800904078005d
:10c65c0080cfb30080c060000e80e80001487800f5
:10c66c0066004700100078008080eb0064004000fa
:10c67c00010878000e80e800e60047009101780080
:10c68c00120020008000780000c5b30066e80700a7
:10c69c00004f78001e4078000080fa000000060071
:10c6ac000800fa008e81e8008009780064004700d9
:10c6bc000108780066004700020878006600470011
:10c6cc00900078000e80e800100078003bf4070022
:10c6dc00004f78001e4078000004e00018003a007b
:10c6ec0066004700900078000e80e800100078008b
:10c6fc0078fc0700004f78001e4078000004e00032
:10c70c000f003a0066004700900078006400470074
:10c71c00100078000d000700004f78001e407800d4
:10c72c000004e00006003a00660047009000780024
:10c73c00640047001000780039000700004f7800b3
:10c74c001e4078000080fa00000006000800fa0085
:10c75c006401470000097800660047000108780072
:10c76c008040eb000e80e800014878008040eb0030
:10c77c000e00e800014878000e80e800e600470053
:10c78c0091017800120020008000780090c5b30061
:10c79c00a3e70700004f78001e4078000004e0007b
:10c7ac001c003a000e80e8001040780080407800b1
:10c7bc000174a1000e00e8000148780064004700f5
:10c7cc00100078001080fb004400de006140600027
:10c7dc000080fb004700dd00804078000e00e80080
:10c7ec001040780000c07000804078000e80e80097
:10c7fc00014878000e80e800e600470091017800bf
:10c80c00120020008000780090c5b30006e80700f5
:10c81c00004f78001e4078000080fa0000000600ef
:10c82c000800fa0064014700000978006600470020
:10c83c00010878008040eb000e00e8000148780009
:10c84c0064004700100078000000e8009040780079
:10c85c000e80e800014878000e80e800e6004700f2
:10c86c0091017800120020008000780000c6b3000f
:10c87c00ede70700004f78001e4078000004e00050
:10c88c0052003a000e80e800e60047009101780063
:10c89c00120020008000780020c6b30060e707007b
:10c8ac00004f78001e4078000004e00047003a007a
:10c8bc000e80e8009040780030cfb30080c060005c
:10c8cc000e00e80001487800640047001000780072
:10c8dc009040780063c060000080fb004200dd00e7
:10c8ec0000407800ec4060000e00e800104078003a
:10c8fc0000c07000804078000e80e800014878008d
:10c90c000e80e80090407800f0ccb30080c060004e
:10c91c000e00e80001487800640047001000780021
:10c92c001080fb004200de00634060000080fb00d2
:10c93c004400dd000040780002c3b3008240600078
:10c94c000e00e8001040780000c0700080407800b5
:10c95c000e80e800014878000e80e8001040780056
:10c96c00804078000114a1000e00e8000148780016
:10c97c0064004700100078001080fb004500de00ca
:10c98c00614060000080fb00000040000040780027
:10c99c00e24060000e00e8001040780000c070001b
:10c9ac00804078000e80e800014878000e80e80096
:10c9bc00e60047009101780012002000800078000a
:10c9cc0020c6b30098e70700004f78001e4078009f
:10c9dc000080fa00000006000800fa00640147001d
:10c9ec000009780066004700010878008040eb00e1
:10c9fc000e80e800014878008040eb000e00e80053
:10ca0c00014878000e80e800e600470091017800ac
:10ca1c00120020008000780020c5b30000e707005a
:10ca2c00004f78001e4078000004e0001c003a0023
:10ca3c000e80e80010407800804078000134a1009e
:10ca4c000e00e800014878006400470010007800f0
:10ca5c0010007800614060000080fb004300dd00a6
:10ca6c0000407800e84060000e00e80010407800bc
:10ca7c0000c07000804078000e80e800014878000b
:10ca8c000e80e800e60047009101780012002000bb
:10ca9c008000780020c5b30063e70700004f7800e2
:10caac001e4078000080fa00000006000800fa0022
:10cabc00640147000009780066004700010878000f
:10cacc000040eb00004f78008000eb000e80e80087
:10cadc00010878006400470010007800900078008e
:10caec00000c2000008060000000e00007003a000d
:10cafc0051c1b3000e80e8000148780031c0b3008a
:10cb0c006300470001487800630037006400470069
:10cb1c001000780090007800000c200080806000ed
:10cb2c0000042000808f500007003a00d1c2b300ef
:10cb3c000e80e800014878008040eb00630047005d
:10cb4c00014878005400370064004700100078005a
:10cb5c0090007800000c200080806000000820000d
:10cb6c00808f500007003a00d1c1b3000e80e8005e
:10cb7c000148780071c0b300630047000148780099
:10cb8c0045003700640047001000780090007800e2
:10cb9c00000c200080806000000c2000808f500072
:10cbac003d003a000e80e800e60047009101780055
:10cbbc002200200080007800a0c7b30098e6070090
:10cbcc008e00e800804878000e00e80010407800e5
:10cbdc000004e00030003a000e80e800904078003d
:10cbec0070ceb30000cf60006400470010007800e6
:10cbfc00100078000000d100634060000080fb0052
:10cc0c004300dd0000407800f84060001e407800d2
:10cc1c0000c07000804078000e80e8000148780069
:10cc2c000e80e8009040780080cfb30000cf600009
:10cc3c006400470010007800100078004300de000c
:10cc4c0067406000e74060001e40780000c0700044
:10cc5c00804078000e80e8000148780063004700af
:10cc6c009040780080cfb30000cf60006400470094
:10cc7c0010007800100078004800de00674060006b
:10cc8c00e74060001e40780000c0700080407800d3
:10cc9c0063004700014878000e80e800e60047007a
:10ccac00910178002200200080007800a0c7b3001a
:10ccbc00dde607008e00e800804878000e00e800f2
:10cccc00104078000080fa00000006000a00fa000c
:10ccdc00e4014700800978006600470001087800ed
:10ccec0068004700020878008040eb000e80e800e6
:10ccfc00014878008040eb000e00e8000148780005
:10cd0c000e80e800e8004700910178001200200036
:10cd1c008000780000c5b30041e60700004f7800a2
:10cd2c001e4078000004e0003a003a00640047001e
:10cd3c00100078000080e80010007800e40f50002c
:10cd4c0017003a000e80e800104078008040780010
:10cd5c000154a1000e00e80001487800660047006d
:10cd6c0010007800100078004b00de00614060007d
:10cd7c000080fb004500dd000040780002c2b300db
:10cd8c00824060000e00e8001040780000c0700087
:10cd9c00804078000e80e8000148780015003700cc
:10cdac000e80e80010407800804078000144a1001b
:10cdbc000e00e8000148780066004700100078007b
:10cdcc00100078004b00de00614060000080fb002a
:10cddc004400dd0000407800f04060000e00e800e8
:10cdec001040780000c07000804078000e80e80091
:10cdfc00014878000e80e800e800470091017800b7
:10ce0c00120020008000780000c5b30086e6070001
:10ce1c00004f78001e4078000080fa0000000600e9
:10ce2c000800fa008e81e800800978006400470051
:10ce3c000108780066004700020878006600470089
:10ce4c00900078000e80e800100078005bf207007c
:10ce5c00004f78001e4078000004e0001a003a00f1
:10ce6c0066004700900078000e80e8001000780003
:10ce7c0098fa0700004f78001e4078000004e0008c
:10ce8c0011003a00660047009000780064004700eb
:10ce9c00100078000f000700004f78001e4078004b
:10ceac000004e00008003a0066004700100178001a
:10cebc0064004700900078000e80e80010007800b5
:10cecc003a000700004f78001e4078000080fa00fe
:10cedc00000006000800fa00640147000009780011
:10ceec0066004700010878008040eb000e80e800e7
:10cefc00014878008040eb000e00e8000148780003
:10cf0c000e80e800e6004700910178001200200036
:10cf1c008000780080c5b300c1e50700004f7800a1
:10cf2c001e4078000004e0001d003a000e80e8006e
:10cf3c0010407800804078000134a1000e00e80019
:10cf4c000148780064004700100078001000780059
:10cf5c004a00de00614060000080fb004300dd0001
:10cf6c0000407800e84060000e00e80010407800b7
:10cf7c0000c07000804078000e80e8000148780006
:10cf8c000e80e800e60047009101780012002000b6
:10cf9c008000780080c5b30023e60700004f7800be
:10cfac001e4078000080fa00000006001000fa0015
:10cfbc00ea014700800978006c00470001087800fe
:10cfcc006e004700020878008040eb000e80e800fd
:10cfdc00014878008040eb000e00e8000148780022
:10cfec008000eb0068004700010878008040eb00ef
:10cffc00630047000148780068004700ee004700d6
:10d00c0091017800220020008000780030c6b30027
:10d01c0083e50700004f78001e4078000004e00014
:10d02c0090003a0063004700104078000080fb003d
:10d03c00800047000e00e800e880400011487800ae
:10d04c006a004700100078000080e80010007800ab
:10d05c00e30f500015003a006c00470010007800f8
:10d06c00100078004700de00e740600064004700d5
:10d07c00014878000e00e8009040780080cfb300a3
:10d08c0080c060000e80e800014878006400470012
:10d09c0010407800e74060000e80e80010407800f7
:10d0ac0080c070000e00e800014878006c0047005a
:10d0bc0010007800100078004500de00e1406000b0
:10d0cc0065004700014878000e00e8001040780029
:10d0dc00804078000164a1000e80e80001487800cf
:10d0ec0065004700104078000080fb004600dd0022
:10d0fc000040780002c4b300824060000e80e8005b
:10d10c001040780080c070000e00e80001487800e4
:10d11c006c00470010007800100078004600de001c
:10d12c00e140600066004700014878000e00e8000e
:10d13c0010407800804078000174a1000e80e80057
:10d14c000148780066004700104078000080fb0022
:10d15c004700dd00804078000e80e8001040780029
:10d16c0080c070000e00e8000148780063004700a2
:10d17c00104078000080fb00000047006800400071
:10d18c008e00e800114878006300470010407800da
:10d19c008040e800630047000148780063004700c6
:10d1ac00104078000080fb00800047000e00e80073
:10d1bc00e8804000114878006c00470010007800af
:10d1cc0010007800ff4060006700470001487800bd
:10d1dc000e00e8009040780000ceb30080c06000e4
:10d1ec000e80e80001487800670047001040780086
:10d1fc00ff4060000e80e8001040780080c0700096
:10d20c000e00e800014878006300470010407800e9
:10d21c000080fb0000004700680040008e00e80022
:10d22c001148780063004700104078008040e80007
:10d23c006300470001487800630047001040780005
:10d24c008080fb00680047006e0147009201780067
:10d25c00010178008000780030c6b30072e5070049
:10d26c00004f78001e4078000080fa000000060095
:10d27c000600fa00e4004700800878008040eb00cc
:10d28c000e00e8000148780091c1b3000e80e80060
:10d29c00014878000e80e800e40047009101780016
:10d2ac001200200080007800e0c7b3005ee50700a4
:10d2bc00004f78001e4078000004e00020003a0087
:10d2cc0064004700100078000002b00010017800e4
:10d2dc001000200001002000020001000e00e800f8
:10d2ec00e4004700910178001200200080007800d3
:10d2fc00b0c6b300cae40700004f78000e00e80087
:10d30c0010407800804078000154a0000e00e80026
:10d31c00014878001e4078000004e00008003a0044
:10d32c000e00e800e4004700910178001200200094
:10d33c0080007800b0c6b3003be50700004f7800d2
:10d34c001e4078000080fa00000006000400fa007d
:10d35c008e80e800800878000e00e8008e80e800df
:10d36c0091017800120020008000780040c4b300c6
:10d37c00abe40700004f78001e4078000004e0008a
:10d38c0018003a000e80e80010007800760040008b
:10d39c00100078004400de006f4060008040780090
:10d3ac000e00e800014878000e00e8008e80e800ce
:10d3bc0091017800120020008000780040c4b30076
:10d3cc0019e50700004f78000e80e8001000780087
:10d3dc000002b00010017800a00020000100200025
:10d3ec00020001001e4078000080fa0000000600d8
:10d3fc000600fa000e81e80000097800640047007e
:10d40c00010878000040eb00004f780064004700f2
:10d41c001000780076004000100078004200de001a
:10d42c00634060000080fb00e10f50000f003200f1
:10d43c00e10f500003003c000000e0000600320049
:10d44c0019003700e20f50000d003200e30f5000be
:10d45c0010003200140037000e80e8001000780035
:10d46c001100200001087800120037000e80e8003f
:10d47c001000780021002000010878000d00370012
:10d48c000e80e80010007800610020000108780090
:10d49c00080037000e80e8001000780081002000a2
:10d4ac000108780003003700b0cfb300004f7800bc
:10d4bc00000000001e4078000080fa00000006000a
:10d4cc000400fa008e80e800800878000e80e800e6
:10d4dc001000780066ff0700004f78001e407800af
:10d4ec000004e00004003a000e80e8001000780010
:10d4fc00eae80700004f78001e4078000080fa0030
:10d50c00000006001800fa00ee024700800a7800be
:10d51c00700047000148780072004700020878004c
:10d52c007400470003087800760047000408780070
:10d53c000040eb00004f7800e500470007000900b1
:10d54c008058eb0041c0b3006400470001487800ec
:10d55c008040eb000e00e800014878006e004700a8
:10d56c009000780063004700014878007000370095
:10d57c0070004700f600470091017800120020006f
:10d58c0080007800d0c4b300a7e40700004f7800f7
:10d59c0076004700100078000002b00010017800ff
:10d5ac00a000200001002000020001001e407800b5
:10d5bc000004e0005e003a0065004700f6004700fa
:10d5cc0091017800ee00470011017800800078008e
:10d5dc00640047001040780011e40700004f780009
:10d5ec001e4078000004e0004e003a008040eb0042
:10d5fc000e80e80001487800740047009000780025
:10d60c006e00470010007800808f5000050031003c
:10d61c0074004700900078006300470001487800d0
:10d62c00290037000e00e800104078000080fb0055
:10d63c00f40047009100780000805000ee00470095
:10d64c0091007800810f50001f00310074004700da
:10d65c0010007800804078000e00e8001040780040
:10d66c0080c0500063004700014878001600370066
:10d67c000e00e800104078008080fb000e80e8006f
:10d68c00104078000080fb0000804000f200470052
:10d69c0091007800008040008e80e8009140780076
:10d6ac008180fb0081004700e580400091407800bc
:10d6bc00014878000e80e800104078008040e800b7
:10d6cc000e80e800014878000e80e8009040780059
:10d6dc00630047001040780080cf5000e4ff390011
:10d6ec006e00470010007800804078007000470002
:10d6fc001040780080c0400070004700014878005e
:10d70c006e00470010007800004078008e00e800a2
:10d71c009140780080c040000e00e800014878007d
:10d72c0003003700e0cfb300004f7800070037004c
:10d73c000e00e800104078000080fb00f400470069
:10d74c0091007800810f500089ff39001e4078004d
:10d75c000080fa00000006000800fa00640147008f
:10d76c000009780066004700010878008040eb0053
:10d77c000e80e800014878008040eb000e00e800c5
:10d78c00014878000e80e800e6004700910178001f
:10d79c00120020008000780000c5b300a0e3070051
:10d7ac00004f78001e4078000004e0001e003a0094
:10d7bc000e80e80010407800804078000164a100e1
:10d7cc000e00e80001487800640047001000780063
:10d7dc000080e80010007800614060000080fb00d1
:10d7ec004600dd000040780002c4b30082406000b7
:10d7fc000e00e8001040780000c0700080407800f7
:10d80c000e80e800014878000e80e800e600470032
:10d81c0091017800120020008000780000c5b30050
:10d82c0001e40700004f78001e4078000080fa00e9
:10d83c00000006000a00fa006601470000097800a3
:10d84c0068004700010878008040eb000e00e800fb
:10d85c00014878008040eb000e80e8000148780019
:10d86c008040eb0063004700014878008040eb00eb
:10d87c00640047000148780063004700e800470057
:10d88c0091017800220020008000780050c6b3007f
:10d89c0063e30700004f78001e4078000004e000ae
:10d8ac0084003a000e00e800e300470011487800bd
:10d8bc000e00e80090407800c0cfb30080c060003c
:10d8cc000e80e800014878006600470010007800e0
:10d8dc001000780063406000e34060000e80e800b8
:10d8ec001040780080c070000e00e80001487800fd
:10d8fc000e00e8009040780030cfb30080c060008c
:10d90c000e80e8000148780066004700100078009f
:10d91c00100078004200de00634060000080fb00d5
:10d92c004200dd0000407800ec4060000e80e80012
:10d93c001040780080c070000e00e80001487800ac
:10d94c000e00e80010407800ef4060000e80e80008
:10d95c00014878006600470010007800100078003d
:10d96c004400de006f4060000080fb004400dd00de
:10d97c00804078000e80e8001040780080c0700075
:10d98c000e00e80001487800630047008e00e800b4
:10d99c00114878000e00e800e400470011487800b8
:10d9ac000e00e8009040780000ccb30080c060000e
:10d9bc000e80e800014878006600470010007800ef
:10d9cc00100078004800de00f043b200f2c3b30050
:10d9dc00824060000e80e8001040780080c070002b
:10d9ec000e00e800014878000e00e80010407800b6
:10d9fc00804078000164a1000e80e80001487800a6
:10da0c006600470010007800100078004e00de0021
:10da1c00614060000080fb004600dd0000407800a3
:10da2c0002c4b300824060000e80e8001040780011
:10da3c0080c070000e00e800014878000e00e8007d
:10da4c0010407800804078000174a1000e80e8003e
:10da5c00014878006600470010007800100078003c
:10da6c004f00de00004078000080fb004700dd0026
:10da7c00804078000e80e8001040780080c0700074
:10da8c000e00e80001487800640047008e00e800b2
:10da9c001148780063004700e800470091017800c6
:10daac00220020008000780050c6b3005ee307001f
:10dabc00004f78001e4078000080fa00000006003d
:10dacc000800fa006401470000097800660047006e
:10dadc00010878008040eb000e80e80001487800d7
:10daec008040eb000e00e800014878000e80e80052
:10dafc00e6004700910178001200200080007800b9
:10db0c0000c5b300c6e20700004f78001e40780045
:10db1c000004e0001c003a000e80e8001040780081
:10db2c00804078000174a1000e00e80001487800e4
:10db3c006400470010007800100078004b00de00f5
:10db4c00614060000080fb004700dd0080407800f1
:10db5c000e00e8001040780000c070008040780093
:10db6c000e80e800014878000e80e800e6004700cf
:10db7c0091017800120020008000780000c5b300ed
:10db8c0029e30700004f78001e4078000080fa005f
:10db9c00000006000a00fa00660147000009780040
:10dbac0068004700010878008040eb000e00e80098
:10dbbc00014878008040eb000e80e80001487800b6
:10dbcc008040eb0063004700014878008040eb0088
:10dbdc00640047000148780063004700e8004700f4
:10dbec0091017800220020008000780070c6b300fc
:10dbfc008be20700004f78001e4078000004e00024
:10dc0c004b003a000e00e800e30047001148780092
:10dc1c000e00e8009040780000ccb30080c060009b
:10dc2c000e80e8000148780066004700100078007c
:10dc3c0010007800f043b200f2c3b30082406000e1
:10dc4c000e80e8001040780080c070000e00e800e4
:10dc5c0001487800630047008e00e8001148780006
:10dc6c000e00e800e4004700114878000e00e800c0
:10dc7c0090407800f0ccb30080c060000e80e800cb
:10dc8c00014878006600470010007800100078000a
:10dc9c004900de00634060000080fb004400dd00b2
:10dcac000040780002c3b300824060000e80e800a0
:10dcbc001040780080c070000e00e8000148780029
:10dccc000e00e8009040780080cfb30080c0600068
:10dcdc000e80e800014878006600470010007800cc
:10dcec00100078004600de0067406000e7406000ee
:10dcfc000e80e8001040780080c070000e00e80034
:10dd0c0001487800640047008e00e8001148780054
:10dd1c0063004700e80047009101780022002000d2
:10dd2c008000780070c6b300bfe20700004f780097
:10dd3c001e4078000080fa00000006000800fa007f
:10dd4c00640147000009780066004700010878006c
:10dd5c008040eb000e80e800014878008040eb002a
:10dd6c000e00e800014878000e80e800e60047004d
:10dd7c0091017800120020008000780010c5b300db
:10dd8c0027e20700004f78001e4078000004e000f6
:10dd9c001f003a000e80e8001040780080407800a8
:10ddac000134a1000e00e80001487800640047002f
:10ddbc00100078000080e800104078000080fb0024
:10ddcc004400de00614060000080fb004300dd0089
:10dddc0000407800e84060000e00e8001040780039
:10ddec0000c07000804078000e80e8000148780088
:10ddfc000e80e800e6004700910178001200200038
:10de0c008000780010c5b30087e20700004f78004f
:10de1c001e4078000080fa00000006000800fa009e
:10de2c00640147000009780066004700010878008b
:10de3c008040eb000e80e800014878008040eb0049
:10de4c000e00e800014878000e80e800e60047006c
:10de5c0091017800120020008000780080c5b3008a
:10de6c00efe10700004f78001e4078000004e0004e
:10de7c001e003a000e80e8001040780080407800c8
:10de8c000174a1000e00e80001487800640047000e
:10de9c00100078000080e800104078000080fb0043
:10deac004300de00614060000080fb004700dd00a5
:10debc00804078000e00e8001040780000c0700030
:10decc00804078000e80e800014878000e80e80061
:10dedc00e6004700910178001200200080007800d5
:10deec0080c5b30050e20700004f78001e40780058
:10defc000080fa00000006000a00fa0066014700e4
:10df0c000009780068004700010878008040eb00a9
:10df1c000e00e800014878008040eb000e80e8001d
:10df2c00014878008040eb0063004700014878000e
:10df3c008040eb0064004700014878000e80e80048
:10df4c000080e800e80047009101780012002000f2
:10df5c0080007800c0c5b300b1e10700004f780025
:10df6c001e4078000004e0003c003a0064004700ca
:10df7c0090407800c0cfb30080c060000e00e80075
:10df8c000148780066004700100078000080e80027
:10df9c001040780063406000e34060000e00e80031
:10dfac001040780000c0700080407800640047008a
:10dfbc0001487800640047001040780080407800e9
:10dfcc000124a1000e00e80001487800660047001b
:10dfdc00100078000080e800104078000080fb0002
:10dfec004200de00614060000080fb004200dd006a
:10dffc0000407800e44060000e00e800104078001b
:10e00c0000c0700080407800640047000148780030
:10e01c0066004700100078000000e800904078008f
:10e02c006300470001487800660047001000780044
:10e03c00904078000e80e800014878000e80e800df
:10e04c00e800470091017800320020008000780041
:10e05c00a0c5b300f4e10700004f78001e40780023
:10e06c000080fa00000006000800fa006401470076
:10e07c000009780066004700010878008040eb003a
:10e08c000e80e800014878008040eb000e00e800ac
:10e09c00014878000e80e800e60047009101780006
:10e0ac00120020008000780010c5b3005ce107006e
:10e0bc00004f78001e4078000004e00043003a0056
:10e0cc000e80e80010407800804078000104a10028
:10e0dc000e00e8000148780064004700100078004a
:10e0ec009040780061c06000e14060000e00e800e4
:10e0fc001040780000c07000804078000e80e8006e
:10e10c00014878000e80e8001040780080407800cc
:10e11c000114a1000e00e8000148780064004700db
:10e12c00100078001080fb000000d10061406000fe
:10e13c000080fb000000400000407800e2406000de
:10e14c000e00e8001040780000c07000804078009d
:10e15c000e80e800014878000e80e800104078003e
:10e16c00804078000124a1000e00e80001487800ee
:10e17c0064004700100078001080fb004200de00b5
:10e18c00614060000080fb004200dd000040780030
:10e19c00e44060000e00e8001040780000c0700001
:10e1ac00804078000e80e800014878000e80e8007e
:10e1bc00e6004700910178001200200080007800f2
:10e1cc0010c5b30098e10700004f78001e4078009e
:10e1dc000080fa00000006000800fa006401470005
:10e1ec000009780066004700010878008040eb00c9
:10e1fc000e80e800014878008040eb000e00e8003b
:10e20c00014878000e80e800e60047009101780094
:10e21c00120020008000780080c5b30000e10700e8
:10e22c00004f78001e4078000004e0001c003a000b
:10e23c000e80e80010407800804078000174a10046
:10e24c000e00e800014878006400470010007800d8
:10e25c001080fb004500de00614060000080fb0088
:10e26c004700dd00804078000e00e8001040780088
:10e27c0000c07000804078000e80e80001487800f3
:10e28c000e80e800e60047009101780012002000a3
:10e29c008000780080c5b30063e10700004f780070
:10e2ac001e4078000080fa00000006000a00fa0008
:10e2bc0066014700000978006800470001087800f3
:10e2cc008040eb000e00e800014878008040eb0035
:10e2dc000e80e800014878008040eb0063004700a6
:10e2ec00014878008040eb0064004700014878004a
:10e2fc000e80e800e8004700910178001200200031
:10e30c0080007800c0c5b300c5e00700004f78005e
:10e31c001e4078000004e00028003a000e80e8005f
:10e32c0010407800f2c3b300824060000e00e80099
:10e33c000148780066004700100078001080fb0050
:10e34c004300de00634060000080fb004600dd00ff
:10e35c00804078000e00e8001040780000c070008b
:10e36c00804078000e80e800014878006600470085
:10e37c00100078000080e8009040780063004700af
:10e38c000148780066004700100078000000e800a3
:10e39c009040780064004700014878000e80e80047
:10e3ac00e8004700910178003200200080007800de
:10e3bc00c0c5b3001ce10700004f78001e40780078
:10e3cc000080fa00000006000a00fa00660147000f
:10e3dc000009780068004700010878008040eb00d5
:10e3ec000e00e800014878008040eb006400470014
:10e3fc000148780064004700e8004700910178006c
:10e40c00120020008000780030c5b30084e00700c3
:10e41c00004f78001e4078000004e000b7003a007e
:10e42c006600470010007800e40040000e80e80011
:10e43c000108780066004700100078001000780092
:10e44c00e10f500051003a00640047001040780082
:10e45c00804078000134a1000e00e80001487800eb
:10e46c000e80e80010007800100078006140600019
:10e47c000080fb004300dd0000407800e8406000b5
:10e48c000e00e8001040780000c07000804078005a
:10e49c006400470001487800640047001040780091
:10e4ac00804078000124a1000e00e80001487800ab
:10e4bc000e80e80010007800100078000000d100f9
:10e4cc00614060000080fb004200dd0000407800ed
:10e4dc00e44060000e00e8001040780000c07000be
:10e4ec0080407800640047000148780064004700d1
:10e4fc0010407800804078000114a1000e00e80064
:10e50c00014878000e80e8001000780010007800b8
:10e51c004200de00614060000080fb000000400013
:10e52c0000407800e24060000e00e80010407800e7
:10e53c0000c07000804078006400470001487800fb
:10e54c006400470010407800804078000104a1006e
:10e55c000e00e800014878000e80e80010007800fa
:10e56c00100078004300de0061406000e140600074
:10e57c000e00e8001040780000c070008040780069
:10e58c0064004700014878005400370064004700dd
:10e59c0010407800804078000174a1000e00e80063
:10e5ac00014878000e80e800100078001000780018
:10e5bc00614060000080fb004700dd008040780077
:10e5cc000e00e8001040780000c070008040780019
:10e5dc006400470001487800640047001040780050
:10e5ec00804078000164a1000e00e800014878002a
:10e5fc000e80e80010007800100078000000d100b8
:10e60c00614060000080fb004600dd0000407800a7
:10e61c0002c4b300824060000e00e8001040780095
:10e62c0000c070008040780064004700014878000a
:10e63c006400470010407800804078000154a1002d
:10e64c000e00e800014878000e80e8001000780009
:10e65c00100078004200de00614060000080fb008a
:10e66c004500dd000040780002c2b300824060002b
:10e67c000e00e8001040780000c070008040780068
:10e68c00640047000148780064004700104078009f
:10e69c00804078000144a1000e00e8000148780099
:10e6ac000e80e80010007800100078004300de00b7
:10e6bc00614060000080fb004400dd0000407800f9
:10e6cc00f04060000e00e8001040780000c07000c0
:10e6dc0080407800640047000148780064004700df
:10e6ec00e8004700910178001200200080007800bb
:10e6fc0030c5b3004ce00700004f78001e40780096
:10e70c000080fa00000006000a00fa0066014700cb
:10e71c000009780068004700010878008040eb0091
:10e72c000e00e800014878008040eb0064004700d0
:10e73c000148780064004700e80047009101780028
:10e74c00120020008000780040c5b300b4df070041
:10e75c00004f78001e4078000004e00050003a00a2
:10e76c006600470010007800e40040000e80e800ce
:10e77c00010878006600470010007800100078004f
:10e78c00e10f500016003a0064004700104078007a
:10e79c00804078000144a1000e00e8000148780098
:10e7ac000e80e80010007800100078004400de00b5
:10e7bc00614060000080fb004400dd0000407800f8
:10e7cc00f04060000e00e8001040780000c07000bf
:10e7dc00804078006400470001487800160037003c
:10e7ec006400470010407800804078000154a1007c
:10e7fc000e00e800014878000e80e8001000780058
:10e80c00100078004400de00614060000080fb00d6
:10e81c004500dd000040780002c2b3008240600079
:10e82c000e00e8001040780000c0700080407800b6
:10e83c00640047000148780064004700904078006d
:10e84c0000cfb30080c060000e00e80001487800e3
:10e85c000e80e80010007800100078004500de0003
:10e86c006f406000ef4060000e00e8001040780040
:10e87c0000c07000804078006400470001487800b8
:10e88c0064004700e8004700910178001200200066
:10e89c008000780040c5b300e3df0700004f78002c
:10e8ac001e4078000080fa00000006001800fa00f4
:10e8bc00f6004700800878007600470010007800ca
:10e8cc001b000700004f78001e4078000004e00099
:10e8dc0014003a000e80e800f60047009100780022
:10e8ec0035000700004f78001e4078000004e0005f
:10e8fc000c003a006c004700f600470091007800cd
:10e90c0052000700004f78001e4078000004e00021
:10e91c0004003a00ec0047000e80e800700007008d
:10e92c00004f78001e4078000080fa0000000600be
:10e93c000400fa008e80e800800878000e80e80061
:10e94c001000780011c1b300660040000148780047
:10e95c000e80e8001000780081c0b3006800400011
:10e96c00014878000e80e80010007800dae007001b
:10e97c00004f78001e4078000004e0000b003a00c5
:10e98c00c1c2b3000e00e800014878000e00e80098
:10e99c008e80e80091017800120020008000780041
:10e9ac0000c4b300a0df0700004f78001e407800c1
:10e9bc000080fa00000006000600fa000e81e80054
:10e9cc00000978006400470001087800d1c0b3004a
:10e9dc000e00e800014878000e00e800e400470053
:10e9ec00910178001200200080007800d0c6b3009e
:10e9fc008ddf0700004f78001e4078000004e00017
:10ea0c000f003a0064004700100078000002b000cc
:10ea1c0010017800200320000100200002000100fa
:10ea2c0064004700900178000001eb000e80e800c4
:10ea3c009000780010c0b30035e10700004f78005b
:10ea4c001e4078000080fa00000006000600fa0064
:10ea5c000e81e80000097800640047000108780086
:10ea6c0091c0b3000e00e800014878000e00e800e9
:10ea7c00e40047009101780012002000800078002b
:10ea8c00d0c6b30068df0700004f78001e40780046
:10ea9c000004e0000f003a0064004700100078000a
:10eaac000002b000100178002003200001002000bb
:10eabc000200010064004700900178000001eb00a7
:10eacc000e80e8009000780010c0b30010e1070041
:10eadc00004f78001e4078000080fa00000006000d
:10eaec000600fa000e81e800000978006400470077
:10eafc00010878006400470010007800900078004e
:10eb0c000e80e80010007800100078008080500023
:10eb1c0000002200808f50001b003400640047006e
:10eb2c00100078000080e800900078000e80e8006b
:10eb3c00100078000080e800100078008080500001
:10eb4c0000002200808f50000f003400640047004a
:10eb5c001000780064004000900078000e80e800ff
:10eb6c001000780064004000100078008080500095
:10eb7c0000002200808f5000030034000040eb00a6
:10eb8c00004f78000200370020c0b300004f78001f
:10eb9c001e4078000080fa00000006000400fa0015
:10ebac008e80e800800878000e80e8001000780065
:10ebbc0012000700004f78001e4078000004e000af
:10ebcc000b003a000e80e800100078000002b00044
:10ebdc001001780020032000010020000200010039
:10ebec000e80e800100078002d000700004f780020
:10ebfc001e4078000080fa00000006000400fa00b5
:10ec0c008e80e800800878000e00e8008e80e80016
:10ec1c00910178001200200080007800d0c6b3006b
:10ec2c007fde0700004f78001e4078000004e000f3
:10ec3c0018003a000e00e800104078008040780080
:10ec4c000144a0000e00e800014878000e00e80026
:10ec5c008e80e8009101780012002000800078007e
:10ec6c00d0c6b300f0de0700004f78001e407800dd
:10ec7c000004e00007003a000e80e8001000780065
:10ec8c000002b00010017800f0002000010020000c
:10ec9c00020001001e4078000080fa00000006000f
:10ecac000400fa008e80e800800878000e00e8006e
:10ecbc008e80e8009101780012002000800078001e
:10eccc00b0c1b30056de0700004f78001e4078003c
:10ecdc000004e00011003a000e00e800104078003b
:10ecec000080fb00620060000080d1008040780052
:10ecfc000e00e800014878000e00e8001040780093
:10ed0c00e14f500003003a000040eb00004f780048
:10ed1c000200370010c0b300004f78001e4078008e
:10ed2c000080fa00000006000600fa000e81e800e0
:10ed3c000009780064004700010878000040eb00ef
:10ed4c00004f780064004700100078000000e000dd
:10ed5c000600320064004700100078000002b0008a
:10ed6c00100078000000e00003003a0000c0eb0047
:10ed7c00004f7800180037006400470090007800be
:10ed8c000e80e8001000780016000700004f780095
:10ed9c001e4078000004e0000f003a0064004700b9
:10edac00900078000e80e8001000780083ea0700dd
:10edbc00004f78001e4078000004e00006003a0086
:10edcc0064004700900078000e80e8001000780086
:10eddc0060f30700004f78001e4078000080fa00b6
:10edec00000006000600fa000e81e8000009780019
:10edfc0064004700010878008040eb000e00e8003a
:10ee0c00014878000e00e800e4004700910178000a
:10ee1c00120020008000780010c5b30000de07004f
:10ee2c00004f78001e4078000004e00019003a0002
:10ee3c000e00e80010407800804078000154a100da
:10ee4c000e80e800100078006a0040001000780086
:10ee5c00614060000080fb004500dd000040780050
:10ee6c000042b20000c07000804078000e00e80044
:10ee7c00014878000e00e800e4004700910178009a
:10ee8c00120020008000780010c5b30066de070079
:10ee9c00004f78001e4078000080fa000000060049
:10eeac000600fa000e81e8000009780064004700b3
:10eebc00010878000040eb00004f78006400470028
:10eecc00100078000000e0000600320064004700eb
:10eedc00100078000002b000100078000000e00084
:10eeec0003003a0000c0eb00004f78001800370018
:10eefc0064004700900078000e80e8001000780055
:10ef0c0016000700004f78001e4078000004e00057
:10ef1c000f003a0064004700900078000e80e80073
:10ef2c001000780025ea0700004f78001e4078009a
:10ef3c000004e00006003a006400470090007800ee
:10ef4c000e80e8001000780002f30700004f7800f4
:10ef5c001e4078000080fa00000006000600fa004f
:10ef6c000e81e80000097800640047000108780071
:10ef7c008040eb000e00e800014878000e00e8002d
:10ef8c00e400470091017800120020008000780016
:10ef9c0010c5b300a2dd0700004f78001e407800ba
:10efac000004e0001a003a000e00e800104078005f
:10efbc00804078000164a1000e80e8001000780009
:10efcc006a004000100078000000d1006140600031
:10efdc000080fb004600dd00004078000044b200d9
:10efec0000c07000804078000e00e80001487800f6
:10effc000e00e800e40047009101780012002000a8
:10f00c008000780010c5b30007de0700004f7800c1
:10f01c001e4078000080fa00000006000200fa0092
:10f02c00000f78001e0078007a0040001000780075
:10f03c008000eb0068004000010878001e0078009a
:10f04c007a004000100078008000eb006a0040005d
:10f05c00010878001e0078007a004000100078004b
:10f06c008000eb006c004000010878001e00780066
:10f07c007a004000100178006000b8006e01410079
:10f08c000089be001e0078007a0040001000780055
:10f09c008040eb0072004000014878000080fa00cc
:10f0ac00000006000800fa0064014700000978001f
:10f0bc0066004700010878000040eb00004f780024
:10f0cc0021c2b3000e00e800014878000e80e80071
:10f0dc00e6004700910178002200200080007800b3
:10f0ec000e00e800104078004ddd07001e4f700048
:10f0fc006300470010407800e74060006300470061
:10f10c000148780063004700104078000080fb0045
:10f11c00c800dd000e80e800104078000080fb0085
:10f12c00810070006400470010007800010878002e
:10f13c001e4078000080fa00000006000800fa006b
:10f14c00000f78000e80e80001087800640047008a
:10f15c000208780066004700030878006600470044
:10f16c00100078007a004000100078006800400021
:10f17c00900078001e0078000108780066004700b7
:10f18c00100078007a004000100078006600400003
:10f19c009040780000c4b30080cf50000b003a00c0
:10f1ac006400470010007800104078000080fb00dd
:10f1bc006600b90000007800800078000e80e8003e
:10f1cc001000780001087800440037006600470002
:10f1dc00100078007a0040001000780066004000b3
:10f1ec009040780000ccb30080cf50000b003a0068
:10f1fc006400470010007800104078000080fb008d
:10f20c006c00b90000007800800078000e80e800e7
:10f21c0010007800010878003000370066004700c5
:10f22c00100078007a004000100078006600400062
:10f23c009040780000c6b30080cf50000b003a001d
:10f24c006400470010007800104078000080fb003c
:10f25c006e00b90000007800800078000e80e80095
:10f26c0010007800010878001c0037006600470089
:10f27c00100078007a004000100078006600400012
:10f28c009040780000ceb30080cf50000b003a00c5
:10f29c006400470010007800104078000080fb00ec
:10f2ac007400b90000007800800078000e80e8003f
:10f2bc00100078000108780008003700660047004d
:10f2cc00100078007a004000100078000080e80000
:10f2dc00900078001e007800010878000e80e8008d
:10f2ec00100078009000780066004700100078004d
:10f2fc007a004000100078000080e80010007800d0
:10f30c00808f50000900360066004700100078001e
:10f31c007a004000100078000080e800900078002f
:10f32c000e80e80010007800010878000080fa00d8
:10f33c00000006000a00fa00000f78000e80e800ba
:10f34c000108780064004700020878006600470056
:10f35c0003487800680047000408780066004700fe
:10f36c00104078000080fb00c1082000810f500085
:10f37c0067003200c1082000810f500017003c00cc
:10f38c0001062000810f500095003200010620007c
:10f39c00810f500007003c0001022000810f50003b
:10f3ac00f700320001042000810f500025003200cc
:10f3bc000b01370041082000810f50002100320062
:10f3cc0081082000810f5000f50032000108200058
:10f3dc00810f5000f200320001013700c1092000fa
:10f3ec00810f5000b2003200c1092000810f500083
:10f3fc000a003c0041092000810f500078003200c7
:10f40c0081092000810f5000ed003200010920001d
:10f41c00810f5000da003200f1003700010c20009f
:10f42c00810f50003a003200010e2000810f500075
:10f43c009f003200010a2000810f5000e0003200d2
:10f44c00e70037000e80e80010007800100078000c
:10f45c0066004000e800470091007800fa80400008
:10f46c00910078008180e80091007800810f5000b5
:10f47c000a00360068004700100078007a0040004f
:10f48c00100078000080e800900078000e80e80002
:10f49c001000780001087800d10037000e80e800d9
:10f4ac00100078009001780064004700100078008c
:10f4bc00104078000080fb006a00b9000000780062
:10f4cc001e004000e800470011017800830078001e
:10f4dc00c50007000e80e8001000780010007800ce
:10f4ec00e60040000e80e80010007800010878006b
:10f4fc006400470010007800104078000040e800dd
:10f50c00e40047009100780080487800b400370090
:10f51c000e80e80010007800100078006c004000ad
:10f52c00e800470091007800fa80400091007800d4
:10f53c008180e80091007800810f50000a003600ad
:10f54c0068004700100078007a0040001000780036
:10f55c000080e800900078000e80e8001000780031
:10f56c00010878009e0037000e80e800100078003b
:10f57c0010007800e601400064004700100078009d
:10f58c00104078000080fb006a00b9000000780091
:10f59c001e004000e800470011017800830078004d
:10f5ac00910007000e80e800100078001000780031
:10f5bc00ec0040000e80e800100078000108780094
:10f5cc006400470010007800104078000040e8000c
:10f5dc00e4004700910078008048780080003700f4
:10f5ec000e80e80010007800100078006e004000db
:10f5fc00e800470091007800fa8040009100780004
:10f60c008180e80091007800810f50000a003600dc
:10f61c0068004700100078007a0040001000780065
:10f62c000080e800900078000e80e8001000780060
:10f63c00010878006a0037000e80e800100078009e
:10f64c0010007800e80140006400470010007800ca
:10f65c00104078000080fb006a00b90000007800c0
:10f66c001e004000e800470011017800830078007c
:10f67c005d0007000e80e800100078001000780094
:10f68c00ee0040000e80e8001000780001087800c1
:10f69c006400470010007800104078000040e8003b
:10f6ac00e400470091007800804878004c00370057
:10f6bc000e80e80010007800100078007400400004
:10f6cc00e800470091007800fa8040009100780033
:10f6dc008180e80091007800810f50000a0036000c
:10f6ec0068004700100078007a0040001000780095
:10f6fc000080e800900078000e80e8001000780090
:10f70c0001087800360037000e80e8001000780001
:10f71c0010007800ee0140006400470010007800f3
:10f72c00104078000080fb006a00b90000007800ef
:10f73c001e004000e80047001101780083007800ab
:10f74c00290007000e80e8001000780010007800f7
:10f75c00f40040000e80e8001000780001087800ea
:10f76c006400470010007800104078000040e8006a
:10f77c00e4004700910078008048780018003700ba
:10f78c000e80e8001000780010007800e8004000bf
:10f79c000e80e80010007800010878001000370097
:10f7ac000e80e8001000780010007800e6004000a1
:10f7bc000e80e8001000780001087800080037007f
:10f7cc000e80e8001000780010007800ee00400079
:10f7dc000e80e8001000780001087800000000009e
:10f7ec000080fa00000006000a00fa00e40147005d
:10f7fc00800978006600470001087800680047001f
:10f80c000208780068004700100078007a00400079
:10f81c001000780090007800660047001000780017
:10f82c0000804000104078000080fb00000f780042
:10f83c0066004700100078008000e8006600470072
:10f84c000108780068004700100078007a0040003a
:10f85c0010007800900078006600470010007800d7
:10f86c0000804000104078008080fb000e80e80093
:10f87c000108780066004700100078008000e8005e
:10f88c0066004700010878000e80e8001000780040
:10f89c004800dd001e007000800078006400470006
:10f8ac00100078000108780068004700100078000c
:10f8bc007a00400010007800900078006600470045
:10f8cc001000780000804000104078000080fb00a1
:10f8dc00000f780066004700100078008000e800f8
:10f8ec0066004700010878006800470010007800a7
:10f8fc007a00400010007800900078006600470005
:10f90c001000780000804000104078008080fb00e0
:10f91c000e80e800010878006600470010007800af
:10f92c008000e80066004700010878000e80e800bf
:10f93c00100078004800dd001e0070008000780088
:10f94c0064004700100078000080e800010878008f
:10f95c0068004700100078007a0040001000780022
:10f96c00900078006600470010007800008040008e
:10f97c00104078000080fb00000f78006600470004
:10f98c00100078008000e80066004700010878004d
:10f99c0068004700100078007a00400010007800e2
:10f9ac00900078006600470010007800008040004e
:10f9bc00104078008080fb000e80e8000108780081
:10f9cc0066004700100078008000e80066004700e1
:10f9dc00010878000e80e800100078004800dd0077
:10f9ec001e00700080007800640047001000780052
:10f9fc0064004000010878000080fa000000060056
:10fa0c000c00fa00e6014700800978006800470006
:10fa1c00010878006a004700020878000040eb00fb
:10fa2c00004f78008040eb006400470001487800ec
:10fa3c006a004700100078007a004000100078003f
:10fa4c0068004000900078000e80e8000108780003
:10fa5c00b90037006a004700100078007a004000b7
:10fa6c0010007800900078000e80e80010007800fc
:10fa7c000080400090407800c0cfb30000cf600001
:10fa8c000e80e800100078008000e8000e80e8008e
:10fa9c00010878001e80fb006101b90000fc2f00fa
:10faac00f1ff2f000200400083804800c2052000b7
:10fabc0003002000820f5000838f580094003e00fa
:10facc00006001007e003700930037009200370081
:10fadc0091003700750037008f0037008e0037001b
:10faec008d0037007b0037008b0037008a00370011
:10fafc008900370088003700870037008600370000
:10fb0c0085003700840037008300370082003700ff
:10fb1c0081003700800037007f0037007e003700ff
:10fb2c007d0037007c0037007b0037007a003700ff
:10fb3c0079003700780037007700370076003700ff
:10fb4c0075003700740037007300370072003700ff
:10fb5c0071003700700037006f0037006e003700ff
:10fb6c006d0037006c0037006b0037006a003700ff
:10fb7c0069003700680037006700370066003700ff
:10fb8c0065003700640037006300370062003700ff
:10fb9c0061003700600037005f0037005e003700ff
:10fbac005d0037005c0037005b0037005a003700ff
:10fbbc0059003700580037005700370056003700ff
:10fbcc00550037004900370053003700520037000a
:10fbdc0051003700180037004f0037004e00370037
:10fbec004d003700250037004b0037004a00370026
:10fbfc004900370010003700470037004600370037
:10fc0c00450037001700370043003700420037002b
:10fc1c0041003700080037003f0037003e00370036
:10fc2c003d0037001b0037003b0037003a0037001f
:10fc3c003900370000003700e40047000e80e80070
:10fc4c006a014700120278009e4178000101780099
:10fc5c00800078006600470010007800b5fd0700b2
:10fc6c002e0037000e80e800ea00470011017800f2
:10fc7c0081c0b300b2060700280037000e80e800f0
:10fc8c00ea0047001101780061c0b300ac06070020
:10fc9c00220037000e80e800ea00470011017800ce
:10fcac00e1c0b300a60607001c0037000e80e80078
:10fcbc00ea00470091007800c806070017003700db
:10fccc000e80e800ea004700910078002a07070040
:10fcdc00120037000e80e800ea004700110178009e
:10fcec0011c0b300960607000c0037006a004700ed
:10fcfc00100078007a004000100078000080e800c6
:10fd0c00900078000e80e8000108780003003700ae
:10fd1c0000000000010037000000000068004700f0
:10fd2c001000780090407800640047001040780084
:10fd3c0080cf50000b0032006a00470010007800a2
:10fd4c007a004000100078000080e80090007800f5
:10fd5c000e80e80010007800808f50003dff3e00c0
:10fd6c0001003700000000006400470010407800dc
:10fd7c00e800470091007800804878006a0047004e
:10fd8c00100078007a004000900078000e80e800a7
:10fd9c001001780068804000020878000080fa00aa
:10fdac00000006000800fa00000f78000e80e80042
:10fdbc0001087800640047000208780066004700dc
:10fdcc000308780066004700100078007a004000b5
:10fddc00100078006a004000900078001e00780047
:10fdec000108780066004700100078007a00400097
:10fdfc0010007800660040009040780000c8b30006
:10fe0c0080cf50000b003a006400470010007800cf
:10fe1c00104078000080fb006600b90000007800fc
:10fe2c00800078000e80e80010007800010878004f
:10fe3c004400370066004700100078007a0040004c
:10fe4c0010007800660040009040780000ccb300b1
:10fe5c0080cf50000b003a0064004700100078007f
:10fe6c00104078000080fb006c00b90000007800a6
:10fe7c00800078000e80e8001000780001087800ff
:10fe8c003000370066004700100078007a00400010
:10fe9c0010007800660040009040780000cab30063
:10feac0080cf50000b003a0064004700100078002f
:10febc00104078000080fb006e00b9000000780054
:10fecc00800078000e80e8001000780001087800af
:10fedc001c00370066004700100078007a004000d4
:10feec0010007800660040009040780000ceb3000f
:10fefc0080cf50000b003a006400470010007800df
:10ff0c00104078000080fb007400b90000007800fd
:10ff1c00800078000e80e80010007800010878005e
:10ff2c000800370066004700100078007a00400097
:10ff3c00100078000080e800900078001e00780027
:10ff4c00010878000e80e80010007800900078001e
:10ff5c0066004700100078007a004000100078001e
:10ff6c000080e80010007800808f500009003600f7
:10ff7c0066004700100078007a00400010007800fe
:10ff8c000080e800900078000e80e80010007800f7
:10ff9c00010878000080fa00000006000a00fa0050
:10ffac00000f78000e80e80001087800640047001c
:10ffbc000208780066004700034878006800470094
:10ffcc000408780066004700104078000080fb00b1
:10ffdc00c1082000810f500067003200c1082000ca
:10ffec00810f500017003c0001062000810f5000cb
:10fffc00c800320001062000810f500007003c00b1
:020000040001f9
:10000c0001022000810f5000ca00320001042000c0
:10001c00810f5000030132000a0137004108200013
:10002c00810f5000ff00320081082000810f50002a
:10003c001e00320001082000810f50001b0032000e
:10004c0000013700c1092000810f50007d003200f3
:10005c00c1092000810f50000a003c00410920001a
:10006c00810f5000ab00320081092000810f50003d
:10007c00b800320001092000810f5000ad003200a1
:10008c00f0003700010c2000810f50003a003200c4
:10009c00010e2000810f50006a003200010a20007e
:1000ac00810f5000ab003200e60037000e80e800f4
:1000bc00100078001000780066004000e80047004f
:1000cc0091007800fa804000910078008180e8006f
:1000dc0091007800810f50000a003600680047003c
:1000ec00100078007a004000100078000080e800d2
:1000fc00900078000e80e80010007800010878006d
:10010c00d00037000e80e8001000780090017800d5
:10011c006400470010007800104078000080fb005d
:10012c006a00b900000078001e004000e80047009b
:10013c001101780083007800c40007000e80e800ed
:10014c001000780010007800e60040000e80e800f7
:10015c001000780001087800640047001000780057
:10016c00104078000040e800e4004700910078005f
:10017c0080487800b30037000e80e800100078004b
:10018c00100078006c004000e800470091007800f7
:10019c00fa804000910078008180e800910078009e
:1001ac00810f50000a0036006800470010007800ec
:1001bc007a004000100078000080e8009000780081
:1001cc000e80e80010007800010878009d003700d0
:1001dc000e80e80010007800900178006400470061
:1001ec0010007800104078000080fb006a00b90015
:1001fc00000078001e004000e80047001101780064
:10020c0083007800910007000e80e8001000780051
:10021c0010007800ec0040000e80e8001000780020
:10022c000108780064004700100078001040780046
:10023c000040e800e4004700910078008048780016
:10024c00800037000e80e800100078001000780065
:10025c0074004000e800470091007800fa804000ec
:10026c00910078008180e80091007800810f5000a7
:10027c000a00360068004700100078007a00400041
:10028c00100078000080e800900078000e80e800f4
:10029c0010007800010878006a0037000e80e80032
:1002ac001000780010007800e8014000640047005e
:1002bc0010007800104078000080fb006a00b90044
:1002cc00000078001e004000e80047001101780093
:1002dc00830078005d0007000e80e80010007800b5
:1002ec0010007800f40040000e80e8001000780048
:1002fc000108780064004700100078001040780076
:10030c000040e800e4004700910078008048780045
:10031c004c0037000e80e8001000780010007800c8
:10032c00ee0040000e80e800100078000108780014
:10033c00440037000e80e8001000780010007800b0
:10034c00e80040000e80e8001000780001087800fa
:10035c003c0037000e80e800100078001000780098
:10036c006e004000e800470091007800fa804000e1
:10037c00910078008180e80091007800810f500096
:10038c000a00360068004700100078007a00400030
:10039c00100078000080e800900078000e80e800e3
:1003ac001000780001087800260037000e80e80065
:1003bc001000780010007800e8014000640047004d
:1003cc0010007800104078000080fb006a00b90033
:1003dc00000078001e004000e80047001101780082
:1003ec0083007800190007000e80e80010007800e8
:1003fc0010007800ee0040000e80e800100078003d
:10040c000108780064004700100078001040780064
:10041c000040e800e4004700910078008048780034
:10042c00080037000e80e8001000780010007800fb
:10043c00e60040000e80e80010007800010878000b
:10044c00000000000080fa00000006000a00fa001c
:10045c00e401470080097800660047000108780035
:10046c006800470002087800680047001000780018
:10047c007a00400010007800900078006600470079
:10048c001000780000804000104078000080fb00d5
:10049c00000f780066004700100078008000e8002c
:1004ac0066004700010878006800470010007800db
:1004bc007a00400010007800900078006600470039
:1004cc001000780000804000104078008080fb0015
:1004dc000e80e800010878006600470010007800e4
:1004ec008000e80066004700010878000e80e800f4
:1004fc00100078004800dd001e00700080007800bd
:10050c00640047001000780001087800680047007c
:10051c00100078007a0040001000780090007800fd
:10052c006600470010007800008040001040780002
:10053c000080fb00000f7800660047001000780078
:10054c008000e8006600470001087800680047005a
:10055c00100078007a0040001000780090007800bd
:10056c0066004700100078000080400010407800c2
:10057c008080fb000e80e8000108780066004700d0
:10058c00100078008000e800660047000108780041
:10059c000e80e800100078004800dd001e0070009e
:1005ac008000780064004700100078000080e800ac
:1005bc000108780068004700100078007a004000bd
:1005cc00100078009000780066004700100078005a
:1005dc0000804000104078000080fb00000f780085
:1005ec0066004700100078008000e80066004700b5
:1005fc000108780068004700100078007a0040007d
:10060c001000780090007800660047001000780019
:10061c0000804000104078008080fb000e80e800d5
:10062c000108780066004700100078008000e800a0
:10063c0066004700010878000e80e8001000780082
:10064c004800dd001e007000800078006400470048
:10065c001000780064004000010878000080fa0067
:10066c00000006000c00fa00e60147008009780043
:10067c0068004700010878006a004700020878000b
:10068c000040eb00004f78008040eb006400470016
:10069c00014878006a004700100078007a0040009a
:1006ac00100078006a004000900078000e80e8008e
:1006bc0001087800b90037006a0047001000780084
:1006cc007a00400010007800900078000e80e8005e
:1006dc00100078000080400090407800c0cfb3003c
:1006ec0000cf60000e80e800100078008000e80069
:1006fc000e80e800010878001e80fb006101b90043
:10070c0000fc2f00f1ff2f00020040008380480006
:10071c00c205200003002000820f5000838f580078
:10072c0094003e00006001007e003700930037000b
:10073c009200370091003700750037008f003700aa
:10074c008e0037008d0037007b0037008b003700a0
:10075c008a0037008900370088003700870037008f
:10076c00860037008500370084003700830037008f
:10077c008200370081003700800037007f0037008f
:10078c007e0037007d0037007c0037007b0037008f
:10079c007a0037007900370078003700770037008f
:1007ac00760037007500370074003700730037008f
:1007bc007200370071003700700037006f0037008f
:1007cc006e0037006d0037006c0037006b0037008f
:1007dc006a0037006900370068003700670037008f
:1007ec00660037006500370064003700630037008f
:1007fc006200370061003700600037005f0037008f
:10080c005e0037005d0037005c0037005b0037008e
:10081c005a0037005900370058003700570037008e
:10082c005600370055003700490037005300370099
:10083c005200370051003700230037004f003700bb
:10084c004e0037004d003700140037004b003700c6
:10085c004a003700490037001000370047003700c6
:10086c0046003700450037001d00370043003700b5
:10087c0042003700410037001f0037003f003700af
:10088c003e0037003d003700040037003b003700c6
:10089c003a0037003900370000003700e400470009
:1008ac000e80e8006a014700120278009e41780031
:1008bc000101780080007800660047001000780085
:1008cc00b6fd07002e0037000e80e800ea00470056
:1008dc001101780061c0b3009903070028003700ac
:1008ec000e80e800ea0047001101780081c0b300d7
:1008fc0093030700220037000e80e800ea0047004f
:10090c001101780081c0b3008d0307001c00370073
:10091c000e80e800ea00470091007800af03070062
:10092c00170037000e80e800ea00470091007800bd
:10093c0011040700120037000e80e800ea0047009f
:10094c001101780011c0b3007d0307000c003700c3
:10095c006a004700100078007a0040001000780010
:10096c000080e800900078000e80e8000108780014
:10097c0003003700000000000100370000000000f9
:10098c006800470010007800904078006400470031
:10099c001040780080cf50000b0032006a004700f6
:1009ac00100078007a004000100078000080e80009
:1009bc00900078000e80e80010007800808f5000c6
:1009cc003dff3e00010037000000000064004700be
:1009dc0010407800e80047009100780080487800cb
:1009ec006a004700100078007a0040009000780000
:1009fc000e80e800100178006a8040000208780040
:100a0c000080fa00000006000800fa00000f7800d1
:100a1c000e80e800010878006400470002087800a6
:100a2c006600470003087800660047001000780055
:100a3c007a004000100078006a00400090007800b6
:100a4c001e0078000108780066004700100078004e
:100a5c007a0040001000780066004000904078005a
:100a6c0000c2b30080cf50000a003a006400470077
:100a7c0010007800104078000080fb004300dd007f
:100a8c00800078000e80e8001000780001087800e3
:100a9c004400370066004700100078007a004000e0
:100aac0010007800660040009040780000c6b3004b
:100abc0080cf50000b003a00640047001000780013
:100acc00104078000080fb006e00b9000000780038
:100adc00800078000e80e800100078000108780093
:100aec003000370066004700100078007a004000a4
:100afc0010007800660040009040780000cab300f7
:100b0c0080cf50000b003a006400470010007800c2
:100b1c00104078000080fb006e00b90000007800e7
:100b2c00800078000e80e800100078000108780042
:100b3c001c00370066004700100078007a00400067
:100b4c0010007800660040009040780000ceb300a2
:100b5c0080cf50000b003a00640047001000780072
:100b6c00104078000080fb007400b9000000780091
:100b7c00800078000e80e8001000780001087800f2
:100b8c000800370066004700100078007a0040002b
:100b9c00100078000080e800900078001e007800bb
:100bac00010878000e80e8001000780090007800b2
:100bbc0066004700100078007a00400010007800b2
:100bcc000080e80010007800808f5000090036008b
:100bdc0066004700100078007a0040001000780092
:100bec000080e800900078000e80e800100078008b
:100bfc00010878000080fa00000006000a00fa00e4
:100c0c00000f78000e80e8000108780064004700af
:100c1c000208780066004700034878006800470027
:100c2c000408780066004700104078000080fb0044
:100c3c00c1082000810f500000013200c1082000c3
:100c4c00810f500017003c0001062000810f50005e
:100c5c005f00320001062000810f500007003c00ad
:100c6c0001022000810f50002800320001042000f6
:100c7c00810f5000f90032000001370041082000bc
:100c8c00810f5000f500320081082000810f5000c8
:100c9c00e200320001082000810f5000df0032001a
:100cac00f6003700c1092000810f5000aa00320065
:100cbc00c1092000810f50000a003c0041092000ae
:100ccc00810f50004200320081092000810f50003a
:100cdc007000320001092000810f50000b0032001f
:100cec00e6003700010c2000810f5000d3003200c9
:100cfc00010e2000810f500097003200010a2000e5
:100d0c00810f500063003200dc0037000e80e800d9
:100d1c00100078001000780068004000e8004700e0
:100d2c0091007800fa804000910078008180e80002
:100d3c0091007800810f50000a00360068004700cf
:100d4c00100078007a004000100078000080e80065
:100d5c00900078000e80e800100078000108780000
:100d6c00c60037000e80e800100078009000780074
:100d7c006400470010007800104078000080fb00f1
:100d8c004300dd001e00400068014700120178009e
:100d9c00bc0007000e80e8001000780010007800fe
:100dac00e80040000e80e800100078000108780090
:100dbc006400470010007800104078000040e80004
:100dcc00e40047009100780080487800ab003700c1
:100ddc000e80e80010007800100078006e004000d3
:100dec00e800470091007800fa80400091007800fc
:100dfc008180e80091007800810f50000a003600d5
:100e0c0068004700100078007a004000100078005d
:100e1c000080e800900078000e80e8001000780058
:100e2c0001087800950037000e80e800100078006b
:100e3c0090007800640047001000780010407800a3
:100e4c000080fb004300dd001e00400068014700ed
:100e5c00120178008b0007000e80e800100078006b
:100e6c0010007800ee0040000e80e80010007800c2
:100e7c0001087800640047001000780010407800ea
:100e8c000040e800e40047009100780080487800ba
:100e9c007a0037000e80e80010007800100078000f
:100eac006e004000e800470091007800fa80400096
:100ebc00910078008180e80091007800810f50004b
:100ecc000a00360068004700100078007a004000e5
:100edc00100078000080e800900078000e80e80098
:100eec001000780001087800640037000e80e800dc
:100efc001000780090007800640047001000780023
:100f0c00104078000080fb004300dd001e00400014
:100f1c0068014700120178005a0007000e80e800b3
:100f2c001000780010007800ee0040000e80e80001
:100f3c001000780001087800640047001000780069
:100f4c00104078000040e800e40047009100780071
:100f5c0080487800490037000e80e80010007800c7
:100f6c001000780074004000e80047009100780001
:100f7c00fa804000910078008180e80091007800b0
:100f8c00810f50000a0036006800470010007800fe
:100f9c007a004000100078000080e8009000780093
:100fac000e80e8001000780001087800330037004c
:100fbc000e80e80010007800900078006400470074
:100fcc0010007800104078000080fb004300dd002a
:100fdc001e0040006801470012017800290007003c
:100fec000e80e8001000780010007800f40040003b
:100ffc000e80e800100078000108780064004700bb
:10100c0010007800104078000040e800e400470031
:10101c009100780080487800180037000e80e800b6
:10102c001000780010007800e60040000e80e80008
:10103c001000780001087800100037000e80e800de
:10104c001000780010007800ec0040000e80e800e2
:10105c001000780001087800080037000e80e800c6
:10106c001000780010007800e60040000e80e800c8
:10107c001000780001087800000000000080fa00e1
:10108c00000006000600fa00000f78000e80e80051
:10109c0001087800640047000208780064004700eb
:1010ac00100078007a004000100078009000780062
:1010bc000e80e8001000780000804000104078009e
:1010cc009e007800804878000e80e80010007800c0
:1010dc008000e8000e80e8000108780064004700fa
:1010ec00100078007a004000100078009000780022
:1010fc000e80e800100078000080400090407800de
:10110c001e0078000000e800014878000e80e8001e
:10111c00100078008000e8000e80e80001087800dc
:10112c0064004700100078007a004000100078003e
:10113c00900078000e80e8001000780000804000dd
:10114c00904078001e0078000080e800014878008c
:10115c000e80e800100078008000e8000e80e800a7
:10116c000108780064004700100078007a00400005
:10117c0010007800900078000e80e80010007800d5
:10118c0000804000904078001e0078006300400012
:10119c00014878000e80e800100078008000e8001c
:1011ac000e80e80001087800640047001000780009
:1011bc007a00400010007800900078000e80e80063
:1011cc001000780000804000904078001e007800ed
:1011dc0064004000014878000e80e80010007800a0
:1011ec008000e8000e80e8000108780064004700e9
:1011fc00100078007a004000100078009000780011
:10120c000e80e800100078000080400090407800cc
:10121c001e00780065004000014878000e80e80050
:10122c00100078008000e8000e80e80001087800cb
:10123c0064004700100078007a004000100078002d
:10124c00900078000e80e8001000780000804000cc
:10125c00904078001e00780066004000014878003d
:10126c000e80e800100078008000e8000e80e80096
:10127c000108780064004700100078007a004000f4
:10128c0010007800900078000e80e80010007800c4
:10129c0000804000904078001e00780067004000fd
:1012ac00014878000e80e800100078008000e8000b
:1012bc000e80e800010878000080fa0000000600ab
:1012cc000c00fa00e601470080097800680047002e
:1012dc00010878006a004700020878000040eb0023
:1012ec00004f78008040eb00640047000148780014
:1012fc006a004700100078007a0040001000780067
:10130c006c004000900078000e80e8000108780026
:10131c00bf0037006a004700100078007a004000d8
:10132c0010007800900078000e80e8001000780023
:10133c000080400090407800c0cfb30000cf600028
:10134c000e80e800100078008000e8000e80e800b5
:10135c00010878001e80fb006101b90000fc2f0021
:10136c00f1ff2f000200400083804800c2052000de
:10137c0003002000820f5000838f580094003e0021
:10138c00006001007e0037009100370090003700ac
:10139c008f003700750037008d0037008c00370048
:1013ac008b0037007b00370089003700880037003e
:1013bc00870037008600370085003700840037002f
:1013cc00830037008200370081003700800037002f
:1013dc007f0037007e0037007d0037007c0037002f
:1013ec007b0037007a00370079003700780037002f
:1013fc00770037007600370075003700740037002f
:10140c00730037007200370071003700700037002e
:10141c006f0037006e0037006d0037006c0037002e
:10142c006b0037006a00370069003700680037002e
:10143c00670037006600370065003700640037002e
:10144c00630037006200370061003700600037002e
:10145c005f0037005e0037005d0037005c0037002e
:10146c005b0037005a00370059003700580037002e
:10147c00570037005600370055003700540037002e
:10148c005300370049003700510037005000370037
:10149c004f0037002f0037004d0037004c0037004d
:1014ac004b0037001f003700490037004800370059
:1014bc004700370021003700450037004400370053
:1014cc00430037000c003700410037004000370064
:1014dc003f003700080037003d0037003c00370064
:1014ec003b00370004003700390037003800370064
:1014fc003700370000003700e40047000e80e8009a
:10150c006a014700120278009e41780001017800c0
:10151c00800078006600470010007800b7fd0700d7
:10152c00340037000e80e800ea0047001101780013
:10153c0061c0b300820007002e0037000e80e80067
:10154c00ea00470011017800c1c0b3007c0007001d
:10155c00280037000e80e800ea00470011017800ef
:10156c0061c0b30076000700220037000e80e8004f
:10157c00ea00470091007800980007001d00370032
:10158c000e80e800ea00470091007800fa0007009e
:10159c00180037000e80e800ea00470011017800bf
:1015ac0011c0b30066000700120037006a00470044
:1015bc00100078007a004000100078000080e800ed
:1015cc00900078000e80e8000108780009003700d0
:1015dc006a004700100078007a0040001000780084
:1015ec000080e800900078000e80e8000108780088
:1015fc000000000068004700100078009040780060
:10160c00640047001040780080cf50000b0032007f
:10161c006a004700100078007a0040001000780043
:10162c000080e800900078000e80e8001000780040
:10163c00808f500037ff3e00010037000000000093
:10164c006400470010407800e800470091007800e3
:10165c00804878006a004700100078007a0040004b
:10166c00900078000e80e800100178006c8040003b
:10167c00020878000080fa00000006000400fa005e
:10168c00000f78000e80e800010878001e0078003a
:10169c00100078000080e8008e80e800910078004f
:1016ac00fa804000910078008180e8009100780079
:1016bc00810f5000200031000e80e80010007800ef
:1016cc007a00400010007800900078001e0078002e
:1016dc0010007800008040009040780000c8b300f3
:1016ec0080cf500014003a000e80e8001000780003
:1016fc007a00400010007800900078001e007800fe
:10170c00100078000000e8000080400010407800d5
:10171c000004e00008003a000e80e8001000780099
:10172c007a004000100078000080e80090007800fb
:10173c001e007800010878000080fa000000060006
:10174c000600fa00000f78000e80e80001487800cf
:10175c0064004700020878001e00780090007800b2
